:020000040800F2
:1000000000060020E1010008190E00081D0E00087E
:10001000750E00081D0E0008490E0008E3010008D7
:10002000E3010008E3010008E3010008452100089E
:10003000E3010008E3010008E3010008E301000810
:10004000E3010008E3010008E3010008E301000800
:10005000E3010008E30100082532000851320008DE
:100060007D320008A9320008D5320008E3010008FB
:10007000E3010008E3010008E3010008E3010008D0
:10008000E3010008E3010008E3010008E3010008C0
:10009000E3010008E3010008E30100080133000860
:1000A000E3010008E3010008E3010008E3010008A0
:1000B00099300008E3010008E3010008E3010008AB
:1000C000E3010008E3010008E3010008E301000880
:1000D000E3010008E3010008E3010008E301000870
:1000E00069330008E3010008E3010008E3010008A8
:1000F000E3010008E3010008E3010008E301000850
:10010000E3010008E3010008E3010008E30100083F
:10011000E3010008E3010008E3010008E30100082F
:10012000E3010008E3010008E3010008E30100081F
:10013000E3010008E3010008E3010008E30100080F
:10014000E3010008E3010008E30100088928000832
:10015000E3010008E3010008E3010008E3010008EF
:10016000E3010008E3010008E3010008E3010008DF
:10017000E3010008E3010008E3010008E3010008CF
:10018000E3010008E3010008E3010008E3010008BF
:10019000E3010008E3010008E3010008E3010008AF
:1001A000E3010008E3010008E3010008E30100089F
:1001B000E3010008E3010008E3010008E30100088F
:1001C000E3010008E3010008E3010008E30100087F
:1001D000E3010008E3010008E3010008E30100086F
:1001E00002E000F000F8FEE772B6394880F30888B4
:1001F000384880F3098838484EF60851CEF200019D
:10020000086040F20000CCF200004EF63471CEF2ED
:1002100000010860BFF34F8FBFF36F8F40F2000003
:10022000C0F2F0004EF68851CEF200010860BFF334
:100230004F8FBFF36F8F4FF00000E1EE100A4EF6C4
:100240003C71CEF200010860062080F31488BFF3F1
:100250006F8F01F0D5FF02F07BFE4FF055301F4944
:100260001B4A91423CBF41F8040BFAE71C49194A6A
:1002700091423CBF41F8040BFAE71A491A4A1B4B5A
:100280009A423EBF51F8040B42F8040BF8E70020F5
:100290001749184A91423CBF41F8040BFAE701F0B4
:1002A000B3FF02F0B1FE144C144DAC4203DA54F823
:1002B000041B8847F9E700F041F8114C114DAC429E
:1002C00003DA54F8041B8847F9E701F09BBF0000EC
:1002D000000600200022002000000008000000208E
:1002E0000006002078370008002200202822002085
:1002F00028220020942D0020E0010008E0010008E1
:10030000E0010008E00100082DE9F04F2DED108A12
:10031000C1F80CD0C3689D46BDEC108ABDE8F08FD3
:10032000002383F311882846A047002001F036FB04
:10033000FEE701F0B7FA00DFFEE700001A4B7A2271
:1003400070B500241A700F225C709C70DC701C71F8
:100350005C719C71DC711C725C729A72DC7201F0CF
:10036000C3FE064601F0E8FE054650B90F4B9E421B
:1003700017D001339E4241F2883412BF0546002453
:100380000125002001F0BAFE0DB100F059F800F08F
:1003900017FD00F09FFB204600F0B0F800F050F889
:1003A000F9E70446EDE700BF28220020010007B06E
:1003B00008B500F061FBA0F120035842584108BD88
:1003C00007B5054B02211B88ADF8043001A800F0E9
:1003D00071FB03B05DF804FB4C34000810B520231A
:1003E00083F311881248C3680BB101F073FB00233B
:1003F000104A0F484FF47A7101F01AFB002383F37F
:1004000011880D4C236813B12368013B2360636896
:1004100013B16368013B6360084B1B7833B96368B1
:1004200023B9022000F03AFC3223636010BD00BF04
:1004300034220020DD030008502300204822002041
:1004400010B5254B254953F8042F013200D110BDBA
:100450008B42F8D1224C234B22689A423AD9224B44
:100460009B6803F1006303F580339A4232D2002087
:1004700000F04AFB1D4B0220187000F007FC1C4BDB
:100480001A6C00221A64196E1A66196E596C5A6435
:10049000596E5A665A6E5A6942F080025A615A6918
:1004A00022F080025A615A691A6942F000521A61B8
:1004B0001A6922F000521A611B6972B60D4A0E4B7E
:1004C00013601B682268202181F311889D4683F305
:1004D0000888104710BD00BFFCFF00081C00010881
:1004E00004000108FFFF0008282200204822002005
:1004F0000038024008ED00E0000001082DE9F04F4F
:1005000099B0B94D00902022FF2110A8AC6800F0EE
:10051000F9FBB64A01951378A3B9B5480121C36028
:100520001170202383F31188C3680BB101F0D2FA54
:100530000023B04AAE484FF47A7101F079FA0023F3
:1005400083F31188009BAC4A03B11360AB4B009D51
:10055000029300261E705660B2463746B14601200F
:1005600000F094FB002D00F02582A34B1B68002BAC
:1005700040F0208219B0BDE8F08F0220FFF718FF8D
:10058000002840F01082009B002E08BF1D469C4BA7
:1005900002211B88ADF82C300BA800F08BFADEE7A7
:1005A0004FF47A7000F068FAB0F10008EBDB02203B
:1005B000FFF7FEFE0028E6D008F1FF38B8F1040F7F
:1005C00000F2F381DFE808F0031E2124270018A8B9
:1005D000052340F8343D042100F06CFA012303FAAE
:1005E00008F848EA0A0A5FFA8AFA4FF0000900F0B0
:1005F000DDFB27B10AF00B030B2B08BF0025FFF72B
:10060000DFFEACE704217848E6E704217D48E3E714
:1006100004217D48E0E74FF01C09484600F076FAD7
:1006200009F104090B9004210BA800F043FAB9F179
:100630002C0FF2D1D2E7002FA5D00AF00B030B2B21
:10064000A1D10220FFF7B4FE804600289BD00120F4
:100650006A4E00F059FA0220307000F017FB0027B4
:100660005FFA87FB584600F05FFA054688B15846A6
:1006700000F06AFA01370028F2D146460025634BA4
:1006800002211B88ADF82C300BA800F013FA474666
:1006900065E701230220337000F0EEFA2C46019B3F
:1006A0009B689C4206D2204600F030FA0130E4D12B
:1006B0000434F4E7029B00241C704F4B46465C60F8
:1006C0004746254693E7002F3FF45DAF0AF00B0342
:1006D0000B2B7FF458AF029B0220187000F0D6FA63
:1006E000322000F0C9F9B0F1000BFFF64CAF1BF05F
:1006F00003087FF448AF019B996804EB0B028A4220
:100700003FF641AFBBF5807F3FF63DAF404A0392D5
:10071000D8450FDA4FF47A7000F0AEF904900499DE
:100720000029FFF630AF039A049908F8021008F187
:100730000108ECE7C820FFF73BFE804600283FF4A5
:1007400022AF1F2C11D8C4F120075F4528BF5F4698
:1007500010AB24F003003A462D49184400F0A8FAE3
:100760003A46FF212A4800F0CDFA4FEAAB03DAB24D
:1007700027490393204600F0CDFA074600283FF4AE
:100780007EAF039B04EB830431E70220FFF710FEEA
:1007900000283FF4F8AE00F0FDF900283FF4F3AE76
:1007A0004FF000084346019A9268904532D2B8F162
:1007B0001F0F12D8109A01320FD028F0030218A987
:1007C0000A4452F8202C0B92184604220BA900F080
:1007D00065FB08F104080346E5E74046039300F093
:1007E00095F9039B0B90EFE7282200204C23002073
:1007F00034220020DD03000850230020482200207E
:100800004E3400082C2200203022002050340008F2
:100810004C22002018A8042140F84C3D00F04AF971
:10082000E5E618A8002340F8343D642100F038F9CB
:1008300000287FF4A8AE0220FFF7BAFD00283FF49D
:10084000A2AE0B9800F092F918AB43F8480D0421C2
:100850001846E3E718A8002340F8343D642100F06F
:100860001FF900287FF48FAE0220FFF7A1FD0028BA
:100870003FF489AE0B9800F087F918AB43F8440DAC
:10088000E5E70220FFF794FD00283FF47CAE00F07E
:1008900091F918AB43F8400DD9E70220FFF788FD26
:1008A00000283FF470AE0BA9142000F089F98046AF
:1008B00018A8042140F83C8D00F0FCF841460BA834
:1008C000ACE7322000F0D8F8B0F10008FFF65BAEDC
:1008D00018F0030F7FF457AE019A926808EB0903F2
:1008E00093423FF650AE0220FFF762FD00283FF42E
:1008F0004AAE28F00308C844C1453FF478AE4846E4
:1009000000F004F904210A900AA800F0D3F809F1D4
:100910000409F1E74FF47A70FFF74AFD00283FF42D
:1009200032AE00F037F9002842D0109B01330BD0D3
:10093000082210A9002000F0EDF9002838D020226C
:10094000FF2110A800F0DEF9FFF73AFD364801F06C
:100950002BF80FE6002F3FF416AE0AF00B030B2B1B
:100960007FF411AE18A8002340F8343D642100F054
:1009700097F8804600287FF406AE0220FFF718FDA6
:1009800000283FF400AE0390FFF71AFD41F28830D3
:1009900001F00AF80B9800F03DFA00F007FA039B0B
:1009A00045461F46DBE5074621E64FF00009EAE52C
:1009B000B84664E6002000F05FF80490049B002B2A
:1009C000FFF6D0AD012000F057F9049B213B122B1C
:1009D0003FF6C5AD01A252F823F000BF7B05000829
:1009E000A1050008370600085F0500085F0500083C
:1009F0005F050008C7060008C30800088B07000849
:100A00002308000855080008830800085F0500084F
:100A10009B0800085F05000815090008EF0500089D
:100A20005F05000855090008A086010070B50F4B4E
:100A30000C4619780131C9B2012906460FD80C4875
:100A400003681D6A4FF47A73534331462246A84720
:100A5000844204D1074B00221A70012070BD4FF46C
:100A6000FA7000F0A1FF002070BD00BF002200203E
:100A7000C02500208423002007B502AB002203F824
:100A8000012D012102461846FFF7D0FF20B19DF845
:100A9000070003B05DF804FB4FF0FF30F9E70000FA
:100AA0000A4608B50421FFF7C1FF80F00100C0B27B
:100AB000404208BD30B4054C2368DD69044B0A464A
:100AC000AC460146204630BC604700BFC025002030
:100AD000A086010070B501F00BFA094C094E208088
:100AE000002530682388834208D901F0FBF9336878
:100AF00005440133B5F5803F3360F2D370BD00BFCC
:100B0000862300205823002001F0A0BA00F10060E5
:100B100000F580300068704700F10060920000F539
:100B2000803001F02BBA0000054B1A68054B1B887A
:100B30009B1A834202D9104401F0D4B900207047B7
:100B4000582300208623002038B5074D0446286826
:100B5000204401F0CFF928B928682044BDE8384086
:100B600001F0E0B938BD00BF5823002010F00303A6
:100B700008D1B0F5047F05D200F10050A0F508407F
:100B80000068704700207047014BC058704700BF95
:100B9000107AFF1F064991F8243033B10023082250
:100BA000086A81F82430FFF7B7BF0120704700BF03
:100BB0005C230020014B1868704700BF002004E050
:100BC00070B52A4B1C68C4F30B03240C63B140F2CC
:100BD0001342934231D040F2194293422FD040F257
:100BE000214293422DD10323214A0C2505FB0323E7
:100BF0005D6893F9082042F201039C4224D0B4F5C9
:100C0000805F23D041F201039C4221D041F20303D3
:100C10009C421FD041F207039C4208BF3122441E70
:100C20000C44013D0B46A3421ED215F9016F581C1E
:100C300096B1034600F8016CF5E70123D4E70223DF
:100C4000D2E73F220B4DD6E73322E3E74122E1E72B
:100C50005A22E4E75922E2E72C2584421D7001D98B
:100C6000981C5A70401A70BD1846FBE7002004E03B
:100C70006034000854340008022802BF024B4FF4CD
:100C800000129A61704700BF00040240022802BFB0
:100C9000014B20229A61704700040240022801BFE4
:100CA000024A536983F020035361704700040240F5
:100CB00010B50023934203D0CC5CC4540133F9E750
:100CC00010BD000030B5441E14F9010F0B4660B191
:100CD00093F90050854201F1010106D11AB993F947
:100CE0000020801A30BD013AEEE7002AF7D1104605
:100CF00030BD000002460346981A13F9011B002973
:100D0000FAD1704702440346934202D003F8011B14
:100D1000FAE770472DE9F047234C94F82430054654
:100D20008846174683BB2E46DFF87C90C7B394F8FD
:100D300024302BB92022FF2148462662FFF7E2FF2C
:100D400094F82400C0F10805BD4228BF3D465FFA73
:100D500085FAAD0041462A4604EB8000FFF7A8FF64
:100D600094F82430A7EB0A079A445FFA8AFABAF19A
:100D7000080F2E44A844FFB284F824A0D6D1FFF770
:100D800009FF0028D2D108E0266A06EB8306B042AC
:100D9000CAD0FFF7FFFE0028C5D10020BDE8F087CC
:100DA0000120BDE8F08700BF5C230020024B1A78C9
:100DB000024B1A70704700BF8423002000220020DD
:100DC00038B5104D104C284600F004F9214628464D
:100DD00000F02CF924680D48626DD2F8043843F015
:100DE0000203C2F8043800F0DFFD0949204600F094
:100DF00029FA626DD2F8043823F00203C2F80438ED
:100E000038BD00BFC02500205435000840420F0007
:100E10007C35000870470000FEE7000000B59BB07D
:100E2000EFF3098168226846FFF742FFEFF305837D
:100E3000044B9A6BDA6A9A6A9A6A9A6A9A6A9A6A06
:100E40009B6AFEE700ED00E000B59BB0EFF309817F
:100E500068226846FFF72CFFEFF30583044B9A6B7B
:100E60009A6A9A6A9A6A9A6A9A6A9B6AFEE700BFC5
:100E700000ED00E000B59BB0EFF309816822684601
:100E8000FFF716FFEFF30583034B5A6B9A6A9A6AD2
:100E90009A6A9A6A9B6AFEE700ED00E030B5084D59
:100EA0000A4491420BD011F8013B09245840013CFF
:100EB000F7D040F300032B4083EA5000F7E730BD42
:100EC0002083B8ED002304491A465A50C818083345
:100ED000802B4260F9D17047882300200268436864
:100EE0001143016003B118477047000013B5446B0C
:100EF000D4F894341A681178042915D1217C022978
:100F000012D11979128901238B4013420CD101A906
:100F100004F14C0001F020FFD4F89444019B2179A6
:100F20000246206800F0DAF902B010BD143001F07A
:100F3000A3BE00004FF0FF33143001F09DBE00004F
:100F40004C3001F075BF00004FF0FF334C3001F022
:100F50006FBF0000143001F071BE00004FF0FF3190
:100F6000143001F06BBE00004C3001F041BF0000B6
:100F70004FF0FF324C3001F03BBF0000D0F894241A
:100F800038B5136819780429054601D0012038BD09
:100F9000017C0229FAD112795C8901209040044039
:100FA000F4D105F1140001F003FE02460028EDD053
:100FB000D5F894544FF480732868697900F07CF96F
:100FC000204638BD406BFFF7D9BF000000207047B6
:100FD000704700007FB5124B0360002343608360BD
:100FE000C360012502260F4B05740446029001934D
:100FF00000F18402294600964FF48073143001F00A
:10100000B3FD094B0193029400964FF4807304F5ED
:101010002372294604F14C0001F07AFE04B070BD41
:10102000B0340008C50F0008ED0E00080B68202240
:1010300082F311880A7903EB820290614A790932BE
:1010400043F822008A7912B103EB820398610223EC
:101050000374C0F89414002383F3118870470000D0
:1010600038B5037F044613B190F85430ABB9201D56
:1010700001250221FFF732FF04F1140025776FF0FC
:10108000010100F0B9FC84F8545004F14C006FF0F9
:101090000101BDE8384000F0AFBC38BD10B50121FA
:1010A00004460430FFF71AFF0023237784F85430F6
:1010B00010BD000038B504460025143001F06CFD69
:1010C00004F14C00257701F03BFE201D84F85450BC
:1010D0000121FFF703FF2046BDE83840FFF74EBF70
:1010E00090F8443003F06003202B19D190F845208C
:1010F000212A0AD0222A4FF000030ED0202A0FD135
:10110000084A82630722C26304E0064B8363072315
:10111000C36300230364012070478363C363F9E75B
:101120000020704701220020D0F8943437B51A68A7
:101130001178042904461AD1017C022917D11979A2
:10114000128901238B40134211D100F14C0528462E
:1011500001F0B6FE58B101A9284601F0FDFDD4F812
:101160009444019B21790246206800F0B7F803B04F
:1011700030BD000000EB8103F7B59C6905460E46C3
:10118000F4B1202383F3118805EB8607201D082185
:10119000FFF7A4FEFB685B691B684C3413B1204663
:1011A00001F0E8FD01A9204601F0D6FD024648B154
:1011B000019B3146284600F091F8002383F3118803
:1011C00003B0F0BDFB685A691268002AF5D01B8A8B
:1011D000013B1340F1D105F14402EAE7093138B58A
:1011E00050F82140DCB1202383F31188D4F89424F3
:1011F0001368527903EB8203DB689B695D6845B134
:1012000004216018FFF76AFE294604F1140001F07A
:10121000D9FC2046FFF7B2FE002383F3118838BDC6
:101220007047000001F082B801230370002343607F
:10123000C36183620362C3624362036303814381C8
:101240007047000038B50446202383F31188002539
:101250004160C56005614561856101F077F8022351
:10126000237085F3118838BD70B500EB8103054606
:101270005069DA600E46144618B110220021FFF7BB
:1012800041FDA06918B110220021FFF73BFD314656
:101290002846BDE8704001F023B90000028902F041
:1012A00001020281428902F00102428100220261B0
:1012B0004261826101F0A8B9F0B400EB8104478972
:1012C000E4680125A4698D403D43458123600023E6
:1012D000A2606360F0BC01F0C3B90000F0B400EBA1
:1012E00081040789E468012564698D403D430581D7
:1012F00023600023A2606360F0BC01F03DBA0000EF
:1013000070B50223002504460370A0F84C5080F805
:101310004E5080F84F5005814581C560056145619B
:10132000856180F8345001F077F863681B6823B159
:1013300029462046BDE87040184770BD037880F804
:1013400050300523037043681B6810B504460BB189
:101350000421984700232381638110BD436890F8DE
:1013600050201B6802700BB1052118477047000020
:1013700090F8343070B5044613B1002380F834304F
:1013800004F14402204601F061F963689B6863BB85
:1013900094F8445015F0600615D194F8453005F0E6
:1013A0007F0545EA032540F202339D4200F00E819D
:1013B0005BD8022D00F0DC803FD8002D00F0878044
:1013C000012D00F0CF800021204601F099FB002183
:1013D000204601F08BFB63681B6813B10621204691
:1013E0009847062384F8343070BD2046984700287B
:1013F000CED094F84B2094F84A3043EA0223E26BB3
:10140000934238BFE36394F94430E56B002B4FF00F
:10141000200380F2FD80002D00F0EC80092284F88A
:10142000342083F311880021E36BA26B2046FFF781
:1014300055FF002383F3118870BDB5F5817F00F05F
:10144000B180B5F5407F49D0B5F5807FBBD194F828
:101450004630012BB7D1B4F84C3023F00203A4F886
:101460004C30A663E6632664C3E740F201639D4205
:101470001ED8B5F5C06F3BD2B5F5A06FA3D1B4F8B7
:101480004430B3F5A06F0ED194F8463084F84E3056
:10149000204601F019F863681B6813B1012120464A
:1014A0009847032323700023A363E3632364A0E727
:1014B000B5F5106F32D040F602439D4252D0B5F5DB
:1014C000006F80D104F14F03A363012324E004F1F2
:1014D0004C03A3630223E36325648AE794F8463050
:1014E000012B7FF470AFB4F84C3043F00203B6E741
:1014F00094F84920616894F848304D6894F8471092
:1015000043EA0223204694F84620A84700283FF4E7
:101510005AAF4368A3630368E363A4E72378042B0B
:1015200010D1202383F311882046FFF7B7FE86F3FE
:101530001188636884F84F601B68032121700BB128
:101540002046984794F84630002BACD084F84F30B2
:101550000423237063681B68002BA4D0022120465B
:101560009847A0E7374BA3630223E36300239DE77B
:1015700094F8481011F0800F204601F00F010ED0B2
:1015800001F056F8012806D002287FF41CAF2E4B3C
:10159000A363E06367E72D4BA363E56363E701F0B3
:1015A00039F8EFE794F84630002B7FF40CAF94F84D
:1015B000483013F00F013FF476AF1A06204602D5EB
:1015C00001F0B2FA6FE701F0A5FA6CE794F8463043
:1015D000002B7FF4F8AE94F8483013F00F013FF47D
:1015E00062AF1B06204602D501F08AFA5BE701F0E4
:1015F0007DFA58E7142284F8342083F311882B46AF
:101600002A4629462046FFF757FE85F3118870BD0C
:101610005DB1152284F8342083F311880021E36B37
:10162000A26B2046FFF748FE03E70B2284F8342024
:1016300083F311882B462A4629462046FFF74EFEA3
:10164000E3E700BFE0340008D8340008DC340008C9
:1016500038B590F834300446152B29D8DFE803F06C
:101660003E28282828283E28280B293928282828D9
:10167000282828283E3E90F84B1090F84A20C36B4B
:1016800042EA01229A4214D9C268128AB3FBF2F5E7
:1016900002FB15356DB9202383F311882B462A46AA
:1016A0002946FFF71BFE85F311880A2384F834309E
:1016B00038BD142384F83430202383F311880023A9
:1016C0001A4619462046FFF7F7FD002383F31188D9
:1016D00038BD036C03B198470023E7E7002101F010
:1016E0000FFA0021204601F001FA63681B6813B16C
:1016F0000621204698470623D8E7000090F83420BA
:10170000152A38B5044622D80123934040F6416299
:1017100013421DD113F480150FD19B0217D50B2353
:1017200080F83430202383F311882B462A4629463B
:10173000FFF7D4FD85F3118838BDC3689B695B68EA
:101740002BB9036C03B19847002384F8343038BDBB
:10175000002101F0D5F90021204601F0C7F96368A6
:101760001B6813B10621204698470623EDE70000C9
:10177000024B00221B605B609A60704708240020C7
:10178000002303748268054B1B6899689142FBD261
:101790005A68036042601060586070470824002057
:1017A00008B5202383F31188037C032B05D0042B79
:1017B0000DD02BB983F3118808BD436900221A604C
:1017C0004FF0FF334361FFF7DBFF0023F2E790E8C0
:1017D0000C001A6002685360F2E7000000230374F3
:1017E0008268054B1B6899689142FBD85A68036070
:1017F000426010605860704708240020054B19694A
:101800000874186802681A60536018610123037431
:10181000FEF77ABD0824002030B54B1C87B0054682
:101820000A4C10D023690A4A01A800F001F92846A1
:10183000FFF7E4FF049B13B101A800F04BF9236903
:10184000586907B030BDFFF7D9FFF8E7082400203A
:10185000A117000838B50C4D41612B6981689A6861
:101860009142044603D8BDE83840FFF789BF1846C7
:10187000FFF7B4FF01232C61014623742046BDE825
:101880003840FEF741BD00BF08240020044B1A6811
:101890001B6990689B68984294BF002001207047A4
:1018A0000824002010B5084C236820691A682260BB
:1018B0005460012223611A74FFF790FF01462069EA
:1018C000BDE81040FEF720BD08240020FEE7000020
:1018D00010B50C4CFFF74CFF00F09CF880220A4931
:1018E000204600F021F8012344F8180C037400F09E
:1018F00039FC002383F3118862B60448BDE8104028
:1019000000F034B830240020E4340008EC3400083F
:1019100000F01AB9034B59685A68521A9042FBD822
:10192000704700BF001000E08260022202740022B3
:10193000427470478368A3F17C0243F80C2C02695F
:1019400043F83C2C426943F8382C074A43F81C2CD6
:10195000C26843F8102C022203F8082C002203F876
:10196000072CA3F1180070472103000810B52023AD
:1019700083F31188FFF7DEFF00210446FFF76AFFBB
:10198000002383F31188204610BD0000024B1B6921
:1019900058610F20FFF732BF08240020202383F373
:1019A0001188FFF7F3BF000008B50146202383F339
:1019B00011880820FFF730FF002383F3118808BD4A
:1019C00049B1064B42681B6918605A601360436056
:1019D0000420FFF721BF4FF0FF307047082400209C
:1019E0000368984206D01A68026050605961184630
:1019F000FFF7C6BE7047000038B504460D462068A4
:101A0000844200D138BD036823605C604561FFF704
:101A1000B7FEF4E7054B03F114025A619A614FF0E7
:101A2000FF32DA6100221A62704700BF08240020EA
:101A3000F8B5274F0361C2600D46044601F074FA01
:101A40003B46022D53F8142F294638BF02219A42F3
:101A50003E461D460AD138627C61BC610844226062
:101A60006260A160BDE8F84001F04CBAD7F820E010
:101A7000A0EB0E035F181FD300279068834217D88E
:101A8000376AAA421F44376201D0C01A9060736956
:101A90009A68914219D85A682360626014605C6049
:101AA000A1609868411A99604FF0FF33F361F8BD67
:101AB00097601B1A1268E0E793689F4203D20EEB0F
:101AC000070001F02DFA3946E1E7891A1B68DFE7C4
:101AD0000824002038B51B4B01685A6990421D4606
:101AE00003F114020CD04468216003680021934282
:101AF0005C60C16025D09A6881680A449A6038BDEC
:101B000059614A605B6900219342C16003D1BDE81D
:101B1000384001F0FFB99A6881680A449A602C6ADB
:101B200001F002FA6A699268001B824209D9111A0F
:101B3000012998BF821C286ABDE83840104401F092
:101B4000EFB938BD082400202DE9F84F204C0027BC
:101B5000656904F11406B84601F0E6F9236AA0EBC2
:101B6000030AAB6853451DD84FF02009236AAA68C1
:101B7000D5F80CB013442362AB68AAEB030A2B68B8
:101B8000B3425E606361EF6001D101F0C3F988F395
:101B900011882869D84789F311886569AB689A4527
:101BA000E4D2D9E76369B34210D020629A68A2EB0D
:101BB0000A029A60226AAB68821A9B1A022B2CBF17
:101BC000C0180230BDE8F84F01F0AAB9BDE8F88F9F
:101BD0000824002000207047FEE700007047000046
:101BE0004FF0FF3070470000022906D0032906D0CD
:101BF0000129064818BF0020704705487047032A8E
:101C00009ABF044800EBC20000207047D835000896
:101C10008C3500080822002070B59AB001AD064648
:101C200008462946144600F095F82846FFF762F862
:101C3000C0B2431C5B0086E8180023700323637066
:101C4000002302341946DAB2904204F1020401D8AA
:101C50001AB070BDEA5C04F8022C04F8011C0133D0
:101C6000F1E7000008B5202383F311880348FFF74C
:101C70005BFA002383F3118808BD00BFC025002054
:101C800010B50446052916D8DFE801F0161503162D
:101C9000161D202383F311880E4A0121FFF7E4FA71
:101CA00020460D4A0221FFF7DFFA0C48FFF702FA3F
:101CB000002383F3118810BD202383F31188074884
:101CC000FFF7CEF9F4E7202383F311880348FFF7E9
:101CD000E5F9EDE70C35000830350008C025002097
:101CE00038B50C4D0C4C0D492A4604F10800FFF79D
:101CF00093FF05F1CA0204F110000949FFF78CFFB8
:101D000005F5CA7204F118000649BDE83840FFF72E
:101D100083BF00BF882A0020082200205C3500080D
:101D2000663500087135000870B5044608460D4652
:101D3000FEF7E0FFC6B22046013403780BB918461F
:101D400070BD32462946FEF7BDFF0028F3D10120C1
:101D500070BD00002DE9F84F05460C46FEF7CAFF9E
:101D60002A49C6B22846FFF7DFFF08B10136F6B2AE
:101D700027492846FFF7D8FF08B11036F6B2632E80
:101D80000DD8DFF88890DFF888A0224FDFF88CB0FC
:101D9000DFF88C802E7846B92670BDE8F88F29468A
:101DA0002046BDE8F84F01F049BB252E29D1072276
:101DB00049462846FEF786FF40B9D8F80030236030
:101DC000D8F80430636007350834E3E70822514649
:101DD0002846FEF777FFA0B90F4BA21C13F8011F8E
:101DE00009095B45C95D02F8021C197801F00F0171
:101DF00002F10202C95D02F8031CEFD11834083564
:101E0000C8E7267001350134C4E700BFF835000883
:101E100071350008093600080F7AFF1F1B7AFF1F73
:101E200000360008BFF34F8F024AD368DB03FCD4AF
:101E3000704700BF003C024008B5094B1B7873B9DE
:101E4000FFF7F0FF074B1A69002ABFBF064A5A6026
:101E500002F188325A601A6822F480621A6008BD62
:101E6000E62C0020003C02402301674508B50B4BDF
:101E70001B7893B9FFF7D6FF094B1A6942F000426D
:101E80001A611A6842F480521A601A6822F4805269
:101E90001A601A6842F480621A6008BDE62C0020BD
:101EA000003C02400B2870B513D80B4A0B4C13783A
:101EB00063B90B4E4FF0006144F8231056F82350DD
:101EC00001330C2B2944F7D10123137054F820005F
:101ED00070BD002070BD00BF182D0020E82C002030
:101EE0001C360008014B53F8200070471C360008D0
:101EF0000C2070470B2810B5044601D9002010BDF6
:101F0000FFF7D0FF064B53F824301844C21A0BB920
:101F1000012010BD12680132F0D1043BF6E700BF8A
:101F20001C3600080B2810B5044621D8FFF77AFFAD
:101F3000FFF782FF0F4AF323D360C300DBB243F401
:101F4000007343F002031361136943F48033136198
:101F5000FFF768FFFFF7A6FF074B53F8241000F0C8
:101F6000DDF8FFF783FF2046BDE81040FFF7C2BF52
:101F7000002010BD003C02401C3600082DE9F8434B
:101F800012F00103154640D18218B2F1016F3CD224
:101F90002C4B1B6813F0010337D02B4CFFF74CFF81
:101FA000F323E360FFF73EFF40F20127032D01D941
:101FB000830713D0244C0F46401A40F20118EB1B44
:101FC0000B44012B00EB0706236924D823F00103FF
:101FD0002361FFF74BFF0120BDE8F883236923F459
:101FE0004073236123693B43236151F8046B06600E
:101FF000BFF34F8FFFF716FF03689E4208D0236997
:1020000023F001032361FFF731FF0020BDE8F883CF
:10201000043D0430CAE723F440732361236943EA93
:1020200008032361B94637F8023B3380BFF34F8F73
:10203000FFF7F8FE3688B9F80030B6B2B342BED02A
:10204000DDE700BF00380240003C0240084908B507
:102050000B7828B153B9FFF7EFFE01230B7008BDD1
:1020600023B1BDE808400870FFF700BF08BD00BFFE
:10207000E62C002010B50244064B0439D2B290423F
:1020800000D110BD441C00B253F8200041F8040FE9
:10209000E0B2F4E750280040104B30B51C6F240428
:1020A00007D41C6F44F400741C671C6F44F4004494
:1020B0001C670B4C236843F4807323600244094B74
:1020C0000439D2B2904200D130BD441C00B251F864
:1020D000045F43F82050E0B2F4E700BF003802404C
:1020E000007000405028004007B5012201A90020DF
:1020F000FFF7C0FF019803B05DF804FB13B5044679
:10210000FFF7F2FFA04206D002A9012241F8044DD8
:102110000020FFF7C1FF02B010BD000070470000B3
:10212000034B1B689B0042BF024B01221A70704791
:1021300074380240192D0020014B1878704700BFF9
:10214000192D0020EFF3098305494A6822F00102A6
:102150004A60683383F30988002383F3118870474A
:1021600030EF00E0202080F3118862B60B4B0C4A60
:10217000D96821F4E0610904090C0A430949DA60CD
:10218000CA6842F08072CA6007490A6842F00102D8
:102190000A601022DA7783F82200704700ED00E031
:1021A0000003FA05F0ED00E0001000E010B5202378
:1021B00083F311880E4B5B6813F4006314D0F1EEC7
:1021C000103AEFF30984683C4FF08073E361094BE8
:1021D000DB68236684F30988FFF758FB10B1064BD0
:1021E000A36110BD054BFBE783F3118810BD00BF51
:1021F00000ED00E030EF00E0330300083603000894
:1022000070470000FEE70000084A094B09498B426D
:1022100004D3094A0021934205D3704752F8040FB2
:1022200043F8040BF3E743F8041BF4E79C3700087A
:10223000942D0020942D0020942D0020836D70B5E6
:10224000446D9E6800214FF0FF354A01A31801310B
:10225000D3F800090028BEBFD3F8000940F0804041
:10226000C3F80009D3F8000B0028BEBFD3F8000B59
:1022700040F08040C3F8000BA3188E42C3F8085901
:10228000C3F8085BE1D24FF00113C4F81C3870BDED
:10229000890141F02001016103699B06FCD41220F1
:1022A000FFF738BB204B03EB80022DE9F047D2F853
:1022B0000CE05D6DDEF81420461CD2F800C005EB82
:1022C000063605EB4018516861450BD3D5F8342824
:1022D000012303FA00F022EA0000C5F8340818468A
:1022E000BDE8F087BEF81040ACEB0103A34228BF65
:1022F0002346D8F81849A4B2B3EB840F10D89468D9
:102300001F46A4F1040959F804AFC6F800A0042F31
:1023100001D9043FF7E71C440B4494605360D2E7B3
:102320000020BDE8F08700BF1C2D002010B5054C33
:102330002046FEF779FF4FF0A0436365024BA3658B
:1023400010BD00BF1C2D0020703600080378012B43
:1023500070B5054650D12A4B446D98421BD1294B8C
:102360005A6B42F080025A635A6D42F080025A65FD
:102370005A6D5A6942F080025A615A6922F080020D
:102380005A610E2143205B6900F0D8FB1E4BE360CD
:102390001E4BC4F800380023C4F8003EC02323605D
:1023A0006E6D4FF40413A3633369002BFCDA012331
:1023B00033610C20FFF7AEFA3369DB07FCD412203F
:1023C000FFF7A8FA3369002BFCDA0026A66028463E
:1023D000FFF734FF6B68C4F81068DB68C4F8146852
:1023E000C4F81C684BB90A4BA3614FF0FF3363611B
:1023F000A36843F00103A36070BD064BF4E700BF80
:102400001C2D002000380240401400400300200230
:10241000003C30C0083C30C0F8B5446D0546002192
:102420002046FFF735FFA96D00234FF001128F689A
:10243000C4F834384FF00066C4F81C284FF0FF3061
:1024400004EB431201339F42C2F80069C2F8006BEB
:10245000C2F80809C2F8080BF2D20B686A6DEB6586
:10246000636210231361166916F01006FBD1122067
:10247000FFF750FAD4F8003823F4FE63C4F80038AC
:10248000A36943F4402343F01003A3610923C4F874
:102490001038C4F814380A4BEB604FF0C043C4F84E
:1024A000103B084BC4F8003BC4F81069C4F800396D
:1024B000EB6D03F1100243F48013EA65A362F8BDEB
:1024C0004C36000840800010426D90F84E10D2F853
:1024D000003823F4FE6343EA0113C2F80038704762
:1024E0002DE9F0410EB200EB86080D46D8F80C102D
:1024F0000F6807F00303022B50D0032B50D03D4A46
:102500003D4F012B18BF1746446D4FEA451E04EBA3
:102510000E030022C3F8102B8A6905F1100C002A63
:1025200040D04A8A05F158035B013A43E250012347
:10253000D4F81C2803FA0CF31343A6444A69C4F8E0
:102540001C380023CEF8103905F13F03002A39D09A
:102550000A8A898B9208012988BF4A43C16D04EB1E
:102560008303561841EA0242C66529465A6020464E
:10257000FFF78EFED8F80C301B8A43EA85531F43C1
:1025800005F148035B01E7500123D4F81C2803FA46
:1025900005F51543C4F81C58BDE8F081174FB3E7A3
:1025A000174FB1E704EB4613D3F8002B22F4004297
:1025B000C3F8002BD4F81C28012303FA0CF322EAF9
:1025C0000303BAE704EB83030E4A5A6004EB461692
:1025D00029462046FFF75CFED6F8003923F4004375
:1025E000C6F80039D4F81C38012202FA05F523EAAE
:1025F0000505CFE70080001000800410008008105F
:1026000000800C1000040002826D1268C265FFF7A2
:1026100015BE00005831436D49015B5813F400406A
:1026200004D013F4001F14BF0120022070470000E3
:102630004831436D49015B5813F4004004D013F452
:10264000001F14BF012002207047000000EB810131
:10265000CB68196A0B6813604B68536070470000C1
:1026600000EB810330B5DD68AA691368D36019B93E
:10267000402B84BF402313606B8A1468426D1C4456
:10268000013CB4FBF3F46343033323F0030302EB95
:10269000411043EAC44343F0C043C0F8103B2B68E9
:1026A00003F00303012B09B20ED1D2F8083802EB74
:1026B000411013F4807FD0F8003B14BF43F08053E7
:1026C00043F00053C0F8003B02EB4112D2F8003B4C
:1026D00043F00443C2F8003B30BD00002DE9F04157
:1026E000244D6E6D06EB40130446D3F8087BC3F807
:1026F000087B38070AD5D6F81438190706D505EB34
:1027000084032146DB6828465B689847FA072FD583
:10271000D6F81438DB072BD505EB8403D968CCB980
:102720008B69488A5E68B6FBF0F200FB12628AB9D8
:102730001868DA6890420DD2121A83E81400202338
:1027400083F311880B482146FFF78AFF84F3118831
:10275000BDE8F081012303FA04F26B8923EA020346
:102760006B81CB6823B121460248BDE8F041184790
:10277000BDE8F0811C2D002000EB810370B5DD6801
:10278000436D6C692668E6604A0156BB1A444FF4F3
:102790000020C2F810092A6802F00302012A0AB2D6
:1027A0000ED1D3F8080803EB421410F4807FD4F85C
:1027B000000914BF40F0805040F00050C4F80009F8
:1027C00003EB4212D2F8000940F00440C2F80009BD
:1027D000D3F83408012202FA01F10143C3F8341896
:1027E00070BD19B9402E84BF4020206020682E8A19
:1027F000841940F00050013C1A44B4FBF6F440EA5E
:10280000C440C6E7F8B504461E48456D05EB4413C1
:10281000D3F80869C3F80869F10717D5D5F8103857
:10282000DA0713D500EB8403D9684B691F68DA68AF
:10283000974218D2D21B00271A605F60202383F3CF
:1028400011882146FFF798FF87F31188330617D5C3
:10285000D5F834280123A340134211D02046BDE807
:10286000F840FFF71FBD012303FA04F2038923EAAE
:10287000020303818B68002BE8D021469847E5E7E7
:10288000F8BD00BF1C2D002097482DE9F84F456D7D
:102890006E69AB691E4016F4805F6E61044605D018
:1028A000FEF72EFDBDE8F84FFFF780BC002E12DAD0
:1028B000D5F8003E8C489B071EBFD5F8003E23F09C
:1028C0000303C5F8003ED5F8043823F00103C5F82A
:1028D0000438FEF743FD370505D58348FFF7AEFC06
:1028E0008148FEF72BFDB0040CD5D5F8083813F05D
:1028F000060FEB6823F470530CBF43F4105343F4FA
:10290000A053EB60310704D56368DB680BB17648F0
:102910009847F2025AD4B3020CD5D4F85480DFF8A9
:10292000C8A100274FF00109A36D9B68F9B28B4243
:1029300080F08780F70619D5616D0A6AC2F30A171D
:1029400002F00F0302F4F012B2F5802F00F0A18024
:10295000B2F5402F0AD104EB830301F58051DB6807
:10296000186A00231A469F4240F087803003D5F84A
:10297000184813D5E10302D50020FFF7AFFEA203EC
:1029800002D50120FFF7AAFE630302D50220FFF75C
:10299000A5FE270302D50320FFF7A0FE750381D50E
:1029A000E00702D50020FFF72DFFA10702D5012087
:1029B000FFF728FF620702D50220FFF723FF230756
:1029C0007FF570AF0320FFF71DFF6BE7D4F854804D
:1029D000DFF814A100274FF00109A36D9B685FFA8F
:1029E00087FB5B4597D308EB4B13D3F8002902F420
:1029F0004022B2F5802F22D1D3F80029002A1EDA16
:102A0000D3F8002942F09042C3F80029D3F80029F6
:102A1000002AFBDB5946606DFFF73AFC228909FA70
:102A20000BF322EA0303238104EB8B03DB689B682F
:102A300013B15946504698475846FFF733FC0137C3
:102A4000CBE708EB4112D2F8003B03F44023B3F587
:102A5000802F10D1D2F8003B002B0CDA628909FAE2
:102A600001F322EA0303638104EB8103DB68DB6883
:102A70000BB150469847013756E79C0708BF0A68D4
:102A8000072B98BF027003F101039CBF120A0130AB
:102A900069E7023304EB830201F5805152689069C3
:102AA0000268D0F808C04068A2EB000E0022104671
:102AB00097420AD104EB830463689B699A683A449D
:102AC0009A605A6817445F6050E712F0030F08BF1E
:102AD0000868964588BF8CF8000002F1010284BFA7
:102AE000000A0CF1010CE3E71C2D0020436D03EB01
:102AF0004111D1F8003B43F40013C1F8003B70478B
:102B0000436D03EB4111D1F8003943F40013C1F8D0
:102B100000397047436D03EB4111D1F8003B23F4BA
:102B20000013C1F8003B7047436D03EB4111D1F82E
:102B3000003923F40013C1F80039704700F16043F5
:102B400000F01F02400903F5614309018000C9B28A
:102B500000F1604083F8001300F5614001239340C9
:102B6000C0F880310360704730B5039C01720433B4
:102B700004FB0325C361049B03630021059B0060E4
:102B80004060C160426102618561046242628162AB
:102B9000C162436330BD00000022416A41610161AE
:102BA000C2608262C2626FF00101FEF725BF0000C1
:102BB00003694269934203D1C2680AB10020704799
:102BC000181D704703691960C2680132C260C2698A
:102BD000134482690361934224BF436A0361002165
:102BE000FEF7FEBE38B504460D46E3683BB16269A8
:102BF000131D1268A3621344E362002038BD237AD8
:102C000033B929462046FEF7DBFE0028EDDA38BD51
:102C10006FF00100FBE70000C368C269013BC360BD
:102C20004369134482694361934224BF436A436109
:102C300000238362036B03B11847704770B52023EC
:102C4000044683F31188866A3EB9FFF7CBFF054639
:102C500018B186F31188284670BDA36AE26A13F89A
:102C6000015BA362934202D32046FFF7D5FF002306
:102C700083F31188EFE700002DE9F84F04460E4674
:102C800090469946202787F311880025AA46D4F854
:102C900028B0BBF1000F09D149462046FFF7A2FF3B
:102CA00020B18BF311882846BDE8F88FA16AE36A4A
:102CB000A8EB050B5B1A9B4528BF9B46BBF1400F59
:102CC0001BD9334601F1400251F8040B43F8040BC1
:102CD0009142F9D1A36A40334036A3624035A26ADB
:102CE000E36A9A4202D32046FFF796FF8AF31188DF
:102CF0004545D8D287F31188C9E730465A46FDF7D3
:102D0000D7FFA36A5B445E44A3625D44E7E700002B
:102D100010B5029C0172043303FB0421C36100233C
:102D20008362C362039B0363049B00604060C460D2
:102D300042610261816104624262436310BD00002E
:102D4000026AC260426A4261026100228262C26219
:102D50006FF00101FEF750BE436902699A4203D148
:102D6000C2680AB100207047184650F8043B0B6057
:102D700070470000C368C2690133C36043691344EC
:102D800082694361934224BF436A43610021FEF795
:102D900027BE000038B504460D46E3683BB1236901
:102DA0001A1DA262E2691344E362002038BD237A4F
:102DB00033B929462046FEF703FE0028EDDA38BD78
:102DC0006FF00100FBE7000003691960C268013A77
:102DD000C260C269134482690361934224BF436A9B
:102DE000036100238362036B03B11847704700003F
:102DF00070B5202304460E4683F31188856A35B9E1
:102E00001146FFF7C7FF10B185F3118870BDA36AA3
:102E10001E70A36AE26A01339342A36204D3E1699C
:102E200020460439FFF7D0FF002080F3118870BDE1
:102E30002DE9F84F04460D4691469A464FF020087A
:102E400088F311880026B346A76A4FB95146204639
:102E5000FFF7A0FF20B187F311883046BDE8F88F57
:102E6000A06AE76AA9EB06033F1A9F4228BF1F46E4
:102E7000402F1BD905F1400355F8042B40F8042BD3
:102E80009D42F9D1A36A4033A3624036A26AE36A45
:102E90009A4204D3E16920460439FFF795FF8BF38A
:102EA00011884E45D9D288F31188CDE729463A4694
:102EB000FDF7FEFEA36A3B443D44A3623E44E5E7C2
:102EC000026943699A4203D1C3681BB91846704727
:102ED0000023FBE7836A002BF8D0043B9B1AF5D054
:102EE0001360C368013BC360C3691A44836902610C
:102EF0009A4224BF436A0361002383620123E5E70A
:102F000000F090B84FF08043002258631A6102220B
:102F1000DA6070474FF080430022DA6070470000AB
:102F20004FF08043586370474FF08043586A7047B2
:102F30004B6843608B688360CB68C3600B694361F7
:102F40004B6903628B6943620B6803607047000042
:102F500008B5224B22481A6940F2FF110A431A6150
:102F60001A6922F4FF7222F001021A611A691A6BBF
:102F70000A431A631A6D0A431A651A4A1B6D1146F1
:102F8000FFF7D6FF184802F11C01FFF7D1FF1748E1
:102F900002F13801FFF7CCFF154802F15401FFF7A9
:102FA000C7FF144802F17001FFF7C2FF124802F197
:102FB0008C01FFF7BDFF114802F1A801FFF7B8FF30
:102FC0000F4802F1C401FFF7B3FF0E4802F1E00120
:102FD000FFF7AEFFBDE8084000F0AAB80038024095
:102FE000000002407C360008000402400008024055
:102FF000000C024000100240001402400018024081
:10300000001C02400020024008B500F007FAFEF75D
:103010005FFCFFF785F8BDE80840FEF761BE0000E1
:1030200070470000104B1A6C42F001021A641A6ECD
:1030300042F001021A660D4A1B6E936843F00103C9
:1030400093604FF0804353229A624FF0FF32DA626E
:1030500000229A615A63DA605A6001225A6108219B
:103060001A601C20FFF76ABD00380240002004E00F
:103070004FF0804208B51369D1680B40D9B2C943FB
:103080009B07116107D5202383F31188FEF740FCCD
:10309000002383F3118808BD08B5FFF7E9FFBDE8F9
:1030A0000840FFF783B800001F4B1A696FEAC2524D
:1030B0006FEAD2521A611A69C2F308021A614FF01C
:1030C000FF301A695A69586100215A6959615A6971
:1030D0001A6A62F080521A621A6A02F080521A6208
:1030E0001A6A5A6A58625A6A59625A6A1A6C42F0E3
:1030F00080521A641A6E42F080521A661A6E0B4A97
:10310000106840F480701060186F00F44070B0F5E3
:10311000007F1EBF4FF4803018671967536823F48F
:103120000073536000F05AB900380240007000404C
:10313000334B4FF080521A64324A4FF440411160D1
:103140001A6842F001021A601A689207FCD59A6860
:1031500022F003029A602A4B19469A6812F00C0278
:10316000FBD1186800F0F90018609A601A6842F400
:1031700080321A600B689B03FCD54B6F43F0010350
:103180004B671F4B5A6F9007FCD51F4A5A601A684D
:1031900042F080721A601B4A53685904FCD5184BE0
:1031A0001A689201FCD5194A9A60194B1A68194B92
:1031B0009A42194B21D1194A1168194A91421CD1DE
:1031C00040F205121A60144A136803F00F03052B2E
:1031D000FAD10B4B9A6842F002029A609A6802F0A8
:1031E0000C02082AFAD15A6C42F480425A645A6E90
:1031F00042F480425A665B6E704740F20572E1E726
:10320000003802400070004008544007009488389D
:10321000002004E011640020003C024000ED00E0CA
:1032200041C20F41084A08B5536911680B4003F0C9
:103230000103536123B1054A13680BB150689847E5
:10324000BDE80840FEF7B2BF003C014088230020E3
:10325000084A08B5536911680B4003F00203536133
:1032600023B1054A93680BB1D0689847BDE8084080
:10327000FEF79CBF003C014088230020084A08B5A7
:10328000536911680B4003F00403536123B1054AED
:1032900013690BB150699847BDE80840FEF786BF37
:1032A000003C014088230020084A08B55369116892
:1032B0000B4003F00803536123B1054A93690BB136
:1032C000D0699847BDE80840FEF770BF003C014058
:1032D00088230020084A08B5536911680B4003F0A1
:1032E0001003536123B1054A136A0BB1506A984722
:1032F000BDE80840FEF75ABF003C0140882300208B
:10330000174B10B55C691A68144004F478725A615E
:10331000A30604D5134A936A0BB1D06A9847600696
:1033200004D5104A136B0BB1506B9847210604D596
:103330000C4A936B0BB1D06B9847E20504D5094A50
:10334000136C0BB1506C9847A30504D5054A936CD8
:103350000BB1D06C9847BDE81040FEF727BF00BF07
:10336000003C0140882300201A4B10B55C691A68A4
:10337000144004F47C425A61620504D5164A136D68
:103380000BB1506D9847230504D5134A936D0BB1CB
:10339000D06D9847E00404D50F4A136E0BB1506E00
:1033A0009847A10404D50C4A936E0BB1D06E984790
:1033B000620404D5084A136F0BB1506F9847230479
:1033C00004D5054A936F0BB1D06F9847BDE8104004
:1033D000FEF7ECBE003C014088230020062108B522
:1033E0000846FFF7ABFB06210720FFF7A7FB0621E6
:1033F0000820FFF7A3FB06210920FFF79FFB06210A
:103400000A20FFF79BFB06211720FFF797FB0621F9
:103410002820BDE80840FFF791BB000008B5FFF782
:1034200043FEFDF74FFDFDF7FDFEFDF7D1FDFFF774
:10343000F7FDBDE80840FFF763BD0000034611F843
:10344000012B03F8012B002AF9D170471210121337
:103450001211000053544D3332463F3F3F000000ED
:1034600000000000543400083F0000001304000076
:10347000903400083F000000190400009A3400084E
:103480003F00000021040000A43400083F000000B9
:1034900053544D3332463430780053544D33324612
:1034A0003432780053544D33324634343658580051
:1034B00000000000490F0008350F0008710F0008D8
:1034C0005D0F0008690F0008550F0008410F000844
:1034D0002D0F0008CD0F00080000000001000000C3
:1034E000000000006D61696E0000000004350008F6
:1034F00048240020C025002001000000CD1800084D
:103500000000000069646C6500000000020000001B
:103510000000000075110008DD11000840004000A7
:10352000582A0020682A0020020000000000000045
:10353000030000000000000021120008000000004D
:1035400010000000782A00200000000001000000A8
:10355000000000001C2D0020010102004172647572
:1035600050696C6F740025424F415244252D424CE6
:10357000002553455249414C25000000811C00089C
:10358000E91B0008E1100008651C0008430000006A
:103590009435000809024300020100C0320904000A
:1035A00000010202010005240010010524010001B0
:1035B000042402020524060001070582030800FF17
:1035C00009040100020A0000000705010240000092
:1035D000070581024000000012000000E0350008ED
:1035E00012011001020000400912415700020102BD
:1035F000030100000403090425424F415244250001
:103600004B616B7574654634003031323334353676
:10361000373839414243444546000000004000002D
:1036200000400000004000000040000000000100D9
:103630000000020000000200000002000000020082
:103640000000020000000200000002000000000074
:103650007113000851160008FD16000840004000D4
:103660007C2D00207C2D0020010000008C2D0020EE
:103670008000000040010000030000000000800204
:1036800000000000AAAAAAAA00000000FFFF000094
:103690000000000000A00A0040040010000000002C
:1036A000AAAAAAAA40000010DFFF00000000000044
:1036B000000000000001040000000000AAAAAAAA5D
:1036C00000010800FFFD00000000000000000000F5
:1036D0000000000000000000AAAAAAAA0000000042
:1036E000FFFF0000000000000000000000000000DC
:1036F00000000000AAAAAAAA00000000FFFF000024
:1037000000000000000000000000000000000000B9
:10371000AAAAAAAA00000000FFFF00000000000003
:10372000000000000000000000000000AAAAAAAAF1
:1037300000000000FFFF000000000000000000008B
:1037400000000000000000000A000000000000006F
:103750000300000000000000000000000000000066
:103760000000000000000000000000000000000059
:103770000000000000000000FF00960000000008AC
:1037800004000000F4350008000000000000000004
:103790000000000000000000000000000000000029
:1037A000FFFFFFFFFFFFFFFFFFFFFFFFFFFFFFFF29
:1037B000FFFFFFFFFFFFFFFFFFFFFFFFFFFFFFFF19
:1037C000FFFFFFFFFFFFFFFFFFFFFFFFFFFFFFFF09
:020000040801F1
:1000000000060020B51201083D320A0899310A089D
:1000100005320A0899310A08D1310A08B7120108D5
:10002000B7120108B7120108B71201083D490C08C0
:10003000B7120108B7120108B7120108B712010878
:10004000B7120108B7120108B7120108B712010868
:10005000B7120108B7120108595B0C08815B0C0844
:10006000A95B0C08D15B0C08F95B0C08E1040C08D7
:1000700009050C0835050C0861050C088D050C08F0
:10008000B5050C08E1050C0865040C08B712010859
:10009000B7120108B7120108B7120108215C0C0859
:1000A000B7120108B7120108B7120108B712010808
:1000B000595D0C086D5D0C08815D0C086D0B0C081A
:1000C000150D0C08B7120108B7120108B712010884
:1000D000B7120108F55C0C08B7120108095D0C089D
:1000E000855C0C08B7120108B7120108A55D0C0861
:1000F000A95D0C08BD5D0C08C15D0C080D060C085F
:10010000B7120108B7120108915D0C08B712010877
:100110001D5D0C08315D0C08B7120108B71201080B
:1001200039060C0861060C088D060C08B9060C0887
:10013000E5060C08B7120108B7120108B71201084A
:10014000B7120108B7120108B712010869500C086C
:100150000D070C0839070C0865070C08455D0C08ED
:10016000B7120108B7120108B7120108B712010847
:10017000B7120108B7120108B7120108B712010837
:10018000B7120108B7120108B7120108B712010827
:10019000B7120108B7120108B7120108B712010817
:1001A000B7120108B7120108B7120108B712010807
:1001B000B7120108B7120108B7120108B7120108F7
:1001C000B7120108B7120108B7120108B7120108E7
:1001D000B7120108B7120108B7120108B7120108D7
:1001E000693501087D660108D9A00108710402087B
:1001F0009D4D0208F1D40208615304080515060854
:100200000D1B06082565060805B70608C9BE0608C1
:1002100001C2060871270708A9480708291D080810
:1002200061900808FD2A0A0895250B0829800B080B
:1002300089A60B0805B10B0889E00B0851E60B08ED
:1002400081F0004102E000BF83F0004330B54FEA87
:1002500041044FEA430594EA050F08BF90EA020FF4
:100260001FBF54EA000C55EA020C7FEA645C7FEA87
:10027000655C00F0E2804FEA5454D4EB5555B8BFAA
:100280006D420CDD2C4480EA020281EA030382EA1B
:10029000000083EA010180EA020281EA0303362DAD
:1002A00088BF30BD11F0004F4FEA01314FF4801C80
:1002B0004CEA113102D0404261EB410113F0004F92
:1002C0004FEA03334CEA133302D0524263EB430349
:1002D00094EA050F00F0A780A4F10104D5F1200EE7
:1002E0000DDB02FA0EFC22FA05F2801841F1000142
:1002F00003FA0EF2801843FA05F359410EE0A5F116
:1003000020050EF1200E012A03FA0EFC28BF4CF046
:10031000020C43FA05F3C01851EBE37101F00045FC
:1003200007D54FF0000EDCF1000C7EEB00006EEB09
:100330000101B1F5801F1BD3B1F5001F0CD3490893
:100340005FEA30004FEA3C0C04F101044FEA4452EA
:1003500012F5800F80F09A80BCF1004F08BF5FEA71
:10036000500C50F1000041EB045141EA050130BD51
:100370005FEA4C0C404141EB0101013C28BFB1F563
:10038000801FE9D291F0000F04BF01460020B1FAAE
:1003900081F308BF2033A3F10B03B3F120020CDA81
:1003A0000C3208DD02F1140CC2F10C0201FA0CF05F
:1003B00021FA02F10CE002F11402D8BFC2F1200CC4
:1003C00001FA02F120FA0CFCDCBF41EA0C0190407A
:1003D000E41AA2BF01EB0451294330BD6FEA0404C3
:1003E0001F3C1CDA0C340EDC04F11404C4F12002AE
:1003F00020FA04F001FA02F340EA030021FA04F3C0
:1004000045EA030130BDC4F10C04C4F1200220FA16
:1004100002F001FA04F340EA0300294630BD21FA54
:1004200004F0294630BD94F0000F83F4801306BF1A
:1004300081F480110134013D4EE77FEA645C18BF0E
:100440007FEA655C29D094EA050F08BF90EA020FA5
:1004500005D054EA000C04BF1946104630BD91EA9D
:10046000030F1EBF0021002030BD5FEA545C05D1A0
:100470004000494128BF41F0004130BD14F58004DF
:100480003CBF01F5801130BD01F0004545F0FE4153
:1004900041F470014FF0000030BD7FEA645C1ABF88
:1004A000194610467FEA655C1CBF0B46024650EABF
:1004B000013406BF52EA033591EA030F41F40021EB
:1004C00030BD00BF90F0000F04BF0021704730B571
:1004D0004FF4806404F132044FF000054FF0000146
:1004E00050E700BF90F0000F04BF0021704730B507
:1004F0004FF4806404F1320410F0004548BF4042DC
:100500004FF000013EE700BF42004FEAE2014FEA30
:1005100031014FEA02701FBF12F07F4393F07F4F0B
:1005200081F06051704732F07F4208BF704793F00E
:100530007F4F04BF41F40021704730B54FF4607421
:1005400001F0004521F000411CE700BF50EA010224
:1005500008BF704730B54FF000050AE050EA0102CD
:1005600008BF704730B511F0004502D5404261EB3D
:1005700041014FF4806404F132045FEA915C3FF47E
:10058000D8AE4FF003025FEADC0C18BF03325FEA1B
:10059000DC0C18BF033202EBDC02C2F1200300FACC
:1005A00003FC20FA02F001FA03FE40EA0E0021FAF1
:1005B00002F11444BDE600BF70B54FF0FF0C4CF4DF
:1005C000E06C1CEA11541DBF1CEA135594EA0C0F91
:1005D00095EA0C0F00F0DEF82C4481EA030621EACC
:1005E0004C5123EA4C5350EA013518BF52EA033507
:1005F00041F4801143F4801338D0A0FB02CE4FF0B9
:100600000005E1FB02E506F00042E0FB03E54FF0E8
:100610000006E1FB03569CF0000F18BF4EF0010EE0
:10062000A4F1FF04B6F5007F64F5407404D25FEADC
:100630004E0E6D4146EB060642EAC62141EA55518F
:100640004FEAC52040EA5E504FEACE2EB4F1FD0CD1
:1006500088BFBCF5E06F1ED8BEF1004F08BF5FEA4F
:10066000500E50F1000041EB045170BD06F0004601
:1006700046EA010140EA020081EA0301B4EB5C04AE
:10068000C2BFD4EB0C0541EA045170BD41F48011A6
:100690004FF0000E013C00F3AB8014F1360FDEBFCB
:1006A000002001F0004170BDC4F10004203C35DAA7
:1006B0000C341BDC04F11404C4F1200500FA05F32A
:1006C00020FA04F001FA05F240EA020001F00042CB
:1006D00021F0004110EBD37021FA04F642EB060141
:1006E0005EEA430E08BF20EAD37070BDC4F10C046B
:1006F000C4F1200500FA04F320FA05F001FA04F22F
:1007000040EA020001F0004110EBD37041F100011A
:100710005EEA430E08BF20EAD37070BDC4F1200525
:1007200000FA05F24EEA020E20FA04F301FA05F28D
:1007300043EA020321FA04F001F0004121FA04F235
:1007400020EA020000EBD3705EEA430E08BF20EA05
:10075000D37070BD94F0000F0FD101F0004640003F
:1007600041EB010111F4801F08BF013CF7D041EAC1
:10077000060195F0000F18BF704703F000465200C5
:1007800043EB030313F4801F08BF013DF7D043EA96
:100790000603704794EA0C0F0CEA135518BF95EA4C
:1007A0000C0F0CD050EA410618BF52EA4306D1D1D3
:1007B00081EA030101F000414FF0000070BD50EAF2
:1007C000410606BF1046194652EA430619D094EA7C
:1007D0000C0F02D150EA013613D195EA0C0F05D166
:1007E00052EA03361CBF104619460AD181EA0301BA
:1007F00001F0004141F0FE4141F470014FF0000072
:1008000070BD41F0FE4141F4780170BD70B54FF00C
:10081000FF0C4CF4E06C1CEA11541DBF1CEA13558C
:1008200094EA0C0F95EA0C0F00F0A7F8A4EB05046E
:1008300081EA030E52EA03354FEA013100F0888065
:100840004FEA03334FF0805545EA131343EA12632E
:100850004FEA022245EA111545EA10654FEA0026E3
:100860000EF000419D4208BF964244F1FD0404F59C
:10087000407402D25B084FEA3202B61A65EB0305F8
:100880005B084FEA32024FF480104FF4002CB6EBB5
:10089000020E75EB030E22BFB61A754640EA0C0035
:1008A0005B084FEA3202B6EB020E75EB030E22BF75
:1008B000B61A754640EA5C005B084FEA3202B6EBB6
:1008C000020E75EB030E22BFB61A754640EA9C0075
:1008D0005B084FEA3202B6EB020E75EB030E22BF45
:1008E000B61A754640EADC0055EA060E18D04FEA03
:1008F000051545EA16754FEA06164FEAC30343EAA3
:1009000052734FEAC2025FEA1C1CC0D111F4801F6F
:100910000BD141EA00014FF000004FF0004CB6E768
:1009200011F4801F04BF01430020B4F1FD0C88BF07
:10093000BCF5E06F3FF6AFAEB5EB030C04BFB6EB12
:10094000020C5FEA500C50F1000041EB045170BD05
:100950000EF0004E4EEA113114EB5C04C2BFD4EB32
:100960000C0541EA045170BD41F480114FF0000EB6
:10097000013C90E645EA060E8DE60CEA135594EA32
:100980000C0F08BF95EA0C0F3FF43BAF94EA0C0F35
:100990000AD150EA01347FF434AF95EA0C0F7FF4AA
:1009A00025AF104619462CE795EA0C0F06D152EAFE
:1009B00003353FF4FDAE1046194622E750EA4106E2
:1009C00018BF52EA43067FF4C5AE50EA41047FF4F3
:1009D0000DAF52EA43057FF4EBAE12E74FF0FF3C58
:1009E00006E000BF4FF0010C02E000BF4FF0010C29
:1009F0004DF804CD4FEA410C7FEA6C5C4FEA430CA2
:100A000018BF7FEA6C5C1BD001B050EA410C0CBFF0
:100A100052EA430C91EA030F02BF90EA020F002052
:100A2000704710F1000F91EA030F58BF994208BFB9
:100A300090422CBFD8176FEAE37040F00100704776
:100A40004FEA410C7FEA6C5C02D150EA013C07D1CD
:100A50004FEA430C7FEA6C5CD6D152EA033CD3D018
:100A60005DF8040B704700BF8446104662468C4612
:100A70001946634600E000BF01B5FFF7B7FF002845
:100A800048BF10F1000F01BD4DF808EDFFF7F4FF6E
:100A90000CBF012000205DF808FB00BF4DF808EDF9
:100AA000FFF7EAFF34BF012000205DF808FB00BF1C
:100AB0004DF808EDFFF7E0FF94BF012000205DF83E
:100AC00008FB00BF4DF808EDFFF7CEFF94BF0120F3
:100AD00000205DF808FB00BF4DF808EDFFF7C4FFEC
:100AE00034BF012000205DF808FB00BF4FEA410C35
:100AF0007FEA6C5C02D150EA013C0AD14FEA430C18
:100B00007FEA6C5C02D152EA033C02D14FF0000054
:100B100070474FF0010070474FEA410212F5001292
:100B200015D211D56FF47873B3EB625212D94FEA34
:100B3000C12343F0004343EA505311F0004F23FA1E
:100B400002F018BF404270474FF00000704750EA73
:100B5000013005D111F0004008BF6FF00040704730
:100B60004FF00000704700BF4A0011D212F500128A
:100B700011D20DD56FF47873B3EB62520ED44FEAF5
:100B8000C12343F0004343EA505323FA02F0704775
:100B90004FF00000704750EA013002D14FF0FF30B3
:100BA00070474FF0000070474FEA4102B2F1E04356
:100BB00024BFB3F5001CDCF1FE5C0DD901F0004C44
:100BC0004FEAC0024CEA5070B2F1004F40EB830094
:100BD00008BF20F00100704711F0804F21D113F1C0
:100BE0003872BCBF01F00040704741F480114FEAF9
:100BF0005252C2F11802C2F1200C10FA0CF320FA82
:100C000002F018BF40F001004FEAC1234FEAD3239E
:100C100003FA0CFC40EA0C0023FA02F34FEA430308
:100C2000CCE77FEA625307D150EA01331EBF4FF091
:100C3000FE4040F44000704701F0004040F0FE40AC
:100C400040F40000704700BF80F0004002E000BFA9
:100C500081F0004142001FBF5FEA410392EA030FA7
:100C60007FEA226C7FEA236C6AD04FEA1262D2EBF1
:100C70001363C1BFD218414048404140B8BF5B42F6
:100C8000192B88BF704710F0004F40F4000020F08F
:100C90007F4018BF404211F0004F41F4000121F0A5
:100CA0007F4118BF494292EA030F3FD0A2F10102EF
:100CB00041FA03FC10EB0C00C3F1200301FA03F12D
:100CC00000F0004302D5494260EB4000B0F5000F50
:100CD00013D3B0F1807F06D340084FEA310102F10F
:100CE0000102FE2A51D2B1F1004F40EBC25008BFC1
:100CF00020F0010040EA03007047490040EB00008B
:100D0000013A28BFB0F5000FEDD2B0FA80FCACF18B
:100D1000080CB2EB0C0200FA0CF0AABF00EBC250B8
:100D200052421843BCBFD0401843704792F0000FA6
:100D300081F4000106BF80F400000132013BB5E7F9
:100D40004FEA41037FEA226C18BF7FEA236C21D06F
:100D500092EA030F04D092F0000F08BF08467047D4
:100D600090EA010F1CBF0020704712F07F4F04D1A2
:100D7000400028BF40F00040704712F100723CBFB5
:100D800000F50000704700F0004343F0FE4040F4DF
:100D9000000070477FEA226216BF08467FEA23639D
:100DA0000146420206BF5FEA412390EA010F40F488
:100DB000800070474FF0000304E000BF10F00043D4
:100DC00048BF40425FEA000C08BF704743F09643BB
:100DD00001464FF000001CE050EA010208BF7047D6
:100DE0004FF000030AE000BF50EA010208BF70475D
:100DF00011F0004302D5404261EB41015FEA010C72
:100E000002BF84460146002043F0B64308BFA3F169
:100E10008053A3F50003BCFA8CF2083AA3EBC2534B
:100E200010DB01FA02FC634400FA02FCC2F120026A
:100E3000BCF1004F20FA02F243EB020008BF20F0A1
:100E40000100704702F1200201FA02FCC2F1200207
:100E500050EA4C0021FA02F243EB020008BF20EAFC
:100E6000DC7070477BB972B90029BEBF00204FF01B
:100E7000004106E008BF00281CBF6FF000414FF0A2
:100E8000FF3000F015BAADF1080C6DE904CE002971
:100E900009DB002B1ADB00F0A3F8DDF804E0DDE944
:100EA000022304B07047404261EB4101002B1BDB81
:100EB00000F096F8DDF804E0DDE9022304B04042DA
:100EC00061EB4101524263EB43037047524263EBD3
:100ED000430300F085F8DDF804E0DDE9022304B007
:100EE000404261EB41017047524263EB430300F023
:100EF00077F8DDF804E0DDE9022304B0524263EB49
:100F00004303704753B94AB9002908BF00281CBFE2
:100F10004FF0FF314FF0FF3000F0CAB9ADF1080CCF
:100F20006DE904CE00F05CF8DDF804E0DDE90223B1
:100F300004B0704730B1012390FAA0F0B0FA80F00D
:100F40001844704708460029FBD02123F4E700BF6E
:100F5000430803F05533C01A830803F0333300F01D
:100F60003330184400EB101000F00F3000EB00207D
:100F700000EB0040000E704707EE900AF5EEC07AD5
:100F8000F1EE10FA01D400F00BB8F1EE677A08B573
:100F900017EE900A00F004F8404261EB410108BDF1
:100FA000D0B5FFF7B1FA0C4B002206460F46FFF70B
:100FB00003FBFFF7D9FD0446FFF784FA074B002235
:100FC000FFF7FAFA02460B4630463946FFF73CF97E
:100FD000FFF7CAFD2146D0BD0000F03D0000F04102
:100FE0002DE9F047089D04468E46002B4DD18A42DC
:100FF000944669D9B2FA82F252B101FA02F3C2F10F
:10100000200120FA01F10CFA02FC41EA030E94409F
:101010004FEA1C48210CBEFBF8F61FFA8CF708FBC0
:1010200016E341EA034306FB07F199420AD91CEB98
:10103000030306F1FF3080F01F81994240F21C81CA
:10104000023E63445B1AA4B2B3FBF8F008FB103312
:1010500044EA034400FB07F7A7420AD91CEB040447
:1010600000F1FF3380F00A81A74240F20781644417
:10107000023840EA0640E41B00261DB1D44000239C
:10108000C5E900433146BDE8F0878B4209D9002D00
:1010900000F0EF800026C5E9000130463146BDE88A
:1010A000F087B3FA83F6002E4AD18B4202D38242F4
:1010B00000F2F980841A61EB030301209E46002DA3
:1010C000E0D0C5E9004EDDE702B9FFDEB2FA82F2F8
:1010D000002A40F09280A1EB0C014FEA1C471FFA56
:1010E0008CFE0126200CB1FBF7F307FB131140EA3D
:1010F00001410EFB03F0884208D91CEB010103F10A
:10110000FF3802D2884200F2CB804346091AA4B2CB
:10111000B1FBF7F007FB101144EA01440EFB00FE9F
:10112000A64508D91CEB040400F1FF3102D2A64504
:1011300000F2BB800846A4EB0E0440EA03409CE7A3
:10114000C6F12007B34022FA07FC4CEA030C20FA50
:1011500007F401FA06F31C43F9404FEA1C4900FA70
:1011600006F3B1FBF9F8200C1FFA8CFE09FB1811ED
:1011700040EA014108FB0EF0884202FA06F20BD960
:101180001CEB010108F1FF3A80F08880884240F2B0
:101190008580A8F102086144091AA4B2B1FBF9F0F4
:1011A00009FB101144EA014100FB0EFE8E4508D9EF
:1011B0001CEB010100F1FF346CD28E456AD9023874
:1011C000614440EA0840A0FB0294A1EB0E01A14259
:1011D000C846A64656D353D05DB1B3EB080261EBC7
:1011E0000E0101FA07F722FA06F3F1401F43C5E9A1
:1011F000007100263146BDE8F087C2F12003D840D7
:101200000CFA02FC21FA03F3914001434FEA1C4718
:101210001FFA8CFEB3FBF7F007FB10360B0C43EA0A
:10122000064300FB0EF69E4204FA02F408D91CEBBA
:10123000030300F1FF382FD29E422DD902386344B8
:101240009B1B89B2B3FBF7F607FB163341EA034158
:1012500006FB0EF38B4208D91CEB010106F1FF38A7
:1012600016D28B4214D9023E6144C91A46EA00469E
:1012700038E72E46284605E70646E3E61846F8E630
:101280004B45A9D2B9EB020864EB0C0E0138A3E779
:101290004646EAE7204694E74046D1E7D0467BE75A
:1012A000023B614432E7304609E76444023842E7D2
:1012B000704700BF02E000F000F8FEE772B6374862
:1012C00080F30888364880F3098836483649086034
:1012D00040F20000CCF200004EF63471CEF2000174
:1012E0000860BFF34F8FBFF36F8F40F20000C0F272
:1012F000F0004EF68851CEF200010860BFF34F8F28
:10130000BFF36F8F4FF00000E1EE100A4EF63C7114
:10131000CEF200010860062080F31488BFF36F8FBF
:10132000B3F06AFBB4F0B4FA4FF055301F491B4AD2
:1013300091423CBF41F8040BFAE71D49184A91421B
:101340003CBF41F8040BFAE71A491B4A1B4B9A426F
:101350003EBF51F8040B42F8040BF8E7002018498F
:10136000184A91423CBF41F8040BFAE7B3F048FB3E
:10137000B4F0E2FA144C154DAC4203DA54F8041BF5
:101380008847F9E702F0E0F8114C124DAC4203DA5D
:1013900054F8041B8847F9E7B3F030BB000600207F
:1013A000002200200000010808ED00E000000020FD
:1013B00000060020A8110F0800220020742C002035
:1013C000782C002050490120E0010108400201086A
:1013D00040020108400201082DE9F04F2DED108A6E
:1013E000C1F80CD0C3689D46BDEC108ABDE8F08FF3
:1013F000002383F311882846A0470020B2F034FA76
:10140000FEE7B2F091F800DFFEE7000001F0FF0117
:10141000102A2BDB10F0070F08D010F8013B013A1F
:101420008B422DD010F0070F42B3F6D1F0B441EA51
:10143000012141EA014122F007047FF00007002367
:10144000F0E80256083C85EA010586EA010685FABD
:1014500047F5A3FA87F586FA47F6A5FA87F68EB917
:10146000EED1F0BC01F0FF0102F0070232B110F83A
:10147000013B013A83EA010313B1F8D10020704720
:1014800001387047002D06BF35460338073815F080
:10149000010F07D1013015F4807F02BF013015F430
:1014A000C03F0130F0BC0138704700BF10F8012B7D
:1014B00011F8013B012A28BF9A42F7D0D01A704791
:1014C000034613F8012B002AFBD1181A0138704784
:1014D00038B50022002304460D46FFF7DFFA28B98D
:1014E00020462946BDE8384000F00AB8204605F1FC
:1014F000004100F005F8404261EB410138BD00BFFA
:10150000D0B50C4B002206460F46FFF755F8FFF703
:101510002BFB0446FEF7D6FF074B0022FFF74CF8E3
:1015200002460B4630463946FEF78EFEFFF71CFB9F
:101530002146D0BD0000F03D0000F04103680022CC
:101540001B6818477FB503914021054680F0B2FB28
:10155000039A18B90124204604B070BD134E0392BB
:1015600096F9E632002BF5D061F038FB437A039A06
:1015700053B961F033FB847A039A2CB90C4B4021A8
:10158000284680F09FFBE6E7D6F8DC3CB6F9E81287
:10159000B3F906309942DDDD064B00934021064B3E
:1015A000284680F08FFB0024D5E700BF804C002048
:1015B00004D00C0823D00C0811D00C08F0B50D464F
:1015C0009DB02021044680F075FB002800F09D802E
:1015D0004F4E96F9E632ABB1D6F8DC2CB6F9E832CC
:1015E000B2F90A1003F10A02914203DD40F28D3292
:1015F000934207DC474B2A462021204680F062FBBD
:10160000002080E096F9D532022B05D1424B2A46C4
:101610002021204680F056FBB6F8A832A3F57A7355
:101620009BB241F6583293420DD83C4F96EDC57AA5
:10163000D7F81C3DD3ED097AB4EEE77AF1EE10FA53
:1016400003DD374BD7E7374BD5E796EDC67AD3EDB9
:101650000B7AB4EEE77AF1EE10FAF2DCB6F9E23288
:10166000002B01DC304BC6E796F874230D2A06D810
:101670000123934013F4215F01D02C4BBBE72C488E
:1016800010F0CCF9012806D1D7F8280D87F068FBB7
:1016900098B101281AD00021602204A80391B7F064
:1016A0006FF92449D7F8240D642303AA86F07AFF42
:1016B00000BB03AB0093204B02E0204B0093204B78
:1016C0002A462021204680F0FDFA99E796F8F03C62
:1016D00073B11C48192150F08DFB48B11948D6F858
:1016E000C062192150F0ACFB8642D4DD164BE5E711
:1016F000164BE3E71649D7F81C0D642303AA83F0C1
:1017000011FE0028D5D01DB0F0BD0120FBE700BFC1
:10171000804C00202CD00C083FD00C08806C00209E
:1017200077D00C0867D00C0891D00C08A6D00C0814
:101730005882002020D10C0824D10C08EBD00C08D2
:10174000C6D00C08C03900200AD10C08FBD00C0808
:1017500036D10C0807B5044888F05AFE00F00100A5
:1017600003B05DF804FB00BF807900202DE9F04351
:10177000DFF844910446D9F8EC000368A5B01B6972
:101780000D469847804615F067FC00210746602209
:101790000CA80B91B7F0F4F864230BAA4146384625
:1017A00014F04EFF064648B93A4A0BAB294620468C
:1017B00080F0AAFC304625B0BDE8F083A9F56B6047
:1017C0006EF014FDB8F1000F03D194F91E30012B17
:1017D0000AD1314812F02CFC80B9304A2946204603
:1017E00080F092FC0026E5E710F0060FE2D0A9F5A4
:1017F000405012F01DFC08B9294AEFE703A938460A
:1018000014F050FD28B19DF80D305B0601D5254A36
:10181000E4E7DFF8A880D8EDC17AF5EEC07AF1EE02
:1018200010FA4FF00003C5DD089309930A930DF1F8
:10183000200907AB019305AA06AB04A9CDF80090D7
:10184000384615F011F9484630F05EFDD8EDC17A02
:10185000B4EEE70AF1EE10FA01DB134ABEE79DEDA4
:10186000057AF4EEC77AF1EE10FA01D80F4AB5E71F
:101870009DED047AF4EEC77AF1EE10FA01D80C4A25
:10188000ACE79DED067AF4EEC77AF1EE10FA91D846
:10189000084AA3E73CD10C08802C002045D10C0855
:1018A0005CD10C0882D10C0890D10C08A5D10C0891
:1018B000BBD10C08D1D10C08805C0020804C0020EA
:1018C00008B5064B93F805319B0704D5044A80F010
:1018D0001BFC002008BD0120FCE700BF805C00204D
:1018E000E8D10C0870B50C4C0546D4F8EC00036840
:1018F0005B690E46984710B10124204670BDA4F5DF
:10190000405012F0A7FB04460028F5D1034A3146A7
:10191000284680F0F9FBF0E7805C0020F8D10C0845
:101920002DE9F046464ED6F8103193F8CB509BB0D7
:1019300081468A4665B9434B1B68986A03685B6BAE
:101940009847044640B9404A5146484680F0DCFB7F
:1019500028461BB0BDE8F08661F040F9202162F016
:10196000B3F958B161F03AF91F2162F0ADF988B3CB
:10197000364A5146484680F0C7FB002496F8E230CC
:1019800003F01403142B05D1314A5146484680F028
:10199000BBFB00245146484681F084FA002188426E
:1019A0004FF0600202A808BF0C460191B6F0E8FFB4
:1019B000D6F81001036801AA1B6864219847054600
:1019C00080B9244A01AB5146484680F09DFB2C4625
:1019D0002546BDE761F002F9A52162F075F90028FE
:1019E000C6D1CBE7002CF3D0D9F808303BB9D9F8F1
:1019F000003051465B6B484698470446E8E751463D
:101A00004846FFF7DBFD514607464846FFF758FFBB
:101A10003840C4B251464846FFF794FD5146044051
:101A20004846FFF75FFF51460440484680F094FB6C
:101A300051460440484681F04DFA0440C8E700BFD3
:101A4000805C0020E08400200CD20C0823D20C081B
:101A50003DD20C0855D20C0808B5FFF761FF054AC6
:101A600092F8E01060F3041182F8E010024A9071DD
:101A700008BD00BF805C0020BD860020F7B505468C
:101A80000F4680F053F9044678B10221284680F0D1
:101A900011F9064648B1154888F0BAFCC205C0F3F2
:101AA0000723C0F3002403D53446204603B0F0BD1D
:101AB0009B07F9D50D4888F0B9FC0D4B03F6CC43D4
:101AC000D3ED007AF8EEE77A30EE670ADFED097AB7
:101AD000B0EEC00AB4EEE70AF1EE10FAE4DD064B10
:101AE0003A460221284680F0EDF8DEE780790020B2
:101AF000806C00200000C84260D20C08F8B5044693
:101B00000F4680F0C9FB10210546204680F0D2F830
:101B100058B12046FFF71EFE064630B9044B3A4640
:101B20001021204680F0CEF835462846F8BD00BF8B
:101B300074D20C0870B505460E4680F05FF8044676
:101B400078B18021284680F0B5F850B1074B93F862
:101B5000AD3643B1064B32468021284680F0B2F8BC
:101B60000024204670BD0446FBE700BF805C0020D7
:101B700088D20C0838B50D4D0446D5F8280D87F0ED
:101B8000EFF8012810D0D5F8280D87F0E9F80228E1
:101B900004D02046BDE8384080F032B804480FF049
:101BA0003DFF0128F5D138BD0020FCE7806C002006
:101BB00058820020F0B5134C04F5005385B0D3F8DB
:101BC000D42C0092D3F8D82C0192D3F8DC2C0292BA
:101BD000D3F8E03C03936A4606460F4681F014F9B9
:101BE00039460546304680F0C7F804F54054284091
:101BF00094F8E03060F3C303C3F3C00084F8E0302E
:101C000005B0F0BD802C00202DE9F843064627489A
:101C1000DFF8A890DFF8A8800F466EF0E7FA0446D8
:101C2000D9F8EC0003681B699847054630B914F0F1
:101C3000060F03D1D9F82031022B09D1394630469D
:101C400080F086F9054618B9002488F807400AE0B4
:101C500039463046FFF78AFD04460028F4D02DB9F6
:101C6000012388F807302046BDE8F8830821304674
:101C700080F020F80028F3D00D4823F0F9FB00286D
:101C8000EED00C4B93F81424B02101FB023203F583
:101C90000053B2F81E22B3F9D6329A42E0DD064B69
:101CA0003A460821304680F00DF8CDE7D04D0020AF
:101CB000A02D0020802C00209CD20C08805C0020ED
:101CC000BD8600202DE9F3410E46054615F0C4F906
:101CD000804614F0A9FA044640B9514A0121284629
:101CE00080F012FA204602B0BDE8F0814D4FD7F8DF
:101CF000EC00036831469B699847044658B9D7F809
:101D0000EC0003681B6C9847474A034601212846AC
:101D100080F0FAF9E6E7AB68002BE3D01021284603
:101D20007FF0C8FF20B3D8ED937A98ED920A20EEA9
:101D3000270AB4F0C7FBDFED3D7AA7F5805320EE0C
:101D4000270AB3F9A832DFED3A7A20EE270A07EE28
:101D5000903AF8EEE77AB4EEE70AF1EE10FA07DD12
:101D6000344B0122102128467FF0ACFF0024B9E754
:101D7000402128467FF09EFF38B3012E1ED0232E2F
:101D80001CD0042E1AD02C4CD4F8DC3CB3F908300B
:101D900000EE103AA4F50050B8EEC00A00F0BCFB0B
:101DA000B5EEC00AF1EE10FA1DDD244B00930122BE
:101DB000234B402128467FF085FFD7E7D7F8EC007A
:101DC0000368DB6B98470028DDD01E4B1B68D86A80
:101DD0000368DB6998470128014619D11A4A284649
:101DE00080F092F9C2E7D7F8EC0003685B69984786
:101DF00030B1D4F8DC3CB3F90830002BE5DDD4E792
:101E0000D7F8EC0003681B6898470B28DDD1F0E792
:101E10003146284602B0BDE8F04180F005BD00BF64
:101E2000ACD20C08805C0020BDD20C08E02E6542CC
:101E30000000C842D1D20C08804C002023D00C08EE
:101E4000D9D20C08E0840020E5D20C0870B5054614
:101E50000E46FFF78BFC084B0446D87131462846E6
:101E6000FFF740FD31460028284608BF002480F0D7
:101E7000B3FE204070BD00BFBD8600202DE9F041BB
:101E80004E4F3B78002B40F096804D4CD4F81051CB
:101E900095F8CB5001263E701DB13B702846BDE839
:101EA000F08181F0C5F8054630B9464A387013789C
:101EB00043F001031370F1E756F0B8F9314655F0DD
:101EC000EFFAA4F5405006F047FD3F4B1E710B267C
:101ED0004AF026FF013E4AF0F1FE16F0FF06F7D168
:101EE0003A4800F083FF15F0B7F8D0F80022C4F8A4
:101EF000382190F87C32DA074DD414F017FC56F0F4
:101F000095F93C2156F0CEF80023C4F8F8300021B2
:101F10002E482F4E00F0F0FF2C4812F089F80146B1
:101F20002C488CF0E7F92C4B1B68D86A0368012118
:101F30001B689847D4F8100103689B6A98470121F1
:101F4000D4F8100189F01EFA56F070F98046D4F8E2
:101F5000EC0003681B68984796F8682201464046E3
:101F600055F076FCA6F5005006F0E8FC53F058FB5F
:101F700052F094FE00233B7091F092F9B4F8E230F5
:101F800006F5005623F4087343F02003C6F8340D19
:101F9000A4F8E23082E79B07B9D431460B4804F03D
:101FA0005FFD0E4888F042FADFED0D7A20EE270A39
:101FB00084ED3E0AABE7002570E700BF782C0020D7
:101FC000805C0020DC860020BD860020802C002064
:101FD000804C00205C570020E084002080790020A5
:101FE0000AD7233C2DE9F043374DD5F8103193F84B
:101FF000CB3087B0002B64D062B1012901D02329F6
:1020000008D195F9E030002B04DB0024204607B00E
:10201000BDE8F08381F0B8F804460028F5D015F04B
:102020001BF807461CF03EF88046384613F006FEC3
:10203000D8B198F92430022B17D100264FF00009AF
:10204000F1B203AA38460191CDF80C90CDF810906A
:10205000CDF8149014F090F9019918B103AA4046F4
:102060001BF0D0FC0136032EEAD11848012106F0FE
:10207000DFFE1648012106F00FFE0021D5F8100101
:1020800089F080F9124832F063FE56F0CFF8002153
:1020900055F006FA0F4B1B68D86A036800211B68CD
:1020A000984795F8E230D5F8EC100B486FF34513DC
:1020B00085F8E2300B1A594259413C308FF000FB51
:1020C000A4E70124A2E700BF805C0020802C002050
:1020D000447C0020E0840020E07D002010B5064C08
:1020E000D4F8EC0003685B6A984718B1D4F8103153
:1020F00093F8CB0010BD00BF805C002030B52DED03
:10210000028B89B00C46B0EE408AFFF7E7FF054628
:10211000002838D0B4EE488AF1EE10FA7CBFDFED2B
:102120001C8ADFED1C7A226863689FED1A0A68BF7B
:10213000DFED198A029278BF68EE288A02A878BF7C
:1021400068EEA78AD4ED027A0393F1EE677ACDEDBB
:10215000047A2FF0DBFCB4EE488A00220123F1EE72
:1021600010FACDE900238DED050ACDED060A9FEDAD
:102170000A0A0A488DED071AF0EE680A68BF13468E
:1021800005A90DF029FD284609B0BDEC028B30BD34
:10219000E02E65420000C84200000000FC800020E4
:1021A00007B50191FFF79AFF30B10199044803B0D8
:1021B0005DF804EB00F0F6BA03B05DF804FB00BF75
:1021C000802C002001486EF09DB900BFD04D00204A
:1021D00008B500F5405090F8E030C3F340128A4251
:1021E0000BD061F3451380F8E03031B156F01EF8A2
:1021F000BDE808400F2155F055BF08BD70B500F58A
:1022000040560546D6F820318B420C4612D00129A3
:1022100011D0022916D059B956F008F81B2155F0F3
:1022200041FF0D4A05F53A500621383058F0FAF8CA
:10223000C6F8204170BD55F0F9FF1A2155F032FF64
:10224000064AEFE7012100F057FE55F0EFFF1D2190
:1022500055F028FF024AE5E750D30C0865D30C0877
:1022600060D30C0810B500F540520C4692F80531C9
:1022700003F00101A14209D064F3000382F80531A3
:10228000DB0704D405F038FF024B9C7210BD06F04A
:1022900019F9F9E7BD86002000F5405090F80531A6
:1022A00061F3410380F80531014B1973704700BF9A
:1022B000BD86002010B5044660F090FC202161F03E
:1022C00003FD04F54053003893F8E22018BF0120C5
:1022D00060F3820283F8E22010BD000010B50446CE
:1022E00053F09EF904F54052436FD2F8102104F5E3
:1022F0008044D360D4F81C2D9366D4F8242DC2F802
:10230000FC32D4F81C0D03685B6D9847D4F81C0DA3
:102310000368BDE810409B6D1847000070B52DEDB7
:10232000028B00F540550446D5F8103193F8CB30B8
:10233000002B71D095F9E030002B6DDB00F5804665
:1023400096F8E83E002B67D1D5F8EC0003685B698E
:102350009847002860D1324BD3F8EC0003681B6823
:1023600098470B2858D0D6F8243D9FED2E7AD3ED10
:10237000DB7AF0EEE77AF4EEC77AF1EE10FA4BD59D
:10238000D5F81001443057F083FB0346DFED260AF1
:1023900093ED000A9F20B7EE001A2CF083F9B5EEFA
:1023A000C00AF1EE10FA37DD04F59A4088F04AF8D9
:1023B000DFED1E7AB0EEC00AB4EEE70AF1EE10FAD5
:1023C0002AD504F58054D6F81C0DD4F8A83407EEAD
:1023D000903A0368D3F89830B8EEE78A984738EE19
:1023E000400ADFED137AB0EEC00AB4EEE70AF1EE70
:1023F00010FA11D5D4F8AC3440F2E63203F2F313FC
:10240000934209D8BDEC028BD5F810019FED090A63
:10241000BDE870408AF038BABDEC028B70BD00BFD9
:10242000805C0020000000340000000000007042CA
:102430000000FA430AD7233C08B500F54050D0F815
:10244000100103681B699847F6EE007A20EE270A10
:10245000B5EEC00AF1EE10FA48BF9FED010A08BDC3
:102460000000000038B52DED028B00F580450446D4
:10247000D5F81C3DDFED110A93ED370A04F5405401
:102480007120B7EE001A2CF00DF9D4F81001D5F830
:10249000245D03681B69B0EE408A984738EE400A15
:1024A000BDEC028BDFED067A05F50575284620EEBA
:1024B000270ABDE8384078F0B9BC00BF0000000032
:1024C00000007A4400F5A853D3ED005AD2ED007A0B
:1024D000D3ED036A91ED006A26EEE77A67EEA57AFE
:1024E000A6EE257AE6EE267A81ED007AC2ED007A34
:1024F0007047000000F50050B0F98C3B33B9B0F9DB
:10250000E2020028B8BF404280B2704783EAE3701D
:10251000A0EBE370F8E7000070B52DED028B00F53D
:10252000405382B093F8051111F00106044605D01E
:102530009FED2E0A02B0BDEC028B70BD8DED010A3D
:1025400060F04CFB037F002BF2D0DFED298ADFED3A
:10255000270A9DED010AB0EE681A4E202CF0A2F871
:1025600004F500554FF4C8723146B5F9EA02B0EEF1
:10257000408A2CF0D5F8A5F8EA02204611F006FBB7
:10258000B5F9EA3207EE900AB8EEE77A07EE903A2C
:10259000F8EEE77A77EE676AB4EEE68AF1EE10FAC3
:1025A0000DD52046FFF7A6FF07EE900A38EE668AA3
:1025B000B8EEE70A20EE088A88EE260ABAE777EE38
:1025C000877AB4EEE78AF1EE10FAB1DDB5F9E232BE
:1025D00000EE103A38EE678AB8EEC00A78EEE77A75
:1025E00020EE088A88EE270AA4E700BF000000005A
:1025F00000007A44002070470020704770470000B8
:1026000000F50B5038307047004870474C030D08F8
:1026100000F54050D0F8EC0003681B681847000034
:10262000034808603221117008221A60704700BF09
:102630000CD70C0800F54050D0F8EC000368DB6CB8
:102640001847000000F54050D0F8EC0003689B6C80
:102650001847000000F5405300F59F40D3F8EC30D8
:1026600008301B1A584258417047000010B500F559
:1026700040500C46D0F8EC000368DB6D984707EE3D
:10268000900A9FED057AF8EE677A012067EE877A67
:10269000C4ED007A10BD00BF0AD7233C10B500F589
:1026A00040500C46D0F8EC0003689B6D984707EE4D
:1026B000900A9FED057AF8EEE77A012067EE877AB7
:1026C000C4ED007A10BD00BF0AD7233C10B500F559
:1026D00040500C46D0F8EC0003681B6E9847DFEDC5
:1026E000047A20EE270A012084ED000A10BD00BF05
:1026F0000AD7233C67F0A2B86AF0EABC62F01ABDC0
:1027000052F0D8BE29F008BF55F048B818F042BBC7
:1027100063F090B85FF0BCBE5DF0C6BF10F0CEBEF7
:1027200011F028BB06F0B8BD12F040BB05F038BD73
:1027300005F084BA05F0AAB968F000BE10F00CB834
:10274000FFF7ECBD10F0FEBF11F06CBA03F03EB91C
:1027500010F082BF10F0FABE60F08EB94BF0D4BC1E
:1027600024F034B906F064B902F0F8BC63F072B832
:1027700011F076BA06F048BD04F05EB906F0A0BECE
:1027800005F016BA06F004BA10F024BEFFF7A6BD95
:102790002AF0E0B905F014BF0AF072BA0AF05CB989
:1027A0000AF0F0B81FB500F540530446D3F8EC002A
:1027B000039103685B6A984760B1DFED070A0399EC
:1027C000002304F5A8400093B0EE600A1A467C305E
:1027D0000DF058F804B010BD0000000010B52DED4C
:1027E000028B00F540530446D3F8EC0003685B6AA3
:1027F000B0EE408A984720B90024BDEC028B2046F9
:1028000010BD9FED080A04F5A84028EE000A7C30B0
:102810000CF002FB04460028EED003480121FFF72C
:10282000D7FCEAE70000C842802C00200A4A92F94F
:10283000E020002A0B4605DA00228A604A600A601E
:102840000120704700F58040D0F81C2D783207CA6F
:1028500083E80700F4E700BF805C002070B5204BE0
:10286000036000F500531F4AC3F8B82E00F540532B
:102870000446586F08B11AF04DFE1B4B236004F557
:10288000805393F8342F42B9D3F8305F2DB12846E6
:1028900028F04AFC28461AF039FE04F58D501C3009
:1028A0007EF052FC04F58650043062F077FE04F6A8
:1028B000F44504F69446B54204D0183D284628F065
:1028C00089F8F8E7094BC4F8C83804F6C41056F084
:1028D000BBFD04F5136056F0B7FD204670BD00BF88
:1028E00004DB0C08A4E50D0848C60D0814900D087B
:1028F00038B54B4B044640F8043B67F0BFF804F191
:10290000100017F0E3FE04F1680052F061FB04F5DB
:10291000907022F0BDFC04F58C6016F029FC04F2E6
:1029200084501AF0F9FD04F6C80029F099FC04F56A
:10293000476066F081FE04F554604FF081F904F5BC
:102940007F6054F00DFD04F5855008306CF030FFC9
:1029500004F58650043062F009FE04F5885019F041
:10296000FDFB04F58D501C307EF0DAFB04F58E5033
:10297000183052F0EFFE04F591500C3068F028FA50
:1029800004F580530025274A83F8505204F59253EA
:10299000103304F5935013604AF016F804F595507F
:1029A0002946103012F03AFE04F5C85078F07CFC4D
:1029B00004F5EE5004307BF0E5FB04F5F6501C30D6
:1029C0007DF008FD04F5FA507EF03EF904F5FC5068
:1029D000183012F025FC04F50350383079F0A0F9D6
:1029E00004F5055010306DF0A5FA04F508501030CC
:1029F0007EF032FF04F5005304F50A5083F8685264
:102A0000094D7FF04BF82B6813B1084890F01AFC81
:102A1000204607494DF0D2FF2C60204638BD00BF4C
:102A200048C60D08A0900020A887002074D30C0889
:102A300050C50D0810B511F01DF860F0CFF803680F
:102A4000BDE810405B681847FFF7F4BF10B50446B7
:102A500006F03AF9204611F013FB204603F03CFE45
:102A60002046BDE8104003F09DBF0000FFF7EEBF19
:102A700070B500F544553C350446284617F000FD76
:102A80001BF010FB90F9213093B390F840337BB3E7
:102A900004F5405304F28456D3F81001443056F044
:102AA000F7FF0346DFED130A93ED000A9F20B7EE10
:102AB000001A2BF0F7FD94F9B835012B284608BF12
:102AC00086ED0E0A002117F06FFADFED0B7A04F2A3
:102AD000DC7494ED287A20EE270ADFED087AA7EE61
:102AE000270A304684ED280ABDE870401BF0EAB999
:102AF00070BD00BF00000000CDCCCC3D6666663FD7
:102B0000FFF7B6BF10B50121044611F0F5FA60B128
:102B1000114BD3F8EC0003689B6A984728B920460C
:102B200002F02AFA204602F037FA4FF4001120464C
:102B300011F0E2FA18B12BF087F829F06DFA4FF492
:102B40008021204611F0D8FA28B12BF07DF8BDE89D
:102B5000104029F06FB910BD805C0020FFF7D2BF94
:102B600070B500F580450446D5F81C0D9FED5A0A56
:102B700086B06C302EF0CAFF04F5955003A91030D2
:102B80008DED030ACDED040A8DED051A12F0F2FB6E
:102B90000221204611F0B0FA70B10121204611F057
:102BA000ABFA48B94D4BD3F8EC0003689B6A9847E1
:102BB00010B9204602F0E0F90121204611F09CFAFC
:102BC00048B9464BD3F8EC0003689B6A984710B9A4
:102BD000204602F0E1F90121204611F08DFA10B9EA
:102BE000204602F031FA4FF40031204611F084FA09
:102BF00030B104F54053D3F8100103685B6C98477B
:102C00004021204611F078FA60B104F57F60019010
:102C100053F064FF04F58053019893F9C4300BB16D
:102C200054F09EF84FF48061204611F065FA18B117
:102C300004F57F6053F0ECFF2021204611F05CFA90
:102C400058B104F54056D6F8EC0003681B69984764
:102C500018B3D5F8240D84F0E1FB8021204611F053
:102C60004BFA38B32AF0F0FF29F008F9102120467A
:102C700011F042FA18B1D5F81C0D81F015F94FF496
:102C80000041204611F038FA18B304F59B403C305F
:102C900006B0BDE8704062F00FBF20460DF0ACFCFE
:102CA0000028D6D1D6F8EC0003685B699847002865
:102CB000CFD0D2E74FF48021204611F01DFA002832
:102CC000D0D14FF40021204611F016FA0028C9D1C6
:102CD000CCE706B070BD00BFE02E6542805C0020EE
:102CE000FFF73EBF10B50121044611F005FA10B1FF
:102CF000204602F0A9F98021204611F0FDF958B1D3
:102D00004FF48021204611F0F7F928B92AF09CFFF2
:102D1000BDE8104029F08EB810BD0000FFF7E2BFFB
:102D200010B5044605F020FD204605F06BFB20465B
:102D300005F060FD204612F0A9F82046BDE81040DD
:102D400003F0A6BCFFF7ECBF70B54FF6FF71044669
:102D500011F0D2F904F5405528B1D5F8E02007214B
:102D6000204602F0A1F9D5F8103193F8CB308BB999
:102D70002046FFF79FFAD5F8100104F500530268CA
:102D800093F87413166A93F8FE22B047D5F8100131
:102D900089F046FD61F082FD61F07EFA204612F076
:102DA00073F895F8E0300F4A04F58044DB43D4F81B
:102DB0001C5DC3F3C01353712B681E6F52F030FCBF
:102DC00052F098F82846B047D4F8244D52F028FC29
:102DD00004F5057452F08EF82046BDE8704077F097
:102DE0008BBE00BFBD860020FFF7AEBF70B500F5FB
:102DF000A85300F540551B68C5F8243100F58056EE
:102E000006F20C5304461B68C5F82831D6F8B00406
:102E100000F58C4050302BF019FCD5F82431C5F862
:102E20003031D5F82831C5F82C01C5F834314FF6CA
:102E3000FF71204611F060F938B1D6F8B024204671
:102E40000921BDE8704002F007B970BD30B500F54A
:102E50004053D3F82041002C4CD093F8E120D10707
:102E600048D56FF3000283F8E12000F50052012CF1
:102E7000D2F8D41CD2F8D85CB1F908400BBFD3ED1E
:102E80004A5AD3ED4D5AD3ED497AD3ED4C7A07EE39
:102E9000104AB5F9084006EE904A0CBFF8EEE66A13
:102EA000F8EEE66AB8EEC77A25EEE66A00F5A853B2
:102EB000A7EE276A67EEA67AD3ED006AE7EE257AD9
:102EC00093ED037A27EE877AA6EE267ABDEEC77ACF
:102ED00017EE104A0C8193ED007AD2F8D82C67EEE9
:102EE000877A93ED037AE6EE477AFDEEE77A17EEFE
:102EF000903A138130BD000038B505462DED028BA8
:102F000000F5405471B1284610F03CFCD4F82C3147
:102F10001B1A03F2F31340F2E63293420CD8BDECD5
:102F2000028B38BDD4F82031022BF8D110F00EFC02
:102F3000B0F57A7FE7D2F2E7C4F82C0100F58C40B7
:102F40005030642390FBF3F308EE103ADFED097A7A
:102F5000B8EEC88A28EE278AB0EE480AB3F0C8F85F
:102F600084ED4C0AB0EE480AB3F048FA84ED4D0AFD
:102F7000D5E700BF35FA8E3C00F5955001211030A1
:102F800013F0CEBFFFF7F8BF10B5044610F004FEF3
:102F90001021204611F0B0F870B1204601F048FF32
:102FA0004FF40011204611F0A7F828B92AF04CFE82
:102FB000BDE8104029F030B810BD0000FFF7E4BFB5
:102FC000F8B50446254606F0A3F9224B45F83C3BEC
:102FD000214BA465C4E91734204BC4E91934204BB4
:102FE000E36604F1800019F005FF04F19C0019F07C
:102FF00001FF04F1B80019F0FDFE4FF6FF76194B02
:10300000C4F8CC30A4F8D06004F1D40019F0F2FE7A
:103010004FF0FF37144B1549C4F8307128461D6036
:103020004DF0CCFCA4F87870A4F8946004F5A2707C
:1030300019F0E0FE04F5B07019F0DCFE04F5BE7086
:1030400019F0D8FE002384F89031C4F8B43120463A
:10305000F8BD00BF00300D08992701089D27010821
:10306000A12701080000FFFF88860020F89C0D08BA
:1030700010B5044606F04CF90A4B23600123A387E0
:1030800004F1400019F0B6FE04F1500019F0B2FE50
:1030900004F1600019F0AEFE04F1700019F0AAFE10
:1030A000204610BDE4390D082DE9F047044688B0EC
:1030B000FFF71EFCA44B236004F50C50203004F5F0
:1030C000005502F027F904F50B532C3304F5335661
:1030D000C5F8E83C062385F8EC3C4FF07C5705A981
:1030E00006F13800059756F0C5FD06F150008FF047
:1030F0008BFA002304F59A4985F8283D192304A981
:1031000085F8343D04F53456C5F8309D04F5355046
:10311000049756F0AFFD06F158008FF075FA0126BE
:10312000182304F5365004F5375785F87C3D3837B9
:1031300085F8706DC5F8789D103061F029FE38462D
:103140007EF068FD814B8DF8186006AEC5F8F83D3D
:103150003146381D4EF050FA04F5385030304AF000
:1031600091FF04F5395030307EF03EFD784B794FB9
:10317000C5F8703E04F53A5031460830069756F0CF
:1031800079FD04F53A5031461430069756F072FD39
:1031900004F53A503146203004F53A5A06970AF1C0
:1031A000380A56F067FD6C4BC5F8B83E0AF11400BA
:1031B0008FF02AFA04F53B5704F53D58303708F1F3
:1031C0001408384614375BF037FBB845F9D104F5DD
:1031D00040580723C8F878300023A8F87C304FF413
:1031E000CB701AF091F9C8F8740004F542508FF0D2
:1031F0000BFA04F5435004308FF006FA574B1A6867
:103200000AB9C3F800A004F5AC47554BC5F8B83E61
:10321000643704F54350C8F8EC7030307FF0D4FFC9
:10322000504B07934FF07E554F4BC8F82451C8F8C8
:1032300030510694009304F5445096E80C004FF486
:1032400000713C3016F062FD04F55A50303070F0D9
:1032500019FE04F5994003A95030039556F030FD4E
:1032600004F5994003A96430039556F003FD04F575
:10327000994004F58045703019F0BCFD05F60C53FB
:103280000026C9F80060C9F80460C9F808601E602B
:103290005E609E6004F595531033C5F8183D04F543
:1032A0009A40002385F8393D4FF400413C3017F037
:1032B000F7FA04F59B403C3062F0A6FA04F59C4016
:1032C00040306EF06DFF04F59C407C304EF0CAFA41
:1032D000264BC5F87C3E04F59D40254B2549103012
:1032E00004F59D48186008F130084DF067FBFF2396
:1032F00085F8C03E85F8C83E1F4940464DF05EFB4C
:103300001E4A136813B11E488FF09CFF1D491E48CA
:10331000C2F8008004F59D42583208604FF0140E48
:103320001FFA83FC0EFB0C010133097C0029F7D145
:10333000164BA3F800C0164BD3F80080B8F1000F6D
:103340002AD01448E0E700BF04DB0C08FCD20C08CC
:103350003CD30C080000A040A4E50D08F08A002032
:1033600084DB0C0895270108F4DA0C084CD30C0810
:10337000A890002070FA0D08448D0E083C910020A2
:1033800088D30C08648700206C1D0D08608700201E
:1033900018870020A9D30C0804F59D401A6003A9E2
:1033A000584B03936C3056F065FC04F59E400C308E
:1033B00005F0AEFF544BC5F80C3F04F59E404C3071
:1033C00005F0A6FF04F5A249504BC5F84C3F04F5A3
:1033D0009F4009F16009083004F5A045FFF7F0FDB2
:1033E000484605F095FF4A4BC5F8603109F13C00AD
:1033F0008CF0EEFD474BC5F89C3104F5A64020301B
:1034000005F086FF444BC5F8203304F5A640643030
:1034100005F07EFF414BC5F8643304F5A74085F8FD
:10342000A083243005F074FF3D4BC5F8A43304F5A8
:10343000A740603005F06CFF3A4BC5F8E03305F269
:103440001C4304F5A8401E605E609E60343005F0A9
:103450005FFF354BC5F8343404F5A840C5F87084D7
:103460007C3005F055FF314BC5F87C3404F5A9409C
:10347000C5F8B884403005F04BFF2D4BC5F8C0347B
:1034800004F5AA40083005F043FF2A4BC5F808357B
:1034900004F5AA40443005F03BFF274BC5F84435FE
:1034A00005F2BC5304F5AB401E605E605830FFF778
:1034B000DFFD384605F02CFF204BC5F8643604F5D7
:1034C000AD40203005F024FF1D4BC5F8A03604F5B3
:1034D000AD40A5F8DC867030FFF7CAFD194BC5F882
:1034E000F036012385F8793704F5AF4318461E609E
:1034F0005E609E600C300AF04BFD204608B0BDE8CF
:10350000F08700BFCDCC4C3DF82B0D089C2C0D084E
:10351000A4300D0834310D08F0310D0890320D083B
:1035200030330D08C8330D0804360D08A4360D08D5
:1035300034370D08CC370D086C380D08403B0D08AA
:10354000DC3C0D089C3A0D0838B5054B1C68236817
:103550000A461D68034B01462046A847002038BD97
:10356000E0840020802C002010B58FF0C3FA064CB8
:10357000064B18602046FFF797FD2046044A054990
:10358000BDE81040B2F08EBC802C0020E08400200A
:103590005CE400205D2801080120704790F89C3011
:1035A0008B4286BF283150F8210000207047000070
:1035B00090F89C308B4286BF283150F821000020C3
:1035C00070470000FA207047014B93F8AE02704735
:1035D000804C0020034BD3F82001431E5842584131
:1035E000704700BF805C0020034BD3F82001831E8E
:1035F00058425841704700BF805C0020034BD3F80D
:10360000100108B187F0B6BF01487047805C002008
:1036100070DB0C0838B5C36A2E4D43F4E052C26229
:10362000026B42F4E0520263426B42F4E0524263A6
:10363000D5F8242D0446E2B143F4F843C362D5F82B
:10364000240D83F0ABFA38B1236B43F4804323633A
:10365000636B43F480436363D5F8240D83F0C0FBB0
:1036600038B1236B43F400532363636B43F400537B
:103670006363194B1D6845B1192128464EF0BAFB0A
:1036800018B1E36A43F48073E362144B93F8F03C9F
:103690006BB1236B43F48073236345B11921284632
:1036A0004EF0E0FB18B1636B43F480736363E36A2D
:1036B00043F08043E362236B43F080432363084B72
:1036C000D3F8103193F8C1301BB9636B43F08043DA
:1036D000636338BD806C002074870020804C00201C
:1036E000805C002013B54FF44470CDE9002119F03F
:1036F00005FF044628B1DDE900215DF0A7FF024B7C
:103700002360204602B010BDC8DD0C0800207047C1
:10371000704700000320704708207047014B93F862
:10372000B0027047804C0020034B93F968030038C7
:1037300018BF0120704700BF804C0020014B93F957
:10374000B2027047804C00207047000070470000B4
:1037500008B50C4BD3F8240D70B910230A4AD2F8DF
:10376000102143F0400022B192F8CB200AB143F07F
:10377000C00040F0010008BD83F010FA0028ECD032
:103780001823EBE7806C0020805C002038B5C578FA
:103790000B46352D044628BF352535220021184615
:1037A000B5F0EEF82A4604F10C01BDE83840B5F05A
:1037B0009DB800001FB5184C94F8E610A4F16800FD
:1037C00011F01AFD78B194F8E610A4F1680011F038
:1037D00015FD40B194F8E610A4F1680004B0BDE80E
:1037E000104011F00DBD002301930293039313F0D9
:1037F00033FC01A913F0FCF920B101A82EF084FDDF
:1038000004B010BD23F020F990F8F432B02202FB8E
:10381000030090ED3B0AF3E7804C002008B50D4B08
:10382000D3F81001A8B1443056F032F9034693EDB5
:10383000000ADFED090A9F20B7EE001A2AF032FFD6
:10384000DFED067A20EE270ABDEEC00A10EE103A30
:1038500018B208BD805C0020000000000000C842D3
:103860002DE9F04FDFF8D880344F8DB004460425A1
:1038700008F5005617F8019BB8F9083309F1FF3A2B
:1038800043FA0AF3D90742D5207C57F095FD8346C9
:10389000207C58F095FC00F121039B4505D2207C4B
:1038A0000DB0BDE8F04F56F0DDBFBAF1030F2ED8D2
:1038B000DFE80AF00234393ED6F81C0D03689B6835
:1038C000984700F194035A69D3F800A0D3F804E0B4
:1038D000D8681969D3F818C008925A6A1B6ACDF8DB
:1038E0002520CDF8293062222123CDE9003206902F
:1038F0000791207CCDF80CA0192303AAC221CDF892
:1039000010E0CDF814C08DF8249057F0BFFD013DB4
:1039100015F0FF05AED10DB0BDE8F08FD6F81C0D47
:103920000368DB68CCE7D6F81C0D03681B69C7E7A2
:10393000D6F8243D03F52A73C5E700BF9CDE0C08CA
:10394000804C002013B504460748019108F0CCFFD5
:1039500030B90199204602B0BDE8104058F070BE61
:10396000042002B010BD00BF087C0020014808F010
:1039700097BD00BF087C002037B504460D460648B9
:10398000019211468BF0E8F8019A2946204603B0CF
:10399000BDE830405CF028BD1858002010B588B054
:1039A00004465AF04BF80C4BD3F8100138B90B4AC7
:1039B0000621204608B0BDE810405AF027B86946F5
:1039C0001E2287F0DBFD064A6B46062120465AF090
:1039D0001DF808B010BD00BF805C0020BCDB0C08E7
:1039E00076290D08034A92F8D03C013382F8D03C86
:1039F00059F0E8B8804C002007B50846019119F04D
:103A0000CFFA38B10448019902F0DEFC002003B07F
:103A10005DF804FB0420FAE7EC840020F7B58B8BFB
:103A2000CD2B06460C4617461DD1D1ED067AFCEE8D
:103A3000E77ACDED017A9DF80430022B13D10E4DBB
:103A400095F8351E05F6BC5061F014FF58B195F895
:103A5000351E05F6BC5061F015FF20B994ED020A41
:103A6000064802F091FC3A462146304603B0BDE8D4
:103A7000F04059F039B900BF806C0020EC84002080
:103A8000162A10B40C4605D0542A03D05DF8044B16
:103A900058F0F2BD0323237001205DF8044B7047FA
:103AA00008B559F045F840F41C6040F00D0008BD21
:103AB00010B5044619F02AFD204610BD10B50C4C77
:103AC00094F9E030002B0FDBD4F8EC000368DB6CDA
:103AD000984758B9D4F8EC0003689B6C98470028C5
:103AE0000CBF0220032010BD0120FCE70420FAE7F0
:103AF000805C002010B44C69012C05D101465DF8B2
:103B0000044B034802F0F4BF5DF8044B59F074B85D
:103B1000802C00202DE9F341B1F90430002B06463A
:103B20000C46154635DB4FF00008CDE900281A4F4A
:103B3000B1F902209FED190AD7F8D41C4FF47A731B
:103B40005CF03AFF0123CDE900539FED140AB4F96C
:103B50000020D7F8D81C4FF47A7330465CF02CFF65
:103B60009FED0F0AB4F90420D7F8DC1C4346304619
:103B7000CDE900585CF020FFCDE900589FED070A21
:103B8000B4F90620D7F8E01C4FF47A7330465CF0A5
:103B900013FF02B0BDE8F081804C00200000FA4421
:103BA00000007A44044B187820B9044B93F8E200E3
:103BB000C0F38010704700BF58860020805C002052
:103BC0000B4B93F8AD267AB993F8052192060BD1E9
:103BD00093F9E020002A09DB93F8E13013F0200F7D
:103BE00014BF042001207047052070470320704750
:103BF000805C002008B5074B93F9FC32032B03D0FF
:103C0000BDE8084059F07ABF034A022159F0FEFE90
:103C1000042008BD804C0020D4DB0C08094BD3F8ED
:103C20006C23920701D458F01BBD03F5005303F633
:103C3000F44393ED000ADFED047AB8EEC00A20EEFB
:103C4000270A7047804C00200AD7233C10B594B057
:103C5000044603A819F0CEF81C4BD3F8EC00036817
:103C600003A95B6D984778B3002103A819F05AF9AE
:103C700050B3247C8FF014FB059BDDED047A089390
:103C8000069B09930023F8EEE77A9FED117A0B93D8
:103C90000C930D930E930F931093119312934FF671
:103CA000F853ADF84C300023962267EE877A8DF8F2
:103CB0004E303323CDE90032079007AA5721204622
:103CC000CDED0A7A57F0E2FB14B010BD805C002005
:103CD0000AD7233C30B52DED0A8B774C0546D4F836
:103CE000EC00036899B05B6A984700285BD004F544
:103CF0000054D4F8B834062B00F2C980DFE803F092
:103D00000404045788AB53006C489FED6D8A0BF098
:103D100081FF9FED6C0A0168426883680D930BA8D0
:103D20000B910C922DF0F2FEF0EE489AB0EE40CAE4
:103D3000F0EE60BAB0EE419AB0EE48AAF0EE488AD2
:103D4000F0EE48AAB0EE48BA40F6F8542D7C8FF059
:103D5000A7FA00231593169301238C228DF85E3069
:103D60003323CDE900320B90B1EE499AF1EE688A27
:103D7000B1EE488A0BAA552128468DED0CCACDED2F
:103D80000DBA8DED0E9A8DED0FBACDED10AACDEDD9
:103D9000118A8DED12AACDED139A8DED148AADF82E
:103DA0005C4057F073FB19B0BDEC0A8B30BD434843
:103DB0000BF030FF9FED430A0168426883680D9362
:103DC0000BA80B910C922DF0A1FE3C48F0EE60BACE
:103DD000B0EE419AB0EE40CA0BF020FF9FED390AD9
:103DE0002DF094FE3548B0EE40BAF0EE60AAF0EE49
:103DF000418A0BF017FF9FED330A2DF087FE4FF439
:103E00004064B0EE40AAF0EE609AB0EE418A9DE7C1
:103E10002A489FED2B9A0BF001FF9FED2A0A2DF007
:103E200075FE2648B0EE40BAF0EE60AAF0EE418A88
:103E30000BF0F8FE9FED230A2DF068FEF0EE49BA74
:103E4000B0EE40AAF0EE609AB0EE418AB0EE49CAF8
:103E500040F607447AE71948DFED198A0BF0E2FED5
:103E60009FED180A2DF052FEF0EE68AAB0EE40AABF
:103E7000F0EE609AB0EE418AB0EE68BAB0EE689AA1
:103E8000F0EE68BAB0EE68CA40F63F445EE79FEDD8
:103E90000C8A0024F0EE489AB0EE48AAF0EE488A68
:103EA000F0EE48AAB0EE48BAB0EE489AF0EE48BA42
:103EB000B0EE48CA4AE700BF805C0020FC800020CA
:103EC000000000000AD7233C2DE9F0412DED068BC0
:103ED0003B4D95F8E13099068CB004466AD505F55E
:103EE00080579FED380AD7F81C0DDFED378A6C300C
:103EF0002DF00CFE8DED041A21EE281AD5F8EC6099
:103F00008DED020ABDEEC11ACDED030A11EE103A95
:103F10001DB2336894F810809B6D304660EE289A8D
:103F200020EEA89A984707EE900AF8EEE77A304616
:103F300067EEA87AFDEEE77A17EE903A1CB2336886
:103F4000DB6D984707EE900AB8EE678AD7F8243DF4
:103F5000DFED1E7A93ED0FAA336828EE288A1B6ED8
:103F6000B4EEE78AF1EE10FA58BFB0EE678A304639
:103F70009847BCEEC88A0023089318EE103AB7227F
:103F80002AEE28AA20EE280AADF82C301A23CDE913
:103F900000323E2105AA4046CDED059A8DED069AE8
:103FA0008DED07AA8DED090AADF82850ADF82A402D
:103FB00057F06CFA0CB0BDEC068BBDE8F08100BF89
:103FC000805C00209F0CB3450AD7233C00FF7F474D
:103FD0002DE9F04F2DED028B1A4B047CD3F81C3DDC
:103FE0008DB0D3F88480D3F88870D3F88C60D3F880
:103FF000905093ED258AD3F898B0D3F89CA0D3F8CD
:10400000DC908FF04DF900238DF82C3016222523FB
:10401000CDE90032029002AA532120468DED078A95
:10402000CDF820B0CDF824A0CDF82890CDF80C80A4
:1040300004970596069557F029FA0DB0BDEC028B52
:10404000BDE8F08F806C002070B58A7A4B7A43EA25
:104050000223CA7A43EA02439D2B06460C4621D12D
:10406000134D95F8351E05F6BC5061F003FCC8B140
:1040700095F8351E05F6BC5061F010FC022811D1F0
:1040800095F8351E05F6BC5061F0FCFB50B9D4ED37
:10409000057A9FED080A0848F8EEE77A27EE800ACD
:1040A00002F072F921463046BDE8704058F08ABCF3
:1040B000806C00200AD7233CEC840020054BD3F809
:1040C00010312BB193F8CA00002808BF02207047B6
:1040D00002207047805C002008B5034BD3F8EC0049
:1040E00003681B68984708BD805C0020024B93F86A
:1040F000E100C0F340107047805C002070B52C4E8A
:104100002DED028B0546D6F8EC0091ED018A03688F
:1041100086B05B6A0C46984750B9BDEEC88A18EE67
:10412000103ADB0704D4022006B0BDEC028B70BD50
:10413000D4E904012BF044FB0028F4D002A818F0C5
:1041400059FE02AA214628465CF0A6FB0028EAD0C8
:10415000184902A818F030FF03460028E3D1DFED2C
:10416000160A00900246B0EE600A144802A90BF04D
:1041700089FBD8B1D6F8EC0003685B6A984704461F
:1041800008B10020D0E70E480222042105F058FCB7
:1041900060B1DFED090A094800942346B0EE600AD9
:1041A000224602A90BF06EFB0028EAD10420BBE7EF
:1041B000805C00207079002000000000FC8000205E
:1041C000802C002008B591F82030032B1CD1D1EDB4
:1041D000027A9FED0E7A91ED060A0D4BF0EEE77A2A
:1041E000F4EEC77ADFED0B7AD3F8EC00F1EE10FABB
:1041F0004CBF0121002120EE270A10F095FA00287B
:1042000014BF0020042008BD0220FCE70000003499
:10421000805C00200000C84210B52DED028BD1ED6E
:10422000007AF5EEC07AF1EE10FA82B00C4604DAAC
:10423000042002B0BDEC028B10BD9FED197AF4EEA4
:10424000C77AF1EE10FAF3D891ED030A9FED158AC3
:10425000F0EEC07AF4EEC87AF1EE10FA19D5D4ED8A
:10426000037A1148D4ED010A94ED000AF4EEC87AFD
:10427000D4ED027AFDEEE77AF1EE10FACDED017A97
:104280009DF90410ACBF0122002201F0DFFF0020E5
:10429000CFE7F7EE000A2AF001F90028C8D0DEE7E0
:1042A0000000B44300000034EC84002091ED010ACA
:1042B000B5EEC00AF1EE10FA08B501DC042008BD25
:1042C0009FED107A104BD1ED007AD3F8EC0020EE80
:1042D000070A9FED0E7A0368F4EEC77AF1EE10FA42
:1042E00005DDDB6E98470028E8D00020E7E79FED6A
:1042F000087AF4EEC77AF1EE10FACCBF9B6E5B6ED3
:10430000F0E700BF0000C842805C00209A99394065
:104310003333F33F08B5D1ED007A9FED157AF0EE17
:10432000E77AF4EEC77AF1EE10FA1DD5D1ED017AF5
:10433000F0EEE77AF4EEC77AF1EE10FA14D50D48F4
:104340000222032105F07CFB80B10A480121FDF720
:104350003FFF094890F8C83F012B03D000F6C47016
:1043600030F04CFF002000E0022008BD0420FCE7F4
:1043700000000034802C0020806C002010B5D1EDAE
:10438000007AFCEEE77A17EE903A9CB2012C02D04C
:10439000022C06D04CB90648214667F051F900209E
:1043A00010BD044803F05CF9F9E70420F8E700BF0A
:1043B000107B0020802C00201FB5D1ED017A0B7CF2
:1043C000FCEEE77ACDED027AD1ED007A0093FCEEB7
:1043D000E77AD1ED030ACDED037A91ED020A9DF85B
:1043E00008309DF80C20014602480EF059FF05B038
:1043F0005DF804FB802C002010B50A4C94F80531C0
:10440000DB070CD402220521A4F5405005F018FB6F
:1044100028B902221146A4F5405005F011FB0020F6
:1044200010BD00BF805C002010B5D1ED007AFCEE1D
:10443000E77A044617EE903A13F0FF030FD10F4BC3
:10444000D3F8EC0003689B6F984708B1002010BDBB
:104450000B4A2046062159F0D9FA0420F7E7012B30
:1044600009D1064BD3F8EC000368DB6F98470028AE
:10447000ECD1044AEDE70220E9E700BF805C0020B0
:10448000F8DB0C0808DC0C089FED0B7A01F10C033B
:10449000F1EC017AF4EE677AF1EE10FA0AD6F0EE5A
:1044A000E77AF4EEC77AF1EE10FA03DC9942EFD125
:1044B000012070470020704700007A4430B52DED90
:1044C000028B8DB00023054603930493059312F0ED
:1044D000C3FD03A912F08CFB58B312F0BDFD00F52B
:1044E0005A7393E8070006AC84E80700DDED060A7E
:1044F0009DED070A2D7CF1EE600AB1EE400AB2F0A4
:1045000049F82046B0EE408A2DF0FEFEDFED0B7A32
:10451000089B0B93012228EE278A0C23CDE9003259
:10452000A82109AA28468DED098A8DED0A0A56F0C0
:10453000ADFF0DB0BDEC028B30BD00BFE02E65427B
:10454000242938B505460FD003D81B2907D10124EB
:1045500012E04029FBD0A1F14203012BF7D92846F4
:10456000BDE838405CF084BB0C2156F08DF9044660
:1045700010B12846FFF7A2FF204638BD38B5194CC8
:1045800094F80531DB070D460AD4D4F8103193F8BE
:10459000CB303BB901221146A4F50270FDF76EFC49
:1045A000002038BD94F9E030002B4FF0020212DAFF
:1045B0000521A4F5405005F043FA0028F0D095ED10
:1045C000000ADFED097AD4F8EC0020EE270A012179
:1045D00010F0AAF8E4E70921A4F5405005F030FAFC
:1045E000DEE700BF805C00200000C84210B5214C0F
:1045F00094F80531DB070ED4D4F8103193F8CB30A2
:104600004BB194F9E030002B07DA01220821A4F520
:104610000270FDF7E7FC002010BDD1ED007A9FEDA0
:10462000167AF0EEE77AF4EEC77AF1EE10FA0BD5CF
:1046300012480222112105F003FAA0B90222114604
:104640000E4805F0FDF9E6E7D4F8EC0003681B68B6
:1046500098470428DFD0D4F8EC0003681B6898471B
:104660001428E5D1D7E7064840F6C41108F03EFE0D
:10467000D1E700BF805C002000000034802C0020C7
:10468000A07F002073B58B8BC12B05460C4644D808
:10469000BB2B0DD8202B63D02ED8113B99B2052906
:1046A00018D92146284602B0BDE870405DF0D2BB63
:1046B000BC3B052BF5D801A151F823F0FB470108BD
:1046C00005480108A3460108A346010893470108CD
:1046D0009F470108052BE4D801A151F823F000BF42
:1046E000E1470108A3460108A3460108F547010870
:1046F00007470108B5470108732B2CD006D8542B67
:1047000058D0552BCDD1022209216BE0B22BC8D154
:1047100002B0BDE87040FFF7C9BD4AF21146B3428E
:1047200054D00BD8D12B40D0B3F5967F53D0D02B9B
:10473000B7D102B0BDE87040FFF720BE4AF2124682
:10474000B3423ED04AF21346B342AAD102B0BDE80A
:104750007040FFF74BBF02B0BDE87040FFF75CBD93
:10476000D1ED007AF5EEC07AF1EE10FA4FDD9FED53
:10477000297AF4EEC77AF1EE10FA48D8FCEEE77A1F
:10478000254ACDED017A9DF80430A2F89A3B00202D
:104790002EE0214602B0BDE87040FFF7AFBC2146D5
:1047A00002B0BDE87040FFF73FBE02B0BDE8704008
:1047B000FFF702BE2146284602B0BDE87040FFF771
:1047C00001BD02B0BDE87040FFF7D8BE02B0BDE841
:1047D0007040FFF711BE02B0BDE87040FFF79ABD10
:1047E000022205210D4805F02BF90028CFD1042025
:1047F00002B070BD02220621F4E70221084806F04B
:1048000097FAF2E70221064806F05CFAEDE702208B
:10481000EEE700BF00007F43804C0020802C00208A
:10482000087C002008B591ED007AF6EE007AB4EE2F
:10483000E77AF1EE10FA06DD044801220521FDF7C2
:10484000D1FB002008BD0420FCE700BF785A0020FF
:1048500030B52DED028BCD7893B0272D28BF2725BD
:104860000C462722002108A8B4F08AF82A4604F151
:104870000C0108A8B4F03AF8424BD3F8EC000368F6
:104880005B6A9847002841D09DF8465068063DD4A1
:1048900000244FF07E532906049307940694059450
:1048A00027D504A82CF0DCFBEA07019402940394BA
:1048B00005F006032ED4002B2ED10D9B01930E9BE9
:1048C00002930F9B039330480AF08AFD9DED100A76
:1048D000044630B340F2ED40B7EE001AFFEE000A96
:1048E00029F0E0FE2848234601AA04A90AF080FD29
:1048F0000CE0099B04930A9B05930B9B069304A869
:104900000C9B07932CF0B2FB0028CDD113B0BDEC6B
:10491000028B30BD062BD6D001211B480AF0FCFCCF
:10492000F4E7DFED1A0A4FF49E60B7EE001A29F0A3
:10493000B9FEF6EE000AB0EE408A29F0AFFDE8B904
:10494000B6EE000A124BB4EEC08AF1EE10FAD3F8BC
:10495000283D08DD38EE400A30EE008A93ED070A64
:1049600028EE000ABEE730EE480AD3ED087A30EEB2
:10497000000AF0EEE77A27EEC00AB3E79FED030ADC
:10498000B0E700BF805C0020FC8000200000000039
:10499000806C00202DE9F0439DB0814608460EA9A9
:1049A000FEF7F4FE844BD3F8EC0003685B6A98478B
:1049B00050B19DF86C30012B09D0DA1F022A06D9BC
:1049C0007E4801210AF0A8FC1DB0BDE8F083BDF8C7
:1049D0006840A20504F0070604F0380704F4E07507
:1049E00001D5002DF0D04FF00008CDF81480CDF89F
:1049F0001880CDF81C803EBB9FED716A9DED107A4A
:104A0000DDED117ADDED0F6A27EE067A67EEC67AE4
:104A100066EE866A083B012BCDED056A8DED067AC0
:104A2000CDED077A04D8674806AA05A9FDF74AFD27
:104A30009DF86C30073B022B06D8634885F0F2FCEA
:104A4000014605A82DF082F8CDF82080CDF824800D
:104A5000CDF82880F7B9DDED147A129B0893F1EEBA
:104A6000677A139B099308A94846CDED0A7AFFF7A8
:104A70000BFD0028A4D09FED520A08A82DF09AF84B
:104A80009DF86C30083B012B04D84E4809AA08A9B0
:104A9000FDF718FDCDF82C80CDF83080CDF83480AE
:104AA000EDB99FED476A9DED167ADDED177ADDEDE4
:104AB000156A9DF86C3027EE067A67EEC67A66EEC8
:104AC000866A083B012BCDED0B6A8DED0C7ACDED9E
:104AD0000D7A04D83B480CAA0BA9FDF7F3FC14F49B
:104AE000806233D1DFED397A9DED180A9DF86C10A4
:104AF00020EE270ADFED327A0839012920EE270A55
:104B00008CBF0021012114F4006305BFDFED2F7A73
:104B1000DDED190ADFED2E0A60EEA70A04BFDFED16
:104B2000287A60EEA70AAEB9002F35D1B3FA83F325
:104B3000B2FA82F25B0952090291019300920BAB27
:104B400008AA05A91D480AF055FD3DE79FED200A7A
:104B50000021D8E77FB9B3FA83F35B090120009302
:104B6000B2FA82F3CDE901105B0914480BAA08A937
:104B70000AF0D8FF28E7002D7FF422AF0120B3FA16
:104B800083F3B2FA82F2CDE900105B090B485209B7
:104B90000BA90AF06FFF17E7002D3FF411AFB3FA2E
:104BA00083F3B2FA82F2CDE900165B09520905A936
:104BB00002480AF0A1FD07E7805C0020FC8000208D
:104BC0000000C842802C002080790020E02E654241
:104BD000000000002DE9F047A2B08046084614A965
:104BE000FEF7D4FD7E4BD3F8EC0003685B6A984770
:104BF000C0B1BDF88040A30504F0070904F4E077D4
:104C000000D57FB10CAE304618F0F4F8B9F1000FC2
:104C100029D1DDE915012AF0D3FD30B97148012110
:104C20000AF07AFB22B0BDE8F0879DF8841009AA4B
:104C300040465BF01BFE0028F0D0DDED177A9FEDBB
:104C40006A7A099B009367EE877A10ADFDEEE77AEA
:104C5000DDE9151217EE903A284618F0EBF895E8C2
:104C60000F0086E80F00002514F0380A0695079516
:104C7000089514D1DDED1A7A189B0693F1EE677A48
:104C8000199B079306A94046CDED087AFFF7FCFB78
:104C90000028C3D09FED540A06A82CF08BFF09957D
:104CA0000A950B959FB99FED506A9DED1C7ADDED3D
:104CB0001D7ADDED1B6A27EE067A67EEC67A66EE90
:104CC000866A8DED0A7ACDED096ACDED0B7A14F482
:104CD000806805BFDFED457A9DED1E0A9FED440A11
:104CE00020EE270A04BFDFED407A20EE270A14F4F5
:104CF000006405BFDFED3D7ADDED1F0ADFED3C0A04
:104D000060EEA70A04BFDFED387A60EEA70AB9F1BA
:104D1000000F31D1BAF1000F52D13046CDED050A66
:104D20008DED040A18F096F803289DED040ADDEDD8
:104D3000050A3FF473AF10A93046CDED050A8DED9D
:104D4000040A10951195129518F0E4F900283FF423
:104D500065AFB4FA84F46409B8FA88F3DDED050AA6
:104D60009DED040ACDF804A000945B0906AA10A9E1
:104D70001C480AF0AFFC55E7BAF1000F0FD1012330
:104D8000B4FA84F4CDE901A36409B8FA88F31548AC
:104D900000945B0909AA06A90AF0C4FE42E7002FA5
:104DA0007FF43CAF0123CDE90073B8FA88F2B4FA7E
:104DB00084F30C485B09520909A90AF05BFE31E74C
:104DC000002F3FF42BAFB4FA84F3B8FA88F2CDF891
:104DD00000905B095209314602480AF053FD21E771
:104DE000805C0020FC8000200000C842E02E65426C
:104DF0000000000010B44B7A8C7ACA7A43EA04238C
:104E000043EA0243542B07D0562B09D0522B0BD127
:104E10005DF8044BFFF71CBD5DF8044BFFF7BABD0E
:104E20005DF8044BFFF7D6BE5DF8044B5CF0EEB9BD
:104E30002DE9F0432DED028B00F540590446D9F8D9
:104E4000EC00DFED4A8A036891B05B69984704F58E
:104E500080470026002840F08480D7F8243DD3ED19
:104E6000DE7A93EDD88AFDEEE77A28EE288A17EEEF
:104E7000903A1DB204F5365801A940460EF0F4FFF1
:104E800018B953F0D3F93A4B01933722002102A805
:104E9000B3F076FDA3238DF8083095238DF8093003
:104EA0008EF006FAD7F81C3DCDF80B00D9F81001AA
:104EB000D3F8DC20D3F8E030CDF80F104430CDF833
:104EC0001320CDF8173054F0E3FD0346DFED290A37
:104ED00093ED000AB7EE001A9F2029F0E3FB10EED5
:104EE000103AD9F81001CDF81B3003681B699847B8
:104EF00010EE103A04F59A49CDF81F3018EE103A2A
:104F00004846CDF8233085F091FA20EE280A404635
:104F100010EE103ACDF82730D7F8CC3CCDF82B3036
:104F2000019BCDF82F300EF0C1FF10EE103A48462D
:104F3000CDF83330CDF83760ADF83B5085F082FACC
:104F4000BDEEC00A372210EE103A02A904F57F60C8
:104F5000ADF83D3052F0BCFA11B0BDEC028BBDE8AB
:104F6000F08308EE106A002584E700BF0AD7233CCF
:104F70002292CA7F0000000010B500F58044D4F8EA
:104F80001C0D7EF03BF9D4F8241DD4F81C0DBDE8AF
:104F900010407EF099B9000070B54FF4805104467E
:104FA0000FF0AAF800284ED004F5804604F57F657E
:104FB000D6F81C0D03689B689847692100F194029C
:104FC000284652F01DF9D6F81C0D0368DB68984797
:104FD0006A2100F19402284652F012F9D6F81C0D0D
:104FE00003681B6998476B2100F19402284652F030
:104FF00007F9D6F8242D6C21284602F52A7252F0C2
:10500000FFF8202120460FF077F8E0B104F5405377
:10501000D3F8EC0003681B69984778B1D6F8242DC3
:10502000284690326E2152F0EBF8D6F8242D28460F
:10503000BC32BDE870406F2152F0E2B820460BF060
:10504000DBFA0028EAD170BD08B512F005F8BDE81A
:10505000084011F07FBD00007FB50E464FF6FF718E
:10506000044615460FF048F8E0B1102200216846CA
:10507000B3F086FCA3238DF8003095238DF8013022
:1050800003238DF802308EF013F91022CDF80300BF
:10509000CDF8071004F57F6069468DF80B60039525
:1050A00052F096FA04B070BD7FB50E464FF6FF7110
:1050B000044615460FF020F8E0B1102200216846A2
:1050C000B3F05EFCA3238DF8003095238DF80130FA
:1050D00004238DF802308EF0EBF81022CDF8030097
:1050E000CDF8071004F57F6069468DF80B600395D5
:1050F00052F06EFA04B070BD30B52DED048B87B060
:1051000004460D46182200216846B0EE409AF0EEA3
:10511000608AB0EE418AB3F033FCA3238DF80030EF
:1051200095238DF8013006238DF802308EF0C0F8FB
:105130001822CDF80300CDF8071004F57F6069460A
:105140008DF80B508DED039ACDED048A8DED058A17
:1051500052F0BEF907B0BDEC048B30BD10B54FF472
:10516000801104460EF0C8FF30B104F595501030A0
:10517000BDE8104010F0D8B910BD00002DE9F04393
:105180008FB01446054689463122002101A8DDE989
:1051900016769846B3F0F4FBA3238DF804309523DC
:1051A0008DF8053008238DF806308EF081F82368DD
:1051B000049363680593A36806933B68CDF81D309C
:1051C0007B68CDF82130BB68CDF825303368CDF849
:1051D00029307368CDF80700CDF80B10CDF82D30CD
:1051E0003122B3688DF80F9001A905F57F608DF825
:1051F0001C80CDF8313052F06BF90FB0BDE8F08370
:1052000070B52DED068B8CB0144605460E462C224B
:10521000002101A8B0EE409AF0EE608AB0EE418A1B
:10522000B0EE61AAF0EE429AB3F0AAFBA3238DF888
:10523000043095238DF805300B238DF806308EF061
:1052400037F8DFED1A7A94ED007ACDF8070027EEF3
:10525000277A29EE279A8DED077A94ED017ACDF819
:105260000B1027EE277A68EEA78A8DED087A94ED69
:10527000027A8DF80F6028EE278A67EE277A2C22B3
:1052800001A905F57F608DED049ACDED058A8DEDC0
:10529000068ACDED097A8DED0AAACDED0B9A52F072
:1052A00017F90CB0BDEC068B70BD00BFE02E654257
:1052B000A020704730B5154B89B004466946D3F835
:1052C000100104F57F651E2286F058F96A461049E0
:1052D000284652F099FA04F54053D3F8EC000368DD
:1052E0001B68984704F50053014693F86822284646
:1052F00052F0AEFA04F59550103012F013F904F59F
:10530000907020F00BFC09B030BD00BF805C002025
:1053100076290D082E4B2F4A70B543600023436158
:105320008361C361C3632C4B426303644FF08042CB
:105330002A4B43640446826358305DF0CFFA284E0E
:10534000284BA365A82560195DF07EFC66513035B9
:10535000B5F56A7FF7D1244D04F56A705FF076F9F0
:10536000002104F2BC7088F0F9FCC4F8705804F60F
:105370007800A5F5BE6589F0C7F99FED1C1ADFED31
:105380001C0A9FED1C0AC4F8085904F61C107EF094
:1053900027FD9FED161A9FED180AF0EE410A04F65C
:1053A00034107EF01DFD9FED111A9FED130AF0EEF3
:1053B000410A04F64C107EF013FD20460F494BF0D5
:1053C000FDFA20460E494BF0F9FA204670BD00BFA9
:1053D000F03800200000C8410AD7233C0000E0401C
:1053E000E0260D08F4260D080C84002000000000C3
:1053F0009A99993E0000B44300804A435C1A0D0814
:10540000DC1C0D0870B54C4D4C49ADF50E7DD0221D
:1054100006465AA8B3F06AFA0FCD0EAC0FC40FCDF2
:105420000FC40FCD0FC495E80F0084E80F000024CF
:105430005AAB18190021B7EE000A10344AF08CFD5F
:10544000D02CF5D13E4B0FCB02AC84E80F0001A964
:1054500020464AF035FD90B19DF90430DFED396A00
:10546000E06807EE103AB8EEC77AF0EE007AE7EEA1
:10547000267AB7EE000A80EE270A4BF047FE00249A
:105480000EAB181900211034B7EE000A4AF064FD83
:10549000402CF5D12C49902236A8B3F027FA0022EF
:1054A000092136A84AF004FE96F9A469D6B9274D19
:1054B0000FCD1EAC0FC40FCD0FC40FCD0FC495E898
:1054C0000F0084E80F00324604211EA84AF0F0FDC8
:1054D0009FED1F0A1F484BF019FE1F48B7EE000A48
:1054E0004BF014FE1D4C9FED1E0A0FCC06AD0FC5F0
:1054F00094E80F0085E80F00002106A84AF02CFD73
:105500009FED170A002128464AF026FD04F11001FC
:1055100060221EA8B3F0EAF900241EAB181900217E
:10552000B7EE000A10344AF017FD602CF5D15EF09A
:1055300019FE0DF50E7D70BD64CC0C0894CB0C08E3
:10554000A4CC0C08CDCCCC3DB4CC0C0844CD0C087C
:105550000000000044190D0853190D0884CD0C08F3
:10556000000034422DE9F04790B00DF106011D20F6
:105570005EF0ECFE002800F09E809DF80630614A47
:105580000133DBB211210BA88DF806308DF062F8E3
:1055900000220DF107010BA84AF018FA9DF8063019
:1055A000594A112105460BA88DF054F800220DF13F
:1055B00007010BA84AF00AFA9DF80630534A112158
:1055C00006460BA88DF046F800220DF107010BA846
:1055D0004AF0FCF99DF806304D4A03F03F031121D3
:1055E00007460BA88DF036F800220DF107010BA835
:1055F0004AF0ECF98046002D5DD0002E5BD0002FE4
:1056000059D0002857D028464AF0F8FB002852D13C
:1056100030464AF0F3FB00284DD138464AF0EEFB05
:10562000002848D140464AF0E9FB002843D1394CD4
:1056300094E80F000DF10C0C10348CE80F0094E886
:105640000F000DF11C0989E80F0002A960464AF01D
:1056500037FC98B3BDF8084002A948464AF030FC30
:1056600000284AD0BDF8083054BB23B340F2E244CE
:105670009C420FFA84FA0FFA83F927D80DF10A0138
:105680003046ADF80A904CF037F80DF10A01284683
:10569000ADF80AA04CF030F80DF10A013846ADF82B
:1056A0000AA04CF029F800230DF10A014046ADF89C
:1056B0000A304CF03BF810B0BDE8F0870024CBE78F
:1056C00040F2D662002B08BF1346D1E70DF10A0164
:1056D0003046ADF80AA04CF00FF80DF10A0128464B
:1056E000ADF80A904CF008F80DF10A013846ADF813
:1056F0000A904CF001F80123D6E7002CDBD040F2F1
:10570000D663B5E764190D0870190D087C190D08EA
:1057100089190D0804CE0C0837B500F50A51782216
:105720002C31044650F0A0FA00220C2126484AF001
:10573000BFFC2046FFF716FF0022B7EE000A022149
:1057400004F50B504AF03CFD012504F505511F4AB4
:1057500000950023103145204AF0AEFC1C4A136826
:10576000D90709D41B49156004F5035338330B607E
:1057700004F585530833CB6004F50C50154902221B
:10578000203001254AF0EAFC134A0095002304F575
:105790007F61FD204AF090FC104B1A68D20705D4B7
:1057A0000F4A1D6004F58E54183414600C48012112
:1057B0004AF0F0FC4BF008FB0A4A138843F001035F
:1057C000138003B030BD00BF9C190D089C870E08E4
:1057D000E484002000220020E4CC0D08E8840020AE
:1057E000182200204C8700200F299DBF302303FB87
:1057F0000100503000207047014B93F9F3027047CD
:10580000804C0020024B93F8050100F00100704726
:10581000805C0020044BB3F8B832DB075ABF006944
:10582000C0F3401000207047804C0020014BD3F89B
:10583000E00C7047804C002008B503689B689847CF
:1058400030B9044B93F90401B0FA80F0400908BD67
:105850000020FCE7805C002038B50D1E2DDB174CC6
:1058600094F8EC2CEBB29A4227D3D4F8E83C01220E
:10587000595DA4F5005004F0E3F8F0B15DF0AEF925
:1058800003215EF021FAC0B95DF0A8F90D215EF0A8
:105890001BFA90B994F9D832EB40DB075CBF94F95E
:1058A000F212E940A4F5005048BF0221BDE838409B
:1058B00058BF01F00101FCF7A1BC38BD804C0020AD
:1058C000022A10B50C4605D1BDE810400948352222
:1058D00004F0B6B8084BD3F8EC0003681B6898478F
:1058E000A04205D15DF07AF9BDE810405DF000B945
:1058F00010BD00BF802C0020805C002029B102294F
:1059000007D1044BC3F8E4107047024B0122C3F8DF
:10591000E4207047805C002031B1022907D1044B9C
:10592000012283F8E8207047014B83F8E8107047A4
:10593000805C002010B500F50053DFED186AD3F845
:10594000D82CD3F8D43CB2F90820B3F908309FED35
:10595000147A07EE902AF8EEE77A0446C7EEA60A14
:1059600000F595500121103007EE903AF8EEE77AF5
:1059700060EE870A87EEA60A20EE070A11F00AFCFD
:1059800052F054FC262152F08DFB04F53A50054AA2
:10599000BDE810400621383054F044BD0000C84234
:1059A00035FA8E3CB0240D0800F58042002382F8C1
:1059B000383D044A00F53A5013720621024A383045
:1059C00054F030BDBD860020BC240D0870B500F534
:1059D0008045044695F8381D002957D02C4B2D4A98
:1059E000D3F8EC00904204D1D3F8103193F8CB30C7
:1059F00023B92046BDE87040FFF7D6BF264E95F884
:105A0000390D04F54053012293F9E0303272D0BBD6
:105A1000002B3BDB85F8392D0139C9B204F5005361
:105A200085F8381DD3F8D82CD3F8D43CB2F9082027
:105A3000DFED1A6AB3F908309FED197A07EE902A64
:105A4000F8EEE77AB1FA81F1C7EEA60A04F59550AF
:105A50004909103007EE903AF8EEE77A60EE870ACF
:105A600087EEA60A20EE070A11F094FB95F8383D60
:105A700063B904F53A5033720A4ABDE87040062112
:105A8000383054F0CFBC002BC6DAB2E770BD00BF8F
:105A9000805C0020E4820020BD86002000007A4562
:105AA00035FA8E3CD0240D086D2900F3E3800129DE
:105AB00001DC5DF033BF8B1E6B2BFAD80FF2040CA8
:105AC0005CF823F0D35C0108CD5C0108D35C0108CD
:105AD000D35C0108B35A0108D35C0108B35A01082A
:105AE000B35A0108CD5C0108B35A0108D35C010820
:105AF000CD5C0108CD5C0108B35A0108D35C0108F4
:105B0000D35C0108D35C0108B35A0108B35A0108F9
:105B1000CD5C0108D35C0108CD5C0108B35A0108D3
:105B2000CD5C0108CD5C0108B35A0108B35A0108E5
:105B3000B35A0108B35A0108B35A0108CD5C0108F1
:105B4000D35C0108B35A0108B35A0108B35A0108DB
:105B5000D35C0108B35A0108CD5C0108B35A0108AF
:105B6000B35A0108D35C0108CD5C0108B35A01089F
:105B7000B35A0108B35A0108D35C0108D35C010889
:105B8000D35C0108B35A0108B35A0108D35C010879
:105B9000B35A0108B35A0108D35C0108D35C010869
:105BA000D35C0108B35A0108B35A0108D35C010859
:105BB000D35C0108B35A0108B35A0108B35A01086B
:105BC000B35A0108B35A0108B35A0108D35C01085B
:105BD000D35C0108D35C0108D35C0108D35C0108E5
:105BE000D35C0108B35A0108CD5C0108CD5C010803
:105BF000B35A0108B35A0108B35A0108B35A01084D
:105C0000B35A0108B35A0108D35C0108CD5C0108FE
:105C1000B35A0108B35A0108B35A0108B35A01082C
:105C2000B35A0108B35A0108B35A0108B35A01081C
:105C3000B35A0108B35A0108B35A0108B35A01080C
:105C4000B35A0108B35A0108D35C0108B35A0108DA
:105C5000B35A0108B35A0108B35A0108B35A0108EC
:105C6000B35A0108B35A0108B35A0108B35A0108DC
:105C7000CD5C0108A12921DC96297FF71AAFA1F19B
:105C800097030A2B3FF615AF0FF2040C5CF823F0D4
:105C9000D35C0108D35C0108B35A0108D35C010846
:105CA000B35A0108B35A0108B35A0108B35A01089C
:105CB000CD5C0108CD5C0108D35C0108B42908D093
:105CC000DB2903D0B2297FF4F4AE704700235DF0E6
:105CD000F7BD704770B563298AB0034668DC0129B7
:105CE00073DD881E612870D8DFE810F07C00840026
:105CF000940099006F00B3006F006F000C016F00FB
:105D00006F008B001F016F000A013C0143016F000F
:105D10006F004B01520159016F006A0173016F005E
:105D20006F006F006F006F007C0189016F006F00D2
:105D30006F008B016F006F006F006F008D016F00AF
:105D40006F006F006F006F006F006F006F006F00DB
:105D500095016F006F004501470149016F006F0019
:105D60006F006F006F006F006F006F006F006F00BB
:105D70008F0191019301970199019B016F00BC0173
:105D80009D016F006F006F006F006F006F006F006C
:105D900001026F006F006F006F006F006F006F00F7
:105DA0006F006F006F006F006F006F006F000D02DB
:105DB000B22900F068810EDC9A2900F0B0819F2999
:105DC00000F09D81982900F0A08118460AB0BDE836
:105DD00070405DF0E1BAB42900F0C680DB29F4D14F
:105DE000012433E0022AFBD135220E21B04803F012
:105DF00027FEF5E7111E18BF0121AD48FCF7FEF99B
:105E0000EEE7012A04D0022A14BF00210221F4E7A0
:105E10001146F2E706211846FFF752FDE0E7022A95
:105E2000DED1A44DD5F8EC000368DB6A9847044640
:105E30000028D5D0A5F58053D3F8DC3CB3F9083061
:105E4000002BCDD1A5F54050FFF774FD20460AB0D8
:105E500070BD022AC4D1974E974AD6F8EC109142F1
:105E6000BED0D6F8102192F8CB20002AB8D006F583
:105E70008054A6F58056B4F9F82F2AB9D6F8DC3C40
:105E8000B3F90830002BABD01C22002103A805ADCC
:105E9000B2F076FD284616F0ADFFB4F9F83F93B99D
:105EA0001623ADF80E30D4F8F43C8448642BB8BF08
:105EB000642303A906932CF0D3FD20B152F0B6F968
:105EC000272152F0EFF804F54F6494E80F0085E8BD
:105ED0000F00D6F8DC3C7948B3F90830002BCCBF72
:105EE0001023152303A9ADF80E302CF0B9FD0028BE
:105EF0003FF476AF52F09AF9272152F0D3F86FE7CA
:105F0000032188E7022A6E4D03D0002385F8F03C78
:105F100066E71921A5F596504BF06CFF0446002862
:105F2000F3D0012385F8F03C90E7012A0BD0022A38
:105F300011D0002A7FF454AF614B83F81C2352F038
:105F400075F92B21D9E75E4B019283F81C2352F09F
:105F50006DF92C21D1E75A4B83F81C2352F066F9D6
:105F60002D21CAE70F2156E7564811468BF070FDE8
:105F700036E709214FE704214DE705214BE71721BB
:105F800049E7901E414241414F4865F059FB27E7E0
:105F9000022A7FF425AF464801F062FB20E7012A80
:105FA00006D0022A07D0002A7FF41AAF1146EBE789
:105FB00011460192E8E74448012165F041FBEAE718
:105FC000424B911ED3F81C3D4A424A4183F820209F
:105FD00006E7931E594259413C4BD3F81C0D7FF004
:105FE0000BF8FDE6334B013A93F8E210012A8CBF1F
:105FF0000022012262F3041183F8E210F0E611217D
:1060000009E7122107E7152105E7002103E7102121
:1060100001E70221FFE60121FDE61621FBE607214B
:10602000F9E60B21F7E6022A284B0ED1012483F86A
:10603000E84E52F0FBF84A2152F034F85BF0C6F813
:10604000234A062154F0EEF900E7002283F8E82EF7
:1060500052F0ECF84B2152F025F85BF0B7F81D4AEE
:10606000062121E0012A09D0022A0AD0002A7FF461
:10607000B7AE012118480DF02FFFB1E601920021C3
:10608000F8E71146F6E75AB3022A7FF4A9AE094BA6
:10609000D3F8EC0003689B6F984700287FF4A0AE0C
:1060A0005BF094F80D4A042154F0BCF998E600BF67
:1060B000802C0020805C0020087C0020447C002094
:1060C000804C00201C7E0020107B0020806C002073
:1060D000E8240D08F9240D08005A00200B250D08AE
:1060E000184BD3F8EC000368DB6F984778E6184646
:1060F0001146FFF703FC144804F054F870E611460B
:10610000FFF70AFC6CE61B2185E6022A7FF468AEE5
:106110000E48FCF76BFE5BF059F80D4AA0E71146FC
:106120005DF024F80B487BF0B9FD044600283FF4ED
:1061300057AE044A92F8E33043F0020382F8E330AA
:1061400084E600BF805C00208C7B0020802C002037
:1061500024250D08785A002010B50446044884F020
:1061600063F904F10801BDE8104029F0A7BA00BFA7
:106170008079002038B504462DED028B114884F05B
:1061800059F905462BF004FA0F48B0EE408A0DF09D
:106190004FFF90B1DFED0D7AB4EEE78AF1EE10FA21
:1061A0000BDDD5ED000A95ED010AB0F0F3F9DFED56
:1061B000087A20EE270A84ED080ABDEC028B94EDE4
:1061C000080A38BD80790020802C002000401C4641
:1061D000E02E6542074B93F9D902022805D0032827
:1061E00006D0003818BF0120704781F001007047C9
:1061F00004207047804C002003688B4216D004298D
:10620000C0E9001302D007290ED07047084B9FED5C
:10621000097A03F59663D3ED007AF8EEE77A67EE34
:10622000877AC0ED087A704700238362704700BF09
:10623000803C00200AD7233C08B50246FFF7CAFF7E
:10624000BDE8084001461046FFF7D6BF70B52DEDFA
:10625000048B0446F0EE408AB0EE608A0D46164686
:106260008DF01EF89FED329ADFED329AE06176B341
:10627000236843B9304B03F59663D3ED007AF8EE0B
:10628000E77AC4ED097A68EE898A002DB7EE000A34
:10629000FFEE007AB8BFB0EE670A68EE808AC4ED00
:1062A000058A264BB4EEE98AF1EE10FAD3F81C0DFC
:1062B00030DA7DF07FFE20EE090A84ED060ABDEC9F
:1062C000048B20460321BDE87040FFF795BF94ED95
:1062D000090A98EE890A28F08FF9002D84ED050A45
:1062E0000BDAB4EEE90AF1EE10FADADBDFED147A3C
:1062F00030EE670A84ED050AD3E7D2D0DFED117ADC
:10630000B4EEE70AF1EE10FACBD8DFED0D7A30EEFD
:10631000270AEFE77DF04EFEB4EE480AF1EE10FAE0
:1063200048BFB0EE408A28EE098A84ED068AC6E7A7
:106330000000C84200000034803C0020806C002037
:1063400000A00C47000000B410B52DED028B0446F0
:10635000B0EE608AF0EE408A8CF0A2FFDFED090A11
:10636000E06168EEA08A68EE200AC4ED098ABDECFF
:10637000028BC4ED0A0A20460621BDE81040FFF753
:106380003BBF00BF0000C84210B52DED028B044694
:10639000B0EE408A8CF084FF94ED090ADFED097AB3
:1063A000E061A8EE270A28F011F9BDEC028B00236A
:1063B00084ED090AA36220460621BDE81040FFF7DC
:1063C0001BBF00BF0000C84270B54B68154D0646A4
:1063D0000C4673B98B6863B9C96851B91248FFF7A5
:1063E0002BFF95F8351E05F6BC50BDE870405FF0F8
:1063F000A9BB95F8351E0D485FF044FA48B906F17F
:106400000801204616F086FE18B107480221FFF762
:10641000F3FE95F8351E05482246BDE870405FF052
:1064200085BB00BF806C0020EC8400203C7A0020FB
:1064300008B50721FFF7E0FE80ED0A0A08BD00005D
:1064400008B50368032B23D1D0ED057A9FED127AAE
:10645000F0EEE77AF4EEC77AF1EE10FA1AD50F4BA8
:1064600090ED090A03F59663D3ED007AF8EEE77A2A
:1064700037EEC00A28F0C0F8DFED097AB0EEC00AA6
:10648000B4EEE70AF1EE10FA94BF0120002008BD37
:106490000120FCE70020FAE700000034803C0020E7
:1064A0000000484330B50368023B85B00446082B22
:1064B0006DD8DFE803F0050D30374B613F616100B7
:1064C000FFF74AFE84ED090A94ED090A05B030BDD4
:1064D0008CF0E6FEE369DFED310AE061C31A07EEF6
:1064E000903AF8EE677A94ED050A67EEA07AD4ED5B
:1064F000060AF12020EEA71A67EEE00A28F0D2F88B
:10650000D4ED057A77EEC07AC4ED057AD4ED097A38
:1065100037EE800AD6E7FFF72DFEDFED217A20EE79
:10652000270ACFE71F4BD3ED4E7AF8EEE77AC0ED9E
:10653000097AC9E71C4DD5F8300D82F00FF9002813
:10654000C2D0D5F8303D1B6B6362BDE78CF0A8FE6E
:10655000E3699FED127AD4ED0A6AE061C31A07EE8F
:10656000903AF8EE677A67EE877A94ED097AA6EEAC
:10657000A77A84ED097AA7E70B4B9FED0C0AD3F8B5
:106580001C0D6C302BF0C2FA84ED091A9CE7064B07
:10659000D3F8243DD3F84433D6E700BF6F12833AD3
:1065A0000000C842805C0020806C00209F0CB34536
:1065B0000368092B08D8DFE803F0050A050505057F
:1065C000070705100023836290ED0A0A7047044B09
:1065D000D3F8243DD3F84833F5E7C36AF3E700BFA7
:1065E000806C0020F8B50023214FCB6297F805316D
:1065F000204E13F0010F04460D462DD1D7F8EC00C4
:1066000003685B6F984738B3D7F8EC0003F0CEFB14
:10661000DFED197A85ED0B0AB0EEC00AB4EEE70A99
:10662000F1EE10FA03D409213046FFF7E5FD1148D9
:10663000FFF738FF0F4884ED000AFFF7B9FF336812
:1066400084ED010A0A2B0FD8DFE803F00C101010BC
:106650001010100C100C0C003368092BE7D1054802
:106660000021E2E70223A3602046F8BD0123FAE7F8
:10667000805C0020EC84002000000034034B0122E9
:106680001A6000229A60DA601A617047EC84002078
:1066900013B501A904460DF067FB04F5804320B94A
:1066A000012283F8652E02B010BDDDED017ADFED29
:1066B000096A03F65862B8EEE77AD2ED007A67EE1F
:1066C000A67AB4EEE77AF1EE10FA54BF0122002266
:1066D000E7E700BF0000C8422DE9F04F2DED068B23
:1066E00000F5005B00F595599BF92A338DB00546FE
:1066F00000F5804409F1100933B100F54058D8F88D
:10670000103193F8CB707FB90021A4F8DC1E484605
:1067100010F030FF94F8DD1E48460DB0BDEC068B3E
:10672000BDE8F04F10F030BF8CF0BAFD0190D4F806
:10673000240D9FED948A90EDDBAA80F02FFA09AE2C
:10674000002800F0CA80D4F8243D03F55C7393E878
:10675000070086E8070030468DED0B8A2BF0D4FD4C
:10676000B0EE409A28460DF063FC05F59A4A0028E1
:1067700000F0B680504683F05DFE07C886E807004B
:1067800030468DED0B8A2BF0BFFDF0EE409AD8F825
:10679000EC0003681B689847122840F0AA80002389
:1067A00084F8DC3ED8F8EC0003685B69984728B1B0
:1067B000DBF8DC3CB3F90830002B0DDC98F9E03055
:1067C000002B09DA019BC4F8E03E504683F02EFE10
:1067D00004F6E46383ED000A94F8DC3E5BB1019BB0
:1067E000D4F8E00E181A41F28833984240F28F80B4
:1067F000002384F8DC3ED4F81C0D9FED630A6C3056
:106800002BF084F98DED090ACDED0A0A8DED0B1AF6
:1068100096E8070006AB03AE9FED5C0A83E807002D
:1068200086E8070030462BF071F92846B0EE408A22
:10683000F0EE608A8DED060ACDED070A8DED081A9F
:106840000DF0F6FB002874D0DFED517AF4EEE79AF4
:10685000F1EE10FA94BF01250025D4F8240D80F044
:106860009DF930B1DFED4A7AB4EEE79AF1EE10FA15
:1068700009D9002D64D1D8F8EC0003681B6898474B
:10688000022864D00027D4F8240D80F0A9FA054628
:10689000002873D0B5EEC0AAF1EE10FA6DD5DFED89
:1068A0003D7AB4EEE7AAF1EE10FAACBF012600265D
:1068B000504683F0C7FD5EB9DFED377AB0EEC00A0F
:1068C000B4EEE70AF1EE10FA5AD8002D08BF0027FF
:1068D00094F8DC1E84F8DD7E19E7B0EE489A41E7B3
:1068E00028460DF075FB00287FF444AFDFED259AB4
:1068F0004DE7D8F8103193F8CB30002B3FF452AF6E
:1069000098F9E030002BBFF64DAF012348E7504621
:1069100083F08CFD04F6E463D3ED007A30EE670A71
:10692000DFED1E7AB4EEE70AF1EE10FA3FF760AF42
:1069300061E728460DF04CFB0546002884D18CE722
:10694000D4F8240D80F02AF9002894D19BE7B0EE0A
:10695000680AAFF0CDFBF0EE408AB0EE480AAFF027
:10696000C7FBDFED0F7A20EE280AB4EEE70AF1EE5E
:1069700010FACCBF0127002785E700252E4697E7B0
:106980003746A5E7000000009F0CB345D302373916
:106990000000FA420000C8C20000704200004842F5
:1069A00055CF7D3F38B504460DF042FB04F59555B3
:1069B000103548B920460DF00BFB014620B928469A
:1069C000BDE8384010F022B804F54054D4F8EC008B
:1069D00003689B6C984720B9D4F8EC000368DB6C23
:1069E00098470146EBE7000030B5044689B0684699
:1069F00004F5955516F0FEF9103504A816F0FAF9CD
:106A00006946284610F0BCF898B104A9284610F051
:106A100007F970B1059B019323680022DB6C69467E
:106A20002046984728B104F52B5001211C3087F0EF
:106A300061FC09B030BD000000F5805292F82C25B1
:106A4000D2070BD400F54052D2F8102192F8CB10A7
:106A500009B1FFF7C9BF03689B6C18477047000076
:106A600030B587B0044602A8019116F0C3F904F5C9
:106A7000955002A9103010F083F8019A18B900253A
:106A8000284607B030BD236802A9DB6C2046984732
:106A900005460028F3D004F52B5001211C3087F067
:106AA00029FCEDE7F0B5044685B004F59556684637
:106AB00010360F46154616F09DF96946304610F01F
:106AC000AFF810B9002005B0F0BD394630460FF0E0
:106AD0000FFF0028F6D0002DF5D004F5805428468D
:106AE00094F82C3543F0020384F82C35EBE70000D2
:106AF0002DE9F04F2DED0A8BBDB0044624220D4642
:106B000018A80021B1F03CFF2422002121A8B1F0F7
:106B100037FF242200212AA8B1F032FF04F54056A5
:106B20002422002133A8B1F02BFF0023CDE90D333F
:106B30000F9396F8E13013F0080839D104F50059A5
:106B400043F0080399F8D02C079286F8E13017F04B
:106B5000A9FA90F9213003B390F84033EBB104F275
:106B60008457384617F0AEF9C34694F8A6355FFA55
:106B70008BF18B421FD9384617F082F90BF1010BCC
:106B800082460028F1D1C94A0221284656F03EFF2C
:106B900096F8E1306AF3C30308E0C54A02212846AB
:106BA00056F034FF96F8E1306FF3C30386F8E13016
:106BB0004FF001083EE304F53753383301211846FE
:106BC0000BEE903AFAF7F6FF824608B9B94ADBE7CE
:106BD00020460CF04FFFD9F8DC3CB3F908A0BAF11D
:106BE000000F01D0B44AD9E796F9E030002B01DB61
:106BF000B24AC9E7204601F0AFFE04F544533C33E6
:106C0000184652460CA90CEE103A13F01DFA002853
:106C100014BF022301230393F123CDE9133A8F21FB
:106C20000A23CDE9003113AA287CADF854A0032330
:106C30004D2154F02BFCA24B9FEDA28A01225A72E7
:106C40000621A14A284656F0E1FE039B022B0CBF09
:106C50009E4A9F4A062128464FF0000A56F0D6FE6B
:106C600089F8E6A25146384617F076F894F8A6352A
:106C70005FFA8AF18B420CD913AA38468DED138A3C
:106C80008DED148A8DED158A0AF1010A16F0E6FEE3
:106C9000ECE7384617F016F94FF0000A4FF07C0B7E
:106CA00094F8A6255FFA8AF94A4519D94946384623
:106CB00016F0C6FDC0B20BFB00403CAA0C2300F24C
:106CC000146003FB092C07C8ACF1900C8CE807009A
:106CD0003CAA02EB890909ED2F8A0AF1010ADFE7D4
:106CE00041F288310AA823F0C1FFD6F810019FEDC8
:106CF000759A03689FED77AA9B6ADFED77AA98479C
:106D0000D6F81001012184F03DFB744B1B680293FF
:106D1000D86A036801211B6898478CF0C1FA059076
:106D20008CF0BEFAF0EE499A0690002604F5005960
:106D3000079A99F8D03C934240F0D88094F8C6184E
:106D4000384617F09DF8002800F0D08004F5405B2D
:106D5000DBF8103193F8CB300493002B00F0C680A1
:106D600041F288310BA823F081FF8CF099FA059B42
:106D7000C01A132840F2D9808CF092FA0590204670
:106D80000CF078FE5DF08AFD82465DF01DFDD9F8BD
:106D9000DC3CDBF81001B3F9083000EE103AB8EE35
:106DA000C00A20EE0A0A85F05FFF50465DF014FD30
:106DB000384617F087F81CEE100A13F061FBD9F87B
:106DC000DC3CDFED400AB3F9083000EE103AB8EED3
:106DD000C00AA22020EE0A0AB7EE001A27F062FCD1
:106DE000B4EEE90AF1EE10FA1CEE100A4FF00002C0
:106DF0000CA958BFF0EE409AF0EE408A13F024F947
:106E000008B900230C939DED0C8ADFED357AB4EEC2
:106E1000498AF1EE10FAF4EEE78A48BFB0EE498AEB
:106E2000F1EE10FA80F28F809FED2E9ADFED2E8A20
:106E30004FF0000A94F8A6355FFA8AFB5B4540F2F2
:106E400096814FF00C0918AB09FB0BF903EB090015
:106E5000B0EE490A2AF05AFE59463846CDED110ADD
:106E60008DED121A8DED100A16F0EAFC7C23C0B2EB
:106E700003FB0040B0EE680A00F214602AF046FE00
:106E80003CAB13A910A899448DED130ACDED140A5B
:106E90008DED151A2AF00EFE0AF1010A09ED240AF9
:106EA00049ED230A09ED221AC4E700BF21270D0886
:106EB00010270D08933D0D082F270D0841270D08B9
:106EC000BD860020000000004C270D0861270D083A
:106ED00023D00C086F12833A0000C842E0840020DF
:106EE00000000034A4707D3F0AD7233C04F54059CC
:106EF000D9F8100103689B6A9847D9F8100100215E
:106F000084F040FA029BD86A036800211B68984706
:106F1000002E40F05F812846C94A052156F076FDD3
:106F20003146384616F018FF70E1029B986A0368F4
:106F300005215B6898470BA823F0A4FEB0EE498AB0
:106F4000B0EE489AF2E64FF000094FF00C0B04F552
:106F5000B86A94F8A6255FFA89F39A4222D91946AD
:106F60003846089316F06CFC089B0BFB03F13CAB16
:106F70005A18A2F16C034FF07C0CC0B2CDE9083274
:106F80000CFB00A018AB194454302AF0A9FD089B53
:106F9000099A09F1010902ED1B0AC3ED010A83ED0B
:106FA000021AD6E7039B012B4FF0000A46D19FED52
:106FB000A5BA9FEDA59A4FF00C0B94F8A6355FFA91
:106FC0008AF6B34240F286800BFB06F63CAB03EB3D
:106FD0000609A9F14803089321ABB0EE680A981995
:106FE0002AF0A4FD089B09ED120AC3ED010A83ED06
:106FF000021A33ABB0EE4B0A98192AF087FD2AAB80
:1070000098198DED100AB0EE490ACDED110A8DEDFB
:10701000121A2AF07BFD13A910A88DED130ACDEDED
:10702000140A8DED151A2AF05BFD0AF1010A09ED2B
:10703000090A49ED080A09ED071ABEE79FED819A92
:107040009FED81BAF0EE088A94F8A6355FFA8AF9C6
:107050004B4564D99DED0C0AB4EEE80AF1EE10FA46
:1070600035DB0C2303FB09F93CAB03EB090621AB31
:1070700003EB09002AF05AFD33AB46ED110A06ED89
:10708000101A06ED120A03EB0900B0EE490A2AF0C5
:107090003DFD2AAB03EB09008DED100AB0EE4B0A63
:1070A000CDED110A8DED121A2AF030FD13A910A8AA
:1070B0008DED130ACDED140A8DED151A2AF010FD91
:1070C00006ED090A46ED080A06ED071A049E0AF1C4
:1070D000010AB9E74FF000094FF00C0A94F8A63501
:1070E0005FFA89F6B34241D933AB0AFB06302BF085
:1070F0000BF91BEE900AF0EE408A7AF0CBFD07EE1A
:10710000900AB8EE677A3CABC8EE877A03EB860646
:1071100009F1010967EEAA7A46ED2F7ADEE74FF012
:10712000000A4FF00C0B94F8A6355FFA8AF94B452C
:107130001DD933AB0BFB09302BF0E6F8C8EE297AEA
:107140000AF1010A1BEE900A67EE808A7AF0A2FD2E
:1071500007EE900AB8EE677A3CABC8EE877A03EB8D
:10716000890967EEAA7A49ED2F7ADCE7049E8CF054
:1071700097F8069BC01AB0F5FA7F27D98CF090F8E3
:1071800004F50053DDED0D7AD3F8DC3C0C9A1B8935
:107190001392FCEEE77A339A1492ADF85C30349A8D
:1071A000159217EE903A359A1692ADF85E30F022AD
:1071B0001423CDE90032B121069013AA287C54F0A3
:1071C00065F974F071FD297C74F060FC0BA823F064
:1071D00059FDB5E60399384616F0BEFD00264FF07E
:1071E0000C0A94F8A635F1B28B4207D933AB0AFBEF
:1071F0000132384616F032FC0136F2E7384616F016
:107200003FFC124A0621284656F000FC104B002590
:1072100020465D7201F092FB04F50B50263049F0D8
:10722000A3FC99F8E13065F3C30389F8E1300AA8BB
:1072300023F028FD40463DB0BDEC0A8BBDE8F08F41
:107240009DD80E08A4707D3F0AD7233C69270D08FE
:10725000BD860020F0B5534FD7F8983CDA0785B0CB
:10726000044600F19C8000F54055D5F8103193F8A4
:10727000C120002A40F0938093F8CB30002B00F01F
:107280008B8095F9E030002BC0F2868000F58046B7
:1072900096F8E83E002B40F08280D6F81C0D9FED5A
:1072A000420A6C302AF032FCCDED020A60EEA00AF0
:1072B000DFED3E7A8DED010AE0EE000A8DED031A56
:1072C000F4EEE70AF1EE10FA66DCD6F81C3D9FED0D
:1072D000387AD3ED377AF4EEC77AF1EE10FA04D5A6
:1072E000D5F810311B7A002B56D0B5EE007AF4EEAB
:1072F000C77AF1EE10FA4FD404F59A4083F0A2F861
:10730000DFED2C7AB4EEE70AF1EE10FA44D8D6F8A5
:107310001C3D9FED297AD3ED367A67EE877AB3EE7E
:107320000E7AF4EEC77AF1EE10FA35DA234AB4F9A0
:10733000A410138801339BB2138019B9B4F8A210BA
:10734000A4F8A410B4F8A410994228D800261680F6
:1073500050F06CFF0122192150F0C4FED5F8100145
:1073600003685B699847431C04F53A50144A314658
:10737000383053F057F8D5F81031012283F8C12086
:10738000D7F8983C5B070AD504F58550083005B05E
:10739000BDE8F04068F050BA084B00221A8005B0F2
:1073A000F0BD00BF804C00209F0CB3454054094AFB
:1073B0006666663F000000B4E02E65422685002028
:1073C00080270D0870B52DED028B4A4BD3F8983C01
:1073D0009B0784B004461FD400F58045DFED468A44
:1073E000D5F81C0D03681B699847D0ED017AF4EEBF
:1073F000E87AF1EE10FA0FDB04F5405304F59D46F0
:10740000D3F8102192F8C1106C3649B1002303A9BA
:107410003046039352F03EFB04B0BDEC028B70BDCE
:1074200092F8CB20002AF1D093F9E030002BEDDB6D
:1074300095F8E83E002BE9D1D5F81C0D03681B69CF
:107440009847D0F8A430D5F81C0D039303681B6946
:10745000984704F58C7200F1A401304652F018FCF4
:10746000DDED037AB0EEC08AF0EEE77AF4EEC87A8A
:10747000F1EE10FA03D503A9304652F00BFBD5F814
:107480001C0D03681B699847D0ED040AF4EEE80A66
:10749000F1EE10FAC0DBF6EE087A60EEA77AF4EEB1
:1074A000C87AF1EE10FA1DD58BF0FAFED5F8F83E49
:1074B00042F21072C31A9342AED9DFED107AC5F8CA
:1074C000F80E68EE277A04F53A5417EE900AF9F7A9
:1074D0001BF83834CDE90001094A0021204652F05A
:1074E000A1FF99E79DED030A26F0D8FF0028DBD124
:1074F00092E700BF804C0020000000340000C8422A
:107500009C270D0810B5044600F59D40103064F02E
:10751000A9F804F59D400121BDE8104030306CF021
:107520006DBB0000F8B500F58045044695F9903E26
:1075300043B300F5405695F8A42E96F8E030DB43AF
:10754000C3F3C01363F3C30285F8A42E00F59D476F
:1075500000F59A4082F076FFDFED3D7A103720EE9D
:10756000670A384664F0FEF895F8E83E53B93846A5
:1075700064F0A4F8D6F8103193F8CB301BB9354B32
:1075800000221A80F8BD95F8A43EDB07FAD4D6F89D
:10759000EC0003689B6B98470028F0D096F9E03028
:1075A000002BECDB2B4E33884BB9B5F9963E33B14B
:1075B000642213FB02F3D5F8F42C9A42E2DB38463E
:1075C00064F0ECF8D5F81C3D9FED237AD3ED367AC4
:1075D00067EE877AB3EE0E7AF4EEC77AF1EE10FA20
:1075E00005D83388002BCDD0013B3380CAE7B4F9EE
:1075F000A4301BB9B4F8A230A4F8A4303388B4F88E
:10760000A420B4F9A400154993423CBF0133338050
:107610003388D5F8CC2C012B01D10A60B2E7096878
:107620009142ACDD18B9B4F8A220A4F8A420B4F8B3
:10763000A4209A42A6D80023338050F0F7FD0222FE
:107640000C2150F04FFD2046BDE8F840FFF75ABF2F
:107650000AD7233C24850020E02E654220850020A7
:1076600008B500F5804292F9903E6BB300F54053A7
:1076700093F9E030002B0EDA00F53A50134A062158
:10768000383052F0CFFE50F0D1FD0322BDE8084063
:107690000F2150F027BDB2F9963E8BB1D2F8F42CF1
:1076A000642113FB01F39A420ADA00F53A50084AC2
:1076B0000121383052F0B6FE50F0B8FD0222E5E765
:1076C000BDE80840FFF71EBF08BD00BFB4270D0886
:1076D000C6270D08F0B52DED028B00F540555C4E28
:1076E000D5F8103193F8CB308DB0044643B195F9FD
:1076F000E030002B04DB00F5005393F902332BB983
:10770000002333800DB0BDEC028BF0BD00F5804747
:1077100097F8E83E002BF3D101F084FB00287DD1DF
:10772000D5F8EC0003689B6B98470028E8D004F577
:107730009940503052F004FA2AF0E6FDF0EE087A53
:10774000B4EEE70AF1EE10FAF0EE408AD8DA04F56A
:10775000805303F59F6203F2FC43D3ED007A92ED70
:10776000000A20EE270AAEF0ADFEDFED3A7A20EEF9
:10777000270AB2EE0E7AB4EEC70AF1EE10FABFD9BC
:10778000D7F81C3D93ED368A28EE278AF3EE0E7A61
:10779000B4EEE78AF1EE10FAB2D904F59550002361
:1077A00009A9103009930A930B930FF045FA0028AA
:1077B0003DD13388B4F9A42001339BB23380002A31
:1077C00040D0B4F8A420B3EB420F9BDB50F02EFD69
:1077D00001220C2150F086FC1F4B002218EE900A6B
:1077E000CDE90623F8F790FE1C4BCDE904010022F9
:1077F00018EE100ACDE90223F8F786FE04F53A5494
:107800003834CDE90001164A2046002152F00AFE24
:1078100001220C211348FAF7E5FB73E7D5F8EC00D9
:107820000368DB6C984700287FF47AAF68E709A803
:107830002AF06AFDF2EE047AB4EEE70AF1EE10FAED
:10784000B7DB5DE7B4F8A220A4F8A420B9E700BF35
:107850001C850020E02E65420000084000003E40EC
:10786000DC270D08785A0020F0B52DED028B8BB087
:10787000002307930893099305AB0446019300F591
:10788000955007AB009302AA04AB03A910300FF088
:10789000EBF804F50056054686F8AC0E28B900252D
:1078A00028460BB0BDEC028BF0BD8BF0F1FCD6F896
:1078B000B03E9FED327AC31A07EE903AF8EE677A3F
:1078C000074667EE877A04F53A5006AA02A90830FF
:1078D000CDED067A52F0DCF904F53A5006AA03A978
:1078E00014308DED020A52F0D3F904F53A5006AA8D
:1078F00004A920308DED030A52F0CAF996EDC18A31
:10790000C6F8B07EB5EEC08AF1EE10FAC7D9DDED4B
:10791000080A9DED070AAEF071FCDDED090AAEF034
:107920006DFCD6F8302EDDED037AB4EEC08AF1EEB0
:1079300010FA94BF012300231AB196F8342ED2070F
:1079400012D438EE087AB4EEE77AF1EE10FA0BD8DA
:107950000233DBB2DDED027AB4EEE78AF1EE10FA23
:1079600009D8002B9BD09BE7B4EEE78AF1EE10FA22
:10797000F0D80133EDE7012B92D890E7BD3786357B
:1079800070B500F54055044695F8053143F0040301
:1079900085F8053150F04AFC0122112150F0A2FB7C
:1079A000D5F8103193F8CB30002B43D0D5F8EC004C
:1079B00003681B68984709280AD1204608F01CFE76
:1079C00030B104F5A9404030BDE8704008F0FCBD7E
:1079D000194BD3F8EC0003681B69984704F5005372
:1079E00040B993F90133032B24D10621204608F036
:1079F000EFFD0DE093F901130229F6D195F8053159
:107A0000DB07F2D40622204602F01AF80028ECD058
:107A10000A4BD5F8EC0001225A7303681B6C984797
:107A2000034604F53A50064ABDE87040022138305A
:107A300052F0F8BC70BD00BF805C0020BD86002005
:107A400010280D0808B500F5405292F80531590785
:107A500017D56FF3820382F805310A4B5A7B42B186
:107A6000002200F53A505A730221074A383052F08A
:107A7000D9FC50F0DBFBBDE808400022112150F09A
:107A800031BB08BDBD86002034280D08F0B5054681
:107A900085B005F595576846103715F0ABF969467E
:107AA00038460FF0BDF880B105F50053D3EDC17A2B
:107AB000374CF5EEC07AF1EE10FA08D8354A0023BB
:107AC00028462380D373FFF7BDFF05B0F0BD2846DD
:107AD000FFF7CAFE064628460CF07AFA10B9284687
:107AE0000CF052FAA378002E18BF00200343DBB23B
:107AF000A370002BE9D06378A8BB83BB2378013344
:107B0000DBB2082B237003D14EB338460FF018F8C0
:107B10002378092B02D138460FF00AF82378092B75
:107B20001DD94FF48573238050F080FB0222102171
:107B300050F0D8FA8BF0B4FB6368C01A47F23053A8
:107B4000984209D905F53A50134A0221383052F0CB
:107B500069FC8BF0A5FB60602846FFF711FF0D4B19
:107B60006278DA73B1E72678002EF8D0013EF6B2DB
:107B70002670002BF3D0002EF1D1667050F056FB2A
:107B80003246102150F0AEFA2846FFF75BFFE6E7D9
:107B900028850020BD8600204C280D0800F54053A4
:107BA00093F805315B0701D5FFF7EABE7047000087
:107BB00073B5044600F5955001A9103004F5005541
:107BC0000EF09CFDD5F8743E834206460CD004F5B9
:107BD0008043D3F81C0D7DF0B1FDC5F8746E50F0F4
:107BE00025FB3E2150F05EFA04F5805695F9781E8B
:107BF00096F9C02596F8C03591421BD0FF2B19D0BD
:107C000004F58043D3F81C0D7DF098FD96F8C0353F
:107C100085F8783E50F00AFB95F8782E182150F040
:107C200061FA04F53A5095F9783E034A0421383058
:107C300052F0F8FB02B070BD5C280D082DE9F0434E
:107C40008FB005468BF02CFB00230593069307931A
:107C5000089309930A930B930C930D9305F595588C
:107C600004AB019308F1100803AB009306460BAB7D
:107C700008AA05A940460EF0D7FEDFED487A9DED33
:107C8000077AB4EEE77AF1EE10FA074632DB9DEDA3
:107C90000A7AB4EEE77AF1EE10FAACBF01240024C0
:107CA00005F50059404699F8AC3E002B08BF002767
:107CB0000EF0CCFE8046FFB9444699F9343C012BC6
:107CC0002BD174B105F54053D3F8102192F8CB4075
:107CD0003CB1D3F8EC0003685B69984780F0010081
:107CE000C4B299F87C3ECBBBCCB9C9F8806E0FB05A
:107CF000BDE8F0830024D3E7002CDDD005F53A5031
:107D0000143051F0C5FE90ED007AF7EE007AB4EE33
:107D1000E77AF1EE10FAD0DCCEE70024E1E7D9F8FB
:107D2000800E301AB0F57A7FE1D9C9F8843E01247B
:107D300005F5804389F87C4ED3F8243D83F80C4444
:107D400050F074FA22461D2150F0CCF9144A05F582
:107D50003A500221383052F065FBC8E714B1C9F837
:107D6000846EC4E7D9F8840E43F69823361A9E42EF
:107D7000BDD905F58043C9F8804E89F87C4ED3F80B
:107D8000243D83F80C44C9F8844E50F04FFA224643
:107D90001D2150F0A7F9034AD9E700BF00000034C5
:107DA00074280D088E280D080B4B10B501220446CF
:107DB0005A728BF075FA04F58042D2F8D43EC31A99
:107DC000142B07D9C2F8D40E04F59350BDE8104027
:107DD00044F074BF10BD00BFBD8600202DE9F743FD
:107DE000044604F5405600F50B5000233C300DF1DD
:107DF00007018DF8073049F02DFCD6F8100190F9F5
:107E0000C030026883B3083BDBB2012B95692BD9E4
:107E10003221A84704F1100012F0ACFC204B04F50D
:107E20003A581F684FF0000908F13808F86A0368EB
:107E3000DB69984701281ED18BF032FA41F2873373
:107E4000A0EB09029A42054605D9164A062140468A
:107E500052F0E8FAA9462046FFF7A6FFB86A036881
:107E600003215B689847E1E704F500539269B3F892
:107E700010139047CEE70121D6F8100183F082FA63
:107E8000D6F810010368DB6A98475CF005F9F86AD8
:107E900003681B68012103B0BDE8F043184700BF29
:107EA000E0840020AC280D0870B5044600F53A5077
:107EB0002DED028B184A194E9FED198A0621383094
:107EC00052F0B0FA2046FFF789FF2046FFF76CFF1B
:107ED00020460BF0CFFD3368986A036803215B6886
:107EE00098475CF0DBFC05465CF06EFC04F5005343
:107EF000D3F8DC3CB3F9083000EE103A04F54053F7
:107F0000B8EEC00AD3F8100120EE080A84F0ACFEE7
:107F100028465CF061FCD8E7D0280D08E0840020FA
:107F20006F12833A2DE9F047044600F53A502DEDE3
:107F3000028B2A4ADFF8AC900621383052F072FAF0
:107F40002046FFF74BFF5CF0A9FC04F540560546C0
:107F50005CF03AFCB7EE000AD6F8100184F084FE1B
:107F600028465CF039FC8BF09BF941F2873A0746D2
:107F70008BF096F9C01B5045D9F8008017D99FEDBA
:107F8000188A28465CF020FCB0EE480AD6F81001AA
:107F900084F06AFE28465CF01FFC2046FFF704FFD1
:107FA000D8F82800036803215B689847E9E728466A
:107FB0005CF00AFCB7EE000AD6F8100184F054FE1B
:107FC00028465CF009FC2046FFF7EEFED8F82800B2
:107FD000036803215B689847CAE700BF00290D08C2
:107FE00000000000E0840020F7B500F5405304468F
:107FF000D3F8103193F9C030032B2BD0364E6525C2
:1080000000F58047013D15F0FF050CD0D7F8D03EB4
:108010004BB93368986A036814215B689847204617
:108020000BF028FDEEE704F5375001213830F9F761
:10803000C1FD04F5005378B993F9FC3253B1092B13
:1080400008D08DF8070004F50B500DF107013C3006
:1080500049F000FB03B0F0BD93F9FC22032A34D8A9
:10806000DFE802F002252D30D3F8DC3CB3F908201C
:1080700040F2B5339A422ADD04F50B5001250DF18B
:1080800007013C308DF8075049F0E4FA04F53A5006
:10809000124A0221383052F0C5F9114B5D720E4B75
:1080A0001C68A06A036805215B689847F9E7D3F864
:1080B000DC3CB3F9082040F2B5339A4207DD204694
:1080C000FFF7F2FE2046FFF72DFF092AC2D000235A
:1080D0008DF80730B7E700BFE084002024290D08A1
:1080E000BD86002000F53A500B46024A0421383084
:1080F00052F098B944290D0810B5044650F096F88E
:10810000002205214FF0EEFF04F53A50034ABDE886
:1081100010400421383052F085B900BF50290D08B5
:1081200013B50B464AB100F53A5000920421054AB6
:10813000383052F077F902B010BD02B0BDE81040FF
:10814000FFF7D0BF68290D0808B500F53A50064A78
:108150000421383052F066F950F068F8BDE8084064
:10816000002208214FF0BEBF7C290D0838B5044617
:108170000D468BF095F804F540533DB9D3F8FC203B
:10818000C3F800010AB9C3F8FC0038BDD3F80021D8
:10819000801A642884BF0022C3E93F22F5E700006B
:1081A00037B5044600F59A4082F032F904F54052A2
:1081B000C0F3803592F8E230C3F34001A9421DD0EC
:1081C00065F3410304F53A5482F8E23038346DB176
:1081D00050F02CF802220B214FF084FF084A0221B4
:1081E000204603B0BDE8304052F01CB950F01EF8F4
:1081F0002A460B214FF076FF024AF0E703B030BD6C
:1082000094290D08B0290D0838B50A460C460621F8
:10821000054601F015FC28B1054A137843F0080320
:10822000137038BD21462846BDE8384008F0D0B963
:10823000DC86002038B50A460D461521044601F0BB
:10824000FFFB28B1094A137843F00803137038BDC7
:1082500004F53A5004213830054A52F0E3F8294633
:108260002046BDE8384008F0B3B900BFDC860020E6
:10827000C0290D0838B50A460D461521044601F0FF
:10828000DFFB28B1094A137843F00803137038BDA7
:1082900004F53A5004213830054A52F0C3F8294613
:1082A0002046BDE83840FFF7AFBF00BFDC860020A6
:1082B000E8290D0838B50A460D461B21044601F091
:1082C000BFFB28B1094A137843F00803137038BD87
:1082D00004F53A5004213830054A52F0A3F82946F3
:1082E0002046BDE83840FFF78FBF00BFDC86002086
:1082F000FE290D0838B50A460D461121044601F045
:108300009FFB28B1094A137843F00803137038BD66
:1083100004F53A5004213830054A52F083F82946D2
:108320002046BDE8384008F053B900BFDC86002085
:10833000102A0D0810B500F5405494F8E2309A0662
:1083400023D4D4F8EC0003681B689847032808D0AE
:1083500005D802280ED194F8E000C00914E01B28CB
:10836000F9D194F8E00000F0A000A0F18003584299
:10837000584109E0B4F8E00020F4FE4020F07F000E
:1083800080B2003818BF012010BD0120FCE70000BA
:1083900038B500F54055044695F80531184A43F0C4
:1083A000080300F53A5085F805310221383052F0C3
:1083B00039F84FF03BFF012217214FF093FE204682
:1083C000FFF7B8FF40B104F537500122BDE838404F
:1083D00015213830F9F706BED5F8EC0003681B68A4
:1083E0009847062806D104F5AB405830BDE8384020
:1083F00009F0FABA20460B21BDE83840FFF704BF68
:10840000242A0D0870B500F54055D5E93F239B1A85
:1084100041F288329342064611D9D5F8EC00036840
:108420001B6D9847044695F80531C3F3C003A3427A
:1084300013D034B13046BDE87040FFF7A9BF002427
:10844000F1E74FF0F3FE224617214FF04BFE95F86F
:10845000053164F3C30385F8053170BD0B4610B5D3
:1084600011460446072B07D8DFE803F02A04131649
:10847000191C242708F0ACF804F50053D3F8383C55
:108480009B061DD504F585500830BDE8104067F007
:10849000D3B9FFF7B9FEEFE7FFF7ECFEECE7FFF724
:1084A000C9FEE9E700F53750012214213830F9F709
:1084B00099FDE1E7FFF7FEFEDEE7FFF71BFFDBE7D5
:1084C00010BD0000F8B5044604F500574FF0AEFEAD
:1084D000012205214FF006FE97F8E632072B98BFE0
:1084E000304A204694BFD55C0125FFF723FF68B1D1
:1084F0002D4A2E492046FFF713FE04F5375001227E
:1085000010213830F9F76EFD002514E004F54056CF
:10851000D6F8EC000368DB6C984798B196F8AD3656
:1085200083B196F9AC36012B0CDC214A2149204657
:10853000FFF7F6FD0125294620460322BDE8F84055
:10854000FFF78CBFD6F8EC000368DB6C984718B1D6
:10855000D7F8383C190715D4D6F8EC0003681B6827
:108560009847032803D1D7F8383CDA070DD4D6F85A
:10857000EC0003685B6A984768B90C492046FFF72E
:10858000B1FDD8E70A4A0949D1E70B4A0749204615
:10859000FFF7C6FDB8E7D7F8383C5B07EDD5074ACB
:1085A000F4E700BF042B0D08442A0D0826FB0D0834
:1085B0004E2A0D08612A0D08712A0D08812A0D081E
:1085C00038B5044615464FF031FE012206214FF022
:1085D00089FD2046FFF7AEFE98B104F53750012221
:1085E00007213830F9F7FEFC144A15492046FFF7F9
:1085F00097FD0025294620460422BDE83840FFF7B4
:108600002DBF04F54053EDB2D3F8EC000368DB6CEA
:10861000984768B104F50053D3F8383C1B0707D5D9
:1086200035B1084A06492046FFF77AFD0125E1E702
:1086300003492046FFF756FDDCE700BF442A0D083A
:108640009E2A0D084E2A0D082DE9F041044604F536
:1086500000574FF0EBFD012208214FF043FD5AF087
:10866000BDF997F8D532072B98BF384A04F5405624
:1086700098BFD55CD6F8103193F8CB8088BF02251F
:10868000B8F1000F0BD132492046FFF72BFD002532
:10869000294620460522BDE8F041FFF7DFBE20460F
:1086A000FFF748FE60B104F537500122122138303F
:1086B000F9F798FC274A26492046FFF731FDE6E7FF
:1086C000D6F8EC000368DB6C984768B196F8AD36D5
:1086D00053B196F9AC36012B06DC1F4A1F492046E0
:1086E000FFF71EFD0125D3E7D6F8EC000368DB6C2D
:1086F000984718B1D7F8383C190713D4D6F8EC00CE
:1087000003681B689847032803D1D7F8383C9A07B9
:108710000BD4D7F8383CDB0609D40D492046FFF7C7
:10872000E1FCB5E70C4A0A49D9E70D4AC3E7D6F898
:10873000EC000368DB69984706460028EDD1094A3A
:1087400003492046FFF7ECFC3546A1E70C2B0D084A
:1087500045160D08442A0D084E2A0D08982A0D08C2
:10876000A62A0D08BB2A0D08F8B500F500550446E9
:1087700095F9D532B3B300F54056376F97B38AF009
:108780008FFD05F5496595ED000ADFED177A9FED40
:10879000171ADFED170AC71B20EE270A8D2025F0D8
:1087A00081FFBCEEC00A10EE103A9F420CD296F840
:1087B00005319A0716D520460021F9F76DFD2046B0
:1087C000BDE8F840FFF7C0BC0CD996F805319B070F
:1087D00008D420460121F9F75FFD2046BDE8F840A6
:1087E000FFF732BFF8BD00BF00007A440000804FA1
:1087F000000000002DE9F341074600F59A4081F0A2
:1088000007FE07F54054C0F3804801908AF048FD08
:1088100094F808314345454606460DD007F53A50D1
:1088200084F808813830002D41D03C4B3C4AC4F8D4
:108830000C61022151F0F6FD94F8083107F500585B
:1088400043B394F809312BBBB8F9A63C9FED350A28
:108850009FED351ADFED350A07EE903AF8EEE77A2C
:1088600040F2571027EE800A25F01CFFBCEEC00A2C
:10887000D4F80C0110EE103A361A9E420AD90123A0
:1088800007F53A5084F80931294A244B022138303F
:1088900051F0C8FD98F9A53C002B94F805310DDC8A
:1088A0006FF3451384F8053102B0BDE8F0811B4B2E
:1088B000204AC4F80C8184F80981BAE7C3F3401256
:1088C000AA42F1D065F3451384F805319B06EBD538
:1088D000194BD3F8EC0003681B6998470028E3D0D4
:1088E0004FF0A4FC01221F214FF0FCFB3846FFF79C
:1088F00021FD48B107F5375001222121383002B05F
:10890000BDE8F041F9F76EBB98F8A51C3222384655
:1089100002B0BDE8F041FFF7A1BD00BFD42A0D08A9
:10892000E32A0D0800007A440000804F0000000098
:10893000F92A0D08EE2A0D08805C002008B5044BCA
:1089400001221A708AF0A4FC024B186008BD00BF17
:108950003185002034850020014B00221A707047B9
:10896000318500202DE9F04104468AF091FC2A4B24
:10897000B4F8BE201988294E914205460ED01A80BF
:10898000274B18603378A3B1002434704FF04EFCAD
:1089900022461321BDE8F0414FF0A4BB3378214FAC
:1089A000DBB93B782BB11E4B1F4A1B68C31A93429D
:1089B00001D8BDE8F0810123337004F54053D3F8AA
:1089C000100190F8CB3013B103689B6A98474FF0C1
:1089D0002DFC012213214FF085FB3B78002BE8D0C2
:1089E0003378002BE5D00E4A10491368EB1A8B42FE
:1089F000DFD904F540541560D4F8100190F8CB305D
:108A0000002BD6D0002182F0BDFCD4F81001036801
:108A1000BDE8F0415B6A18473285002030850020B0
:108A2000348500203185002080841E0040420F00E4
:108A30002DE9F84300F5405500F500580446D5F8F7
:108A4000EC0098F88C710368DB6C9847014650B9CC
:108A500095F9E030002BA5BFD5F8103193F8CB0085
:108A6000012180F0010104F5055909F1100948467A
:108A700067F0EAFED5F8103193F8CB300646002BAC
:108A80007BD0002865D03E4B93F9E030002B04DB0F
:108A900002463C49484667F0B1FA98F9567157B119
:108AA00095F9E030002B0EDA04F5375001220F2142
:108AB0003830F9F797FA4FF0B9FB3246BDE8F84382
:108AC00009214FF00FBBD5F8EC0003685B699847AC
:108AD00058B195F9E130002B07DA95F80531DA073E
:108AE00003D498F88C31DB07DED53146484667F071
:108AF00011FFDFED257AB4EEE70AF1EE10FA05DD9D
:108B00000A220921204600F09BFFD4E7023F032FF1
:108B100011D801A353F827F0018B0108298B010814
:108B2000478B01084D8B01080A221521204600F0D1
:108B300087FF0028BFD10A220621204600F080FFCF
:108B40000028B8D1DCE70A221121F6E70A22152114
:108B5000F3E797B198F88C317BB9094B93F9E03082
:108B6000002B06DB04F53A50084A0521383051F055
:108B700059FC4FF05BFB0022A0E7BDE8F88300BF83
:108B8000805C0020142B0D080000C8421D2B0D082E
:108B900070B500F5005300F59A4586B093F87C1E39
:108BA0000446284681F0E2FB02A814F023F904F5FC
:108BB000955002A910300DF0E3FF04F58043049AAC
:108BC000C3F8F82C059AC3F8FC2C284681F020FC49
:108BD00082061AD5284681F029FC04F59945FDEE58
:108BE000C07A703504F5805417EE901A0222284698
:108BF00017EE906A14F004F994F82C35DB0706D4CC
:108C000001223146284614F0FBF806B070BD012160
:108C1000284614F087F90028F2D0F6E770B500F581
:108C2000804486B0B4F8043F8B420D46164603D10B
:108C3000D4F8003F934221D08AF032FBD4F8FC3EB6
:108C4000C31A132B1AD9C4F8006FA4F8045FC4F830
:108C5000FC0E4FF0EBFA04468AF02AFB084B094A57
:108C60001B68CDE90453084B0193084B0093CDE9F1
:108C70000201074B074920464FF064F806B070BD6B
:108C800038850020342B0D084C2B0D08C4000D082E
:108C900000E40C08472B0D0838B500F540540D468C
:108CA00094F8E130C3F380138B420BD021B14FF025
:108CB000BDFA11214FF0F6F994F8E13065F386130F
:108CC00084F8E13038BD0000F0B52DED048B00F5DF
:108CD00040568BB0D6F8103193F8CB30054600F5EE
:108CE0008044002B67D096F9E030002B63DBD6F888
:108CF000EC0003685B699847002861D1D4F81C0D2B
:108D00009FED440A6C3028F001FF0AAACDED080A55
:108D10008DED091A8DED070A12E9070004AB01AFCA
:108D200083E8070087E80700384628F03BFCD4F8C2
:108D30001C3D05F599405030D3ED368AB0EE409A8F
:108D400050F0FEFE29F0E0FAD4F8243DD6F8EC000D
:108D5000D3EDDB9A0368DB6CB0EE408A9847DFED19
:108D60002E7AB4EEE79AF1EE10FA02DC96F8E830CB
:108D70000BB100283AD0DFED297A68EEA78AF3EE2E
:108D80000E7AF4EEE78AF1EE10FA2FDCF0EE087AB4
:108D9000B4EEE78AF1EE10FA28DCF5EEC09AF1EEB7
:108DA00010FA23DAD4F81C0D03689B6F98470BB0B8
:108DB000BDEC048BF0BDD4F81C0D03689B6F0FE075
:108DC00005F50055D4F81C0DD5F8DC2C0368B2F974
:108DD0000820002A03DCD6F8E420022AEED1DB6F5B
:108DE0000BB0BDEC048BBDE8F0401847D4F81C5D17
:108DF000DFED0B0A2B68D3F88060D4F8243D40F2F5
:108E0000AB1093EDC90AB7EE001A25F04BFC2846CB
:108E1000B047CCE79F0CB3450080BB44E02E6542D1
:108E20000000000000F5405090F8E8007047000096
:108E30002DE9F04100F54055064695F8E030B1EBDC
:108E4000D31F0C4648D0254B00221A6000293FD082
:108E50004FF0ECF912214FF025F995F8E03064F36A
:108E6000C71385F8E03084F0010873F05DF84146DF
:108E700073F036F806F50057B8F1000F06D097F8F2
:108E80006A321BB98AF00CFAC7F86C0287F86A825A
:108E900014B3B7F8B8325B071ED5D5F8103193F884
:108EA000CB30CBB1D5F8EC0003685B69984798B933
:108EB000D5F8EC00036820219B69984760B106F55E
:108EC00037500122BDE8F0410D213830F9F78AB85A
:108ED0004FF0ACF91C21BEE7BDE8F08138850020D9
:108EE0002DE9F04F2DED0A8B00F540558DB0D5F8EA
:108EF000103193F8CB60044600F580471EB901217C
:108F0000FFF796FF0BE095F9E020002A65DAD5F827
:108F1000EC0003689B6C98470646002841D04FF050
:108F2000000B95F9E020B14E002AC0F25381D6ED36
:108F3000007AB4F9A420B8EE677A1AB9B4F8A2207E
:108F4000A4F8A420B4F8A430DFEDA96A07EE903AA3
:108F5000F8EEE77A67EEA67AB4EEE77AF1EE10FA69
:108F6000ACBF012100212046FFF796FE95F9E020D5
:108F7000002A95F8E120B8BF4BF0010B530697F893
:108F8000E82E48BF4BF0020B0AB14BF0080B3268D9
:108F9000594620460DB0BDEC0A8BBDE8F04FFFF7F7
:108FA0003DBED5F81031204693ED0C8AF9F744FA0E
:108FB000B4EEC80AF1EE10FAB1D5D5F8103193F835
:108FC000A130032BABD14DF03DFC4FF48011422278
:108FD0004DF0F0FB3146204692E797F8E8AEBAF143
:108FE000000F03D0814A0023136098E7D7F81C0DC7
:108FF00093F8079003685B6F984780460090D5F818
:10900000EC0003685B69984720B1D5F8E430022B87
:1090100000F0E280B9F1000F0CBF4FF0000B4FF4ED
:10902000007BB7EE00BAB8F1000F02D04BF4806BB2
:10903000009604F59D4808F1300840466AF0FEFDB0
:109040000130D7F81C0D9FED6B0A9FED6BCADFED69
:109050006B8A0CBF012302236C3008EE103A28F013
:1090600055FD0CABCDED0A0A8DED0B1A8DED090AFD
:1090700013E907000DF10C0E0DF1180C8CE8070038
:109080008EE80700704628F08DFAD7F81C2DDFED2A
:109090005C7A92ED36AA2AEE27AAB4EECC0AF3EE59
:1090A0000EBAF1EE10FA04F59940B4EEEBAAC8BF7F
:1090B0004BF4807B5030F1EE10FAC8BF4BF4807B4C
:1090C000F0EE40AA50F03CFD29F01EF9B8EEC88A37
:1090D00004F59A40B4EEC80AF1EE10FA98BF4BF0CE
:1090E000800BF0EE409A81F0ADF968EE288AB0EE80
:1090F000C09AB4EEE89AF1EE10FA204648BF4BF061
:10910000400B0AF0A1FD002846D14BF0200B019640
:1091100040466AF093FD01284FD14BF0100BB24648
:109120003249B9F1000F53D0009B002B50D0F4EE20
:10913000CCAAF1EE10FA4BDCB4EEEBAAF1EE10FA89
:1091400046DCF4EEC89AF1EE10FA41D8B4EEE89A93
:10915000F1EE10FA3CD5019BD3B3BAF1000F37D032
:109160000A68B4F9A40007EE902AB8EE677A18B935
:10917000B4F8A200A4F8A400B4F8A43007EE903A22
:10918000F8EEE77A67EE8B7AB4EEE77AF1EE10FA52
:1091900019D501320A60C4E604F53350383050F076
:1091A00077FCDFED187A90ED007AB4EEE77AF1EE15
:1091B00010FAAAD400230193AAE740466AF03EFDC4
:1091C0000130ADD1A9E701212046FFF731FEA8E625
:1091D0000022DFE70121C6E6B9F1000FB0EE08BAC0
:1091E0000CBF4FF0000B4FF4007B1FE738850020C9
:1091F000CDCC4C3E9F0CB3450080BB440000C84220
:10920000E02E65420000484310B500F5B052044618
:1092100007CA88B002AB83E807009FED1D7ADDED39
:10922000047A77EE877A9FED1B7ACDED047AD4ED40
:109230002B7AF0EEE77AF4EEC77A04F59940F1EE76
:1092400010FA00F150000BD5B4F9A22007EE902AD5
:10925000F8EEE77AF7EE006A86EEA77A84ED2B7ACD
:10926000D4F8AC200192194601AA50F037FD2046EF
:10927000FFF736FE2046FEF755F92046FEF72AFA9C
:109280002046FDF7E7FF2046FEF79CF808B010BD2A
:109290000AE81C410000003410B504462DED028B95
:1092A0001D205BF0B9F860B304F54053D3F8EC002F
:1092B00000F0C4FA192108EE100A04F5546048F0D1
:1092C0008FFD02281AD00338012808D804F533503E
:1092D000383050F0DDFB90ED008ABDEEC88AB8EE64
:1092E000C88A9FED090A28EE000ABDEC028B04F53E
:1092F0009D403030BDE810406AF026BD9FED038AE6
:10930000EDE7BDEC028B10BD0AD7233C0000000046
:10931000134A0260134A426002F1740181601249EB
:10932000C16002F52A510161083941612439816126
:10933000A2F6FC71C1610D49016202F664614162ED
:1093400002F62821816202F62C21C16202F5236116
:1093500002F634224263064A01638263704700BF0B
:10936000FC3E0D082C4F0020A87900209C7900209D
:10937000982D0020172952D8DFE801F0100C14189E
:10938000221F2A1C5126512E51513236393D41514E
:109390005144484D00F59E400C30704700F5AC40FC
:1093A0006430704700F59E404C30704700F59F4098
:1093B0000830704700F5A640F2E700F5AA40F7E74D
:1093C00000F5A8407C30704700F5A9404030704758
:1093D00000F5AB405830704700F5A7402430704787
:1093E00000F5A7406030704700F5A240FAE700F5AD
:1093F000AA404430704700F5A6402030704700F581
:10940000AD40FAE700F5AD407030704700F5005010
:10941000D0F8900B704700F5A8403430704700201A
:109420007047000073B50B6805461B6C08460C4678
:1094300016469847034605F53A500F4A0096042110
:10944000383050F0EFFF4EF0F1FE236805461B6800
:10945000204698470A21024628464EF043FE074B15
:1094600093F8E1309B0641BF054A137843F00403AB
:10947000137002B070BD00BF502B0D08805C00203F
:10948000DC86002038B50C4A182305460C464DF002
:1094900027F878B121462846FFF76CFF30B1014626
:1094A000064A2846FFF7BEFF002038BD28464CF08C
:1094B0005FFFF9E70120F8E7D02B0D08702B0D08AE
:1094C00010B500F50053002283F88C2D094B04469B
:1094D00093F8E01000F5804304F54054D3F81C0DD8
:1094E000C9097AF0D7FDD4F8EC000368BDE8104054
:1094F000DB681847805C002070B505460868036883
:109500005B690C461646984790B1306803685B6902
:10951000984768B905F54053D3F8102192F8CB204D
:1095200032B193F9E030002B02DB2846F8F79AFFBE
:1095300004480BF055F920680368BDE870409B684B
:10954000184700BF1486002070B500F5405504464A
:10955000D5F8EC000B4E0368DB6998473074D5F8FA
:10956000EC0003681B689847F070D5F8EC000368BE
:109570005B6C9847014604F59350BDE8704043F09A
:10958000B7BB00BFBD86002070B52DED028B244B0C
:1095900093F80531DB0782B006460D461446B0EE5F
:1095A000408AF0EE608A06D500232B60236002B06B
:1095B000BDEC028B70BD59F011FB037F002BF3D083
:1095C000F36A9FED181A1B689FED170AB3F908306C
:1095D00007EE103AB36A1B68B3F9083007EE903A09
:1095E000B8EEC77AF8EEE77A67EE000A68EE811AFD
:1095F00027EE800A28EE011A01A9684625F046FFE9
:10960000DFED0A6A9DED007ADDED017A27EE267A1C
:1096100067EEA67A85ED007AC4ED007AC7E700BF51
:10962000805C00200AD7233C530469390000C842FB
:1096300070B52DED028B88B0002302930393364B57
:1096400093F8053113F0010F0646B0EE408A06ADDF
:1096500002AC03D159F0C2FA037F5BB994E803006E
:1096600085E803009DED060ADDED070A08B0BDECB4
:10967000028B70BDB36ADFED296A1B68B3F908304D
:1096800007EE903AF36A1B68B3F9083007EE103A18
:10969000B8EEC77AF8EEE77A27EE267A67EEA67A72
:1096A000F1EE476ACDED026ADFED1D6ACDED037A7A
:1096B000B0EEC77AB4EEE67AF1EE10FA06D5F0EE27
:1096C000E77AF4EEE67AF1EE10FAC7D403AA21465F
:1096D0001448F8F7F7FEDDED027A9DED037AF0EE1F
:1096E000E77AB0EEC77AF4EE477AF1EE10FACCBF23
:1096F000B0EE670AB0EE470A204627F0A1FE04A8A4
:109700008DED040ACDED050A27F04CFF204688EECA
:10971000000A27F0C5FEA1E7805C002053046939E8
:1097200000000034802C0020094B93F9E020002A2F
:109730000CDAB5EEC00AF1EE10FA07D9D3F8103101
:1097400093F8A100C31E584258417047002070474B
:10975000805C0020436A1B6893F8CB3043B1054B13
:1097600093F8E00000F0A000203818BF01207047F7
:1097700001207047805C002010B5436A04461868D9
:10978000D1B1022181F00EFE236A9FED0C1A1868F8
:109790000368F0EE410ADB6AB0EE410A9847236A9B
:1097A000074A1868D2EDAD0A03689FED040A5B6EA4
:1097B000BDE81040002118470121E3E70000000048
:1097C000804C002010B5436A04461868002930D048
:1097D000022181F0E7FD236A18687AF02BFC636AA6
:1097E0001B6893F8A130012B04D8236A0121186863
:1097F0007BF0BAF9636918687EF0C6FA6369186885
:109800007EF022FB63699FED0C0A18687EF048FD2C
:10981000636918687EF0B6FD236A9FED071A186821
:109820000368BDE81040DB6AF0EE410AB0EE410A81
:1098300018470121CDE700BF0000000013B5044622
:1098400001A90C480AF090FA10B1019802B010BDBD
:10985000636918687DF0A2F918B9074BD3F8F40CC6
:10986000F4E7064801AA032113F000FB0028F4D016
:10987000EBE700BF802C0020806C00207079002076
:1098800070B504462DED028B00296AD18368B3F9C7
:109890006E58642DB8BF6425FFF7D0FFA8426268F8
:1098A000A4BF324B93F8E150B2F93430ACBFC5F3EA
:1098B00080150125002BDBBF63691B685B4293EDBC
:1098C000C48AC8BF07EE903AB2F93230C8BFB8EECA
:1098D000E78A002BB8BF5B429BB25B4207EE903A2F
:1098E000A368F8EEE77AB3F96E68F4EEC87AF1EEA1
:1098F00010FAD8BFB0EE678A2046642EB8BF64263F
:10990000FFF79CFF6369A26B1B68D2ED001A93ED11
:10991000C61AD3ED0E0A311A00EE101AB8EEC00ABC
:1099200025F0A2F96368B3F93230002BB8BF5B426F
:109930009BB25B4201EE103A40F29720B8EEC11A9A
:10994000F0EE480A24F0AEFE6369294618687DF0FF
:10995000C9F9BDEC028B6369BDE8704018687EF000
:1099600011BD9FED030A0025EEE700BF805C0020DB
:1099700000000000436A186803681B69184700006C
:1099800038B52DED028B03680446D3F88030984734
:10999000236B2A481B68F0EE408AB3F908500AF09E
:1099A000F5F84FF47A72041E4FF000012846D8BF34
:1099B0004FF4FA7424F0B4FE8442B6EE000A2ADDB5
:1099C00007EE900AB8EEE77A07EE904A27EE007AA3
:1099D000F8EEE77A87EE278A4FF46D7038EEC00A0A
:1099E000F5EE087AB1EE400A80EE270AB7EE001ACB
:1099F000FEEE000A24F056FEF7EE007A77EEC07A0B
:109A000028EE000A20EE080A20EE080AA7EE880ACF
:109A1000BDEC028B38BD031B07EE103AC4F57A7417
:109A2000B8EEC77A07EE904A27EE007AF8EEE77AAA
:109A300087EE278A38EE008ACEE700BF802C002010
:109A40002DE9F04F2DED028B00F5804900F54058CF
:109A500099F8084F89F8082F0546D8F8EC000368F4
:109A600083B01B680F4616469847B84221D105F5CA
:109A700000551A2E85F8686207D130B905F66C4595
:109A8000D9F81C3D2A68C3F8FC208C4B93F8E130D0
:109A9000980606D40124204603B0BDEC028BBDE835
:109AA000F08FB442F6D0864A137843F00203137065
:109AB000F0E7022E0CD01B2F12D105F59F40314646
:109AC000083003B0BDEC028BBDE8F04F01F066B981
:109AD00039462846FFF7D6FC04460028EBD1DAE7E2
:109AE00039462846FFF746FC0446019018B9284637
:109AF0004CF03EFCCFE7D8F8103193F8CBB00368B8
:109B00005B699847019A05F5A74324338BF0010A56
:109B10009A4208BF0120BBF1000F08D101980368E9
:109B200051465B689847044648BB664A22E098F96C
:109B3000E030002B80F2B380002800F0B080DFF826
:109B40007CB1DBF8EC0003685B69984704460028A9
:109B500040F0A5800198FFF713FFABF54050B0EE41
:109B6000408AF8F769FCB4EEC08AF1EE10FA40F3CF
:109B70009680554A01992846FFF754FC8BE705F576
:109B8000435101AA2C31284605F50054FFF7B4FCD7
:109B90000198C8F8EC0084F8686203681B6898476D
:109BA0003246014605F57F604DF052FE05F53A500C
:109BB0000021383058F026F994F9563123B105F5D3
:109BC0000550103066F0CAFED8F8EC0003681B6838
:109BD0009847C21E5042504104F63C4289F8AC0DF1
:109BE000D9F81C3D1268C3F8F82004F66C42D9F885
:109BF0001C3D1268C3F8FC20012F01D00B2F06D1A9
:109C000004F65444D9F81C3D2268C3F8FC202846C9
:109C1000FFF79AFC294B93F8E1309B063FF543AFE1
:109C200038E705F5005393F85021002A3FF476AF4A
:109C3000B3F86C21D1077FF571AF93F88C21002A1E
:109C40003FF46CAFD8F8102192F8CB20002A3FF4F3
:109C500065AF93F868320A2B7FF460AF98F9E03073
:109C6000002BFFF65BAF194A01992846FFF7DAFB94
:109C7000002410E716480AF0EDF90028D1D1D8F8F1
:109C8000EC0003685B6998470028CAD00198036814
:109C90005B69984704460028C3D10E4A6AE70198D9
:109CA00003681B6998470028E4D009480AF0C0F906
:109CB00004460028DED1084A5CE700BF805C002033
:109CC000DC8600203ED30E08982B0D08BC2B0D0817
:109CD000802C0020AA2B0D08AE860E080148FFF745
:109CE000AFBE00BF802C002013B504468DED010AE5
:109CF00069F03CFF6369A26B1B6892ED001A93ED5B
:109D00000E0AD3EDC60A01A968F0BEFD9DED010A59
:109D100002B010BD436A186803685B6A1847000008
:109D200038B5436A1C6894F8CB10054661B92046E3
:109D300081F038FB6B6A1B6893F8A10018B1012809
:109D400014BF0320022038BD164803783BBBFFF741
:109D5000EBFC20BB144A92F8E03003F0A003202B68
:109D600017D0B5EEC00AF1EE10FA10D592F8E23035
:109D70005B070CD40121204681F014FB6B6A1B6841
:109D800093F8A130012B0CBF02200320DBE7022156
:109D9000F1E72046022181F005FB0420D3E70120F2
:109DA000D1E700BF14860020805C002010B52DEDA7
:109DB000028B134B93F80531DB07044604D59FED66
:109DC000110ABDEC028B10BD58F008FF037F002B79
:109DD000F5D0636B186859F02BF8A368DFED0A7AA9
:109DE00003F5156292ED008A03F65413D3ED000AD1
:109DF00028EE278A25F004FB28EE000AE1E700BFE1
:109E0000805C0020000000000000C8420148F8F714
:109E100083BB00BF802C00200148F9F717B800BFB2
:109E2000802C00200148FFF70BBE00BF802C0020D3
:109E300070B52DED028B7D4D95F8E1308CB000268C
:109E4000044658060496059603D5636918687CF0A5
:109E500019FD95F80531D9075DD463689B899A0788
:109E60001BD573484FF014FEDFED727A90ED007A47
:109E7000B4EEE77AF1EE10FA0FDD4EF0D7F93D219E
:109E80004EF010F96C4809220521FFF7D9FD20B9E1
:109E9000092202212046FFF7C5FF636893F9543079
:109EA000CBB365489FED658AF8F7D0FFE3689FED77
:109EB000647A1B68D3ED0A7AF4EEC87AF1EE10FAF0
:109EC000B8BFF0EE477AB6EE000A27EE800A2046C9
:109ED000FFF7AEFB8DED040AB0EEC00AB4EEC80A7F
:109EE000F1EE10FACDED050A06D5F0EEE00AF4EE3B
:109EF000C80AF1EE10FA0ED495F8E2301B0704D42C
:109F00004EF094F949214EF0CDF895F8E23043F047
:109F1000080385F8E23095F8E3306FF3820385F8A3
:109F2000E330606909960A9609AD2A4604A90068DB
:109F300001237CF011FD636918687DF085FF63697A
:109F400018687DF05DF8A3688DED060ACDED070A6F
:109F50008DED081AD3ED007AF5EEC07AF1EE10FA25
:109F600052DD384B9FED388AB3F9A83200EE903AB3
:109F7000F8EEE00A2046CDED030AFFF75FFCA36888
:109F8000DDED030AD3ED001A9FED2A0AB7EE002A91
:109F900007EE900A31EE822AB8EEE71A22EE082A7E
:109FA00061EE881A24F0BEFADFED287A20EE270A47
:109FB000DFED277A20EE270AACF020FADFED257AD4
:109FC00020EE270A06A820EE088A27F0EBFAB4EE66
:109FD000C08AF1EE10FA17D5C8EE006A63699DEDEC
:109FE000067ADDED077A27EE267A67EEA67A8DED02
:109FF000067ACDED077A1B68D3F88823C3F894233B
:10A00000D3F88C23C3F89823236A13491C68284685
:10A01000FCF7E8FA0B9B009395E80C0006A9204694
:10A020007AF0BAF80CB0BDEC028B70BD805C0020F9
:10A030006479002000002F44802C002000000034B0
:10A0400000007A43804C00200000C8420AD7233C1D
:10A0500035FA8E3C0AE81C41EC84002013B5044616
:10A060000191FFF7E5FE0199204602B0BDE81040DE
:10A07000FFF706BC0148FEF7DBBE00BF802C0020C6
:10A0800000487047385B00200148F8F733BA00BF3A
:10A09000802C002030B50F4D87B000230446694660
:10A0A000D5F8240D0093019302937CF0C1FFD5F8FD
:10A0B000240D02A97DF010F8009B0393019B0493EB
:10A0C0000222029B059303A9204613F09FF9204624
:10A0D00007B030BD806C0020014B01221A70704720
:10A0E0003C8500200020704700207047002070470A
:10A0F0000020704700207047002070470020704704
:10A100000020704700207047002070479FED010A33
:10A11000704700BF0000000000207047002070471B
:10A1200000207047012070470020704700207047D2
:10A1300001207047002070470120704701207047C0
:10A1400000207047012070470120704700207047B1
:10A1500000487047E82B0D0800487047E82B0D08B1
:10A16000836893F86439DB0706D5002380F83C3018
:10A17000024B0222C3F8E42001207047805C0020DB
:10A1800090F83C3043B9836893F86439DB0742BFE9
:10A19000034B0122C3F8E420002380F83C307047D1
:10A1A000805C0020012380F83C3070472DE9F043AB
:10A1B0002DED0C8BF0EE409A20EE000A97B00025B2
:10A1C000A0EEA00A04468946B0EE41CAF0EE60AAAD
:10A1D00090461F46019502950395049505950695B1
:10A1E000ACF022FBF7EE00CAB4EEEC0AF1EE10FA86
:10A1F000C8BFCCEE807AA36803F5126203F624137D
:10A2000092ED009A9FEDC5DAD3ED000AC4BF69EE66
:10A21000A79A6AEEA7AAB0EE690A25F0F1F8A3683A
:10A2200029EE0D9A03F5126203F62413D2ED008A8B
:10A23000D3ED000A29EE009AB0EE6A0A25F0E0F8A4
:10A24000A36868EE8D8A03F6381203F63C13D3ED4B
:10A25000000A92ED008A68EE808AB0EE4C0A25F082
:10A26000CFF8636828EE0D8A93F9703028EE008AE3
:10A27000002B00F0D980236A9FEDA90A18686C3082
:10A2800027F044FCB0EE60AACDED080A8DED091A66
:10A290008DED070A24F0B0F9BDEEC0BAA14940F631
:10A2A000B8321BEE100A24F02BFA434207EE903A24
:10A2B0006368F8EEE77A93ED1A7A67EE877AB0EE84
:10A2C0004A0ACDED017A24F097F9FDEEC0BA40F6C6
:10A2D000B83294491BEE900A24F012FA42426368A5
:10A2E000039507EE902A93ED1B7A93F97030F8EE00
:10A2F000E77A022B67EE877ACDED027A6ED18A4B30
:10A30000B3F9A8320AEE103AB8EECBBAB8EECAAA40
:10A31000236AB4EECABAF1EE10FA1A683DDDA368FA
:10A32000DFED820AA16B92ED051AD1ED001A03F55B
:10A33000126393ED007A27EE0D7A3AEE4B0AC7EEE0
:10A34000200A24F091FCDDED017A37EE800A8DEDD4
:10A35000010AB8EEEB0A236AB4EECA0AF1EE10FA6B
:10A360001A6834DDA368A16B92ED061AD1ED001ACC
:10A3700003F51263D3ED000A20EE8DDADFED6B0AF0
:10A380003AEE400ACDEE200A24F06EFCDDED027AB2
:10A3900037EE800A8DED020A20E0B1EE4A0AB4EEF3
:10A3A000C0BAF1EE10FAD4D5A368A16BDFED5F0A55
:10A3B000D1ED001A92ED051A03F5126393ED007AC0
:10A3C00027EE0D7A30EE4B0AC7EE200AB9E7B1EE60
:10A3D0004AAAB4EECA0AF1EE10FAC3D4236AD3F83B
:10A3E00000C00CF184030FCB12AD85E80F000EAE58
:10A3F0000AAD86E80F0085E80F0004AB01AA2946E4
:10A4000060467AF065FB636893F97030022B16D1D1
:10A41000DDED047A39EE279ADDED057A78EEA78A2C
:10A42000DDED067A38EE278A89ED009AC8ED008ABC
:10A4300087ED008A17B0BDEC0C8BBDE8F083F0EE21
:10A44000E99AF0EEEAAAF4EEE9AAF1EE10FA48BFB2
:10A450006D46CDED009ACDED0AAAD5ED007ADFED7F
:10A46000340AB0EECCCAF4EECC7AF1EE10FAD8BFD2
:10A4700035468DED0ECA95ED007ADFED2E7A87EE2A
:10A48000270AAD20B7EE001A3CEEC00A24F00AF904
:10A49000E369D3ED937A04A820EE270A27F036FB70
:10A4A000F0EEC07A8DED061AB0EEC91A31EE671AD9
:10A4B0008DED040AB0EEC11A39EE000ACDED050AA1
:10A4C000B520F1EE410A24F0EDF8B0EE409A9DED92
:10A4D000050AB0EEE81AF0EEC07A31EE671A38EEEF
:10A4E000800AB0EEC11AF1EE410ABA2024F0DAF87F
:10A4F000F0EE408A9DED060AB0EEC81AF0EEC07A82
:10A5000031EE671A38EE000AB0EEC11ABF20F1EE44
:10A51000410A24F0C7F8B0EE408A85E70000C8423F
:10A520009F0CB34548F4FFFF804C002000007A44A4
:10A530000000000000A08C4510B52DED028B836A51
:10A54000044686B0186858F073FCE36A1868B0EEE9
:10A55000408A58F06DFC636B8DED010A186858F065
:10A5600067FC05ABB0EE401A03A92046DDED010AF9
:10A5700004AAB0EE480AFFF719FE636A186890F85B
:10A58000CB1000293AD180F00DFF2046FFF7F8F9F3
:10A59000636A1B6893F8A1100129B0EE408A3DD090
:10A5A000032944D051B9236A012118687BF092F93C
:10A5B000236A186879F028FD9FED208A236AA26833
:10A5C000186892F8642903689DED030ADDED040A1A
:10A5D0009DED051A92074CBFDB6B9B6B9847236A76
:10A5E000174A1868D2EDAD0A036800215B6EB0EE21
:10A5F000480A984706B0BDEC028B10BD114B93F989
:10A60000E120002A06DBD3F8E430022B04D190F8D5
:10A61000A1300BB90121B6E70221B4E7236A18681B
:10A620007BF058F9236A186879F004FDC4E7D979FA
:10A630000029C3D12046FFF71DFDBFE70000000041
:10A64000804C0020805C0020836893ED140AB5EEF6
:10A65000C00AF1EE10FA01DCFFF78CB97047000078
:10A6600070470000002070470120704702207047AB
:10A67000002070470020704701207047002070477D
:10A6800081F00100704700000120704701207047F1
:10A6900000487047802C0D08004870478C2C0D082E
:10A6A00038B54369044618687CF09AFB18B96369A9
:10A6B00018687DF019FD636920461D68FFF7E4FC0A
:10A6C0006368B3F93820B3F9363000EE903A43426C
:10A6D00001EE102A00EE103AB8EEC11AF8EEE00AC8
:10A6E000B8EEC00A28467CF067FA636920461D6808
:10A6F000FFF7CAFC6368B3F93820B3F9363000EECF
:10A70000903A434201EE102A00EE103A2846B8EE85
:10A71000C11AF8EEE00AB8EEC00A7CF0C7FA0120D0
:10A7200038BD000030B52DED028B0446436985B07D
:10A730001D68FFF7A9FC6368B3F93820B3F9363018
:10A7400000EE903A434201EE102A00EE103AB8EEC5
:10A75000C11AF8EEE00AB8EEC00A28465B4D7CF05C
:10A760002BFA2046FFF758FBB5F9A83208EE103A4D
:10A77000236A186803689B6E9847B8EEC88AF0EEA3
:10A78000400A02AA01A9B0EE480A2046FEF7FCFEE4
:10A790002046FFF70BFB236B1B68B3F90830F0EE84
:10A7A000408A00EE103A2046B8EEC00AFFF72EFBB2
:10A7B0002046B0EE408A8DED030AFFF765FC636822
:10A7C000B3F9363001EE103A434200EE903AB8EE5B
:10A7D000C11AF8EEE00A2B20B0EE480A23F062FF1F
:10A7E00020468DED030AFFF79BFA042813D8DFE813
:10A7F00000F0032F252A4B00236A186879F004FC27
:10A80000236A002118687AF0AFF963699FED300A76
:10A8100018687DF045FD236ADDED020A18689DED9C
:10A82000010A0368B0EE681ADB6A98476369186822
:10A830007DF0A8FD05B0BDEC028B30BD236A01217F
:10A8400018687AF091F9236A186879F0F3FBDCE76D
:10A85000204D2B7863B963689FED1F1ADFED1C0A4A
:10A8600093ED040A452023F01DFF284609F0A0FFC0
:10A8700020469DED030AFFF737FA16488DED030ACF
:10A8800003A909F0CFFFC6E7636A0221186880F0C8
:10A8900089FDB5F9A832114800EE103A02AA01A9C3
:10A8A000B8EEC00A67F020FD20469DED030AFFF7D1
:10A8B0001BFA0B488DED030A09F072FA63699DEDEE
:10A8C000030A18687CF0FEF9A5E700BF804C002061
:10A8D000000000001486002000007A44C07A0020A6
:10A8E000005A00200020704790F8B931002B14BFA7
:10A8F0001B20032070470000002070470120704794
:10A9000090F89001062804D0A0F10A03584258415B
:10A9100070470120704700000120704701207047F8
:10A9200090F8B901034A044B002814BF104618469A
:10A93000704700BF242D0D08CA990E0890F8B90180
:10A94000034A044B002814BF10461846704700BF46
:10A95000302D0D08CA990E0890F890010B3818BFD9
:10A960000120704790F8B9312BB9044BD3F8880C0B
:10A9700000F0010070470020704700BF804C0020AD
:10A9800090F8903123B9034B187880F0010070479C
:10A9900000207047F885002038B590F89041012CD0
:10A9A000054601D0002038BDC368186803681B69DC
:10A9B00098470028F6D1EB681B68204683F8B84812
:10A9C000F1E70000C3681B68002283F8B828012063
:10A9D0007047000070B52DED028B002380F8B9316F
:10A9E000B0F87030012B84B004460D4601D8002920
:10A9F00046D0636A254E1B6893F8CB3073BB24485E
:10AA0000072384F890310368022B02D10021FBF761
:10AA1000F3FB9FED208AE368F0EE480A1868B0EE79
:10AA2000481AF0EE481AB0EE480A01257EF030FFD1
:10AA300084ED738A84ED748A84ED758A84F8B85144
:10AA400004F59A7027F04AFD134805F0D9F896F8F6
:10AA5000E2306FF3C30386F8E23011E096F9E0309C
:10AA6000002BCCDA04F13C0029F02AFE0546002830
:10AA7000C5D12046FFF704FB084A02214FF0D2FC63
:10AA8000284604B0BDEC028B70BD00BF805C002086
:10AA9000EC84002000000000FC800020382D0D0810
:10AAA00038B5094D95F8C83F012B044603D105F68A
:10AAB000C47027F07BFD95F8351E04485AF0F8FE67
:10AAC000002384F8B93138BD806C00203C7A002026
:10AAD00010B52DED028B094B0446D3F8280DB0EECE
:10AAE000408A7EF06DFA9FED060A28EE008A01206A
:10AAF00084ED748ABDEC028B10BD00BF806C002019
:10AB00000AD7233C10B52DED028B094B0446D3F830
:10AB1000280DB0EE408A7EF063FA9FED060A28EE1B
:10AB2000008A012084ED758ABDEC028B10BD00BF48
:10AB3000806C00200AD7233C10B52DED028B094B09
:10AB40000446D3F8280DB0EE408A7EF057FA9FED08
:10AB5000060A28EE008A012084ED738ABDEC028B80
:10AB600010BD00BF806C00200AD7233CC3681B685F
:10AB700018697CF077BB000038B5D0F894310446F2
:10AB80000D461BB988F08CFBC4F8940188F088FB53
:10AB9000D4F89431C01A4FF47A73B0FBF3F0B4F8E0
:10ABA0009231984209D32046FFF76AFA2B88044A6B
:10ABB00006214FF037FC012038BD0020FCE700BF24
:10ABC000542D0D0890F89031052B05D1054BD3F885
:10ABD000303DD8687CF0BEBAC36818680368DB688B
:10ABE000184700BF806C002008B590F89031052B05
:10ABF0000BD1094BD3F8303DD868243026F0D2FC75
:10AC0000BCEEC00A10EE100A08BDC36818680368DD
:10AC10009B689847F4E700BF806C002090F8903163
:10AC20008B4206D00B2B80F8901102D10148FCF723
:10AC3000B5BF7047802C002073B501231E4E80F8ED
:10AC40007530D6F8EC30834205460A4614D101240B
:10AC500085F8B941D6F8EC00019203681B68984763
:10AC6000019A014615484CF0F3FD96F8E1309A063A
:10AC70001BD4204602B070BD01910321FFF7D2F82A
:10AC8000019A04460028E2D185F875004DF0CEFA0D
:10AC90001B220A214DF026FA96F8E1309B06E8D5F2
:10ACA000074A137843F0040303E0054A137843F09E
:10ACB00002031370DDE700BF805C0020703C0020C1
:10ACC000DC86002030B585B004460D460146684656
:10ACD000FFF7E0F9694604F13C002AF0A3FAC8B98D
:10ACE0004DF0A4FA1B220A214DF0FCF90D4B93F80C
:10ACF000E1309B0604D50C4A137843F0040313702B
:10AD00002046FFF7BDF9094A04214FF08BFB0020D4
:10AD100005B030BD2946204605B0BDE83040FFF7FC
:10AD20008BBF00BF805C0020DC860020682D0D08F2
:10AD300030B585B004460D4601466846FFF7AAF9CE
:10AD4000694604F13C002AF091FAC8B94DF06EFA58
:10AD50001B220A214DF0C6F90D4B93F8E1309B06FA
:10AD600004D50C4A137843F0040313702046FFF710
:10AD700087F9094A04214FF055FB002005B030BD8A
:10AD80002946204605B0BDE83040FFF755BF00BF5B
:10AD9000805C0020DC860020A42D0D087FB50546D0
:10ADA0000E4605F13C0401466846FFF773F9694613
:10ADB00020462AF05BFAC0B9204669462AF032FAEA
:10ADC000044690B94DF032FA1B220A214DF08AF95F
:10ADD0000D4B93F8E1309B060FD42846FFF750F94E
:10ADE0000A4A04214FF01EFB04E031462846FFF7D3
:10ADF00023FF0446204604B070BD054A137843F093
:10AE000004031370E9E700BF805C0020DC2D0D080F
:10AE1000DC86002030B5044685B00F4809F008F9FB
:10AE20000546B0B1072384F89031002301930293C3
:10AE30000393E36801A918687EF05CF8E36818687A
:10AE4000036801A95B680022984704480021FBF7CA
:10AE5000D3F9284605B030BD802C0020EC840020BA
:10AE6000F0B5424FD7F8FC2CD7F8F83C2DED028B0B
:10AE70001343D7F8F42C134387B005460C460CD186
:10AE80004BF0E0FC40F275124FF4801107B0BDECBE
:10AE9000028BBDE8F0404BF08DBC80697FF0C6FAB4
:10AEA0002046B0EE408A11F0D5FF03283AD1EB6876
:10AEB00001A918687EF0FAF8064698B3DDED017A2C
:10AEC0006368009338EE678A294BDFED2A7A93F99D
:10AED000E0309FED290A2948002BA8BFB0EE670A91
:10AEE00038EE008A009BBDEEC88A002118EE102AB9
:10AEF0009342ACBF00930092FBF77EF96B69186830
:10AF00007DF0F2F8DDED007A1D48B8EEE70A314633
:10AF100009F008FF00212846FFF780FE07B0BDECCE
:10AF2000028BF0BD94E80F0002AE86E80F00D7F860
:10AF3000F83C04936A46D7F8FC3C0593022130465E
:10AF400011F094FF78B94DF071F9022215214DF0FE
:10AF5000C9F8DDED037AF8EEE77A77EE887AFDEE50
:10AF6000E77ACDED007A0026AEE700BF806C0020C6
:10AF7000805C0020000000000000C842EC8400203B
:10AF8000F885002030B52DED028BC36887B00446EC
:10AF900018680D467EF07EF800284BD194F8902179
:10AFA00000230093019302936AB93148039303A9E4
:10AFB0000493059309F0E8FE28B1039B0093049BDA
:10AFC0000193059B029394ED730A9FED2A8AE3682F
:10AFD000DDED000A9DED011ADDED021A1868B4EEF0
:10AFE000C80AF1EE10FAAABFDFED237A9FED230A1B
:10AFF00020EE270A7EF04CFCD4ED747AF4EEC87A89
:10B00000F1EE10FA07DBE3689FED1B0A186827EEE4
:10B01000800A7DF0D5FFD4ED757AF4EEC87AF1EEB2
:10B0200010FA07DBE3689FED140A186827EE800A20
:10B030007DF0D6FFE368294618687EF051FB05468F
:10B0400088B10F4B1B68022B09D0032B03D10D4B8A
:10B0500093F9D9321BB10A480021FBF7EDF8012121
:10B060002046FFF7DBFD284607B0BDEC028B30BD64
:10B07000F8850020000000340000C84200000000F5
:10B08000EC840020804C002010B52DED028BC368AD
:10B09000DFED348A1B684269D3ED0A0A9FED328ADC
:10B0A00093ED060AF4EEE80A0446F1EE10FA106891
:10B0B000B8BFF0EE480A7BF065FBE36862691B6885
:10B0C0001068D3ED0A0A93ED060AF4EEE80AF1EEF1
:10B0D00010FAB8BFF0EE480A7BF0CCFB6369186841
:10B0E0007BF05CFD18B9636918687CF097FDE36834
:10B0F00062691B68106893ED080A93ED0C1AD3ED92
:10B10000070AB0EEC00A7BF057FDE36862691B686E
:10B11000106893ED080A93ED0C1AD3ED070AB0EE10
:10B12000C00A7BF0C3FD636918687BF059FE18B94B
:10B13000636918687CF0D8FF00210C48FBF75CF8C5
:10B140000B4868F099FE0B4AB2F8E23023F48163B1
:10B15000A2F8E230BDEC028B20460221BDE810408F
:10B16000FFF75CBD0000003400007A43EC8400204F
:10B17000307B0020805C002010B50C4B0446D3F8D7
:10B18000300D90ED0B0A90F8502000F11C017DF07D
:10B19000F9FB07480368022B02D00821FBF72CF8C3
:10B1A00020460521BDE81040FFF738BD806C002027
:10B1B000EC840020F0B52DED028B4A4DDFED4A8A7C
:10B1C000B0EE408A8FB00446D5F8300D0E461746D3
:10B1D0007DF04EFAF0EEC87AF4EEE87AF1EE10FA6D
:10B1E00007D49FED420AD5F8300D28EE000A7DF015
:10B1F000A5FAD5F8300D90ED0B0AB0EEC00A0FB1EC
:10B20000B1EE400A7DF08AFA0023D5F8300D07939D
:10B2100002AA07A9089309937DF0ACFADFED347A0E
:10B220009DED027AB4EEE77AF1EE10FA56DD0222D5
:10B2300007A90AA812F0EAF871680191304611F0E6
:10B2400009FE019902460AA811F0DAFDE3680AA98D
:10B2500018687EF045FA10B92648FDF799F8A069FC
:10B260007FF0E2F802684368D5F8300D049303A933
:10B270001C30039226F0C8F805A88DED050ACDED27
:10B28000060A26F08FF91C4B1B68022B1BD0D5F841
:10B29000303D1948D3ED0A7AF4EEE87AF1EE10FA6F
:10B2A000B8BFD3ED047AF4EEC07AF1EE10FA4FF0A5
:10B2B000000110D5DFED117AB4EEE70AF1EE10FAD5
:10B2C00009DDFAF7B9FF04212046FFF7A7FC0FB00C
:10B2D000BDEC028BF0BDFAF78FFFF4E72046FFF7D5
:10B2E0004BFFF4E7806C0020000000340000C842EF
:10B2F00000009643802C0020EC8400200000FA43DC
:10B3000070B52DED028B294BDFED298AD3F8284D3E
:10B31000D3F8245DD4ED0A0A9FED268A94ED060A3F
:10B32000F4EEE80AF1EE10FAB8BFF0EE480A06466D
:10B3300028467BF027FAD4ED0A0A94ED060AF4EECB
:10B34000E80AF1EE10FAB8BFF0EE480A28467BF0A2
:10B3500091FA28467BF022FC10B928467CF05EFC6E
:10B3600094ED080A94ED0C1AD4ED070AB0EEC00A69
:10B3700028467BF021FC94ED080A94ED0C1AD4EDDC
:10B38000070A2846B0EEC00A7BF090FC28467BF006
:10B3900027FD10B928467CF0A7FE07480021FAF7E0
:10B3A0002BFFBDEC028B0123337070BD806C00203D
:10B3B0000000003400007A43EC84002008B5074800
:10B3C000D0F8883C9B0704D50121A0F50050F6F782
:10B3D000FFFEBDE80840024809F004BB804C002095
:10B3E000F885002030B589B00446FEF7B3F930B1D6
:10B3F0000021204609B0BDE83040FEF7E3B9636A9A
:10B40000022118687FF0CEFFE368186803685B6963
:10B41000984701461048FCF7A9FE636918687CF05C
:10B42000B1FF236A1D68636918687BF0E9FD05AC0C
:10B4300020460A498DED020ACDED030A8DED041A6E
:10B44000FBF7D0F8079B009394E80C0002A928466C
:10B4500078F0A2FE09B030BD802C0020EC840020E2
:10B4600038B50446FEF776F9054628B12046002196
:10B47000BDE83840FEF7A6B9636A022118687FF07C
:10B4800091FF29462046BDE83840FEF7E7BD0000A1
:10B490000148002106F0C2BE5882002030B5174D89
:10B4A0009FED170A05F5804389B00446D3F8300DA7
:10B4B0007DF0C8FA01462846FCF758FE6369186813
:10B4C0007CF060FF236A1D68636918687BF098FD53
:10B4D00005AC20460B498DED020ACDED030A8DED3A
:10B4E000041AFBF77FF8079B009394E80C0002A96D
:10B4F000284678F051FE09B030BD00BF802C0020F6
:10B5000000000000EC84002030B589B00446FEF74E
:10B5100021F930B10021204609B0BDE83040FEF7E6
:10B5200051B9636A022118687FF03CFFE36818682C
:10B5300003685B69984701461048FCF717FE63698A
:10B5400018687CF01FFF236A1D68636918687BF028
:10B5500057FD05AC20460A498DED020ACDED030AE0
:10B560008DED041AFBF73EF8079B009394E80C005E
:10B5700002A9284678F010FE09B030BD802C0020CA
:10B58000EC84002030B52DED028B83B00446FEF72D
:10B59000E1F820B9636A1B6893F8CC3043B9002105
:10B5A000204603B0BDEC028BBDE83040FEF70AB97F
:10B5B00094F89831DA071DD4E3681D682B68284693
:10B5C0009B689847D5ED097A94F89831B4EEE70A6C
:10B5D000F1EE10FA4CBF0122002262F3000384F85E
:10B5E000983107D4204603B0BDEC028BBDE8304053
:10B5F000FFF7F8BE94F898319B0734D4E368DFED89
:10B60000458A1B686269D3ED0A0A9FED438A93ED70
:10B61000060A1068F4EEE80AF1EE10FAB8BFF0EE90
:10B62000480A7BF0AFF8E36862691B681068D3EDE5
:10B630000A0A93ED060AF4EEE80AF1EE10FAB8BF32
:10B64000F0EE480A7BF016F9636918687BF0A6FAF9
:10B6500018B9636918687CF0E1FA94F8983143F0FE
:10B66000020384F898312D4BD4F8A021D3F8F43C90
:10B670009B1A07EE903AB8EEE78AF1EE047AB0EE44
:10B68000C87AB4EEE77AF1EE10FA38D594F898312A
:10B6900043F0040384F89831204684ED678AFEF76E
:10B6A000C7FB6369A26B1B68D2ED001A93EDC61A43
:10B6B000D3ED0E0AB1EE480A23F0D6FA63691B688F
:10B6C00040F2AA4093EDC31AD3EDC40A22F0EAFF78
:10B6D0002046FEF709FB12488DED010A08F060FBD9
:10B6E00063699DED010A18687BF0ECFA63691868DC
:10B6F00003B0BDEC028BBDE830407CF043BED4ED1E
:10B70000677A68EE277AF5EEC07AF1EE10FAC3D5C3
:10B71000BCE700BF0000003400007A43806C0020CA
:10B72000005A002030B52DED028B83B00446FEF7A1
:10B7300011F820B9636A1B6893F8CC3043B9002133
:10B74000204603B0BDEC028BBDE83040FEF73AB8AE
:10B750006369DFED347A1B6894ED710A93EDC31AC7
:10B76000D3EDC40A20EE270A40F2C44022F09AFF2B
:10B770002046FEF7B9FA236A186803689B6EB0EE9C
:10B78000408A9847284BB3F9A83207EE903AB4F8AC
:10B79000BC316425F8EEE77A13FB05F3B4EEE70A53
:10B7A00007EE103A94F9BE31F1EE10FAD8BFF0EE80
:10B7B000407A13FB05F39FED1D0AF8EEC76A07EE0A
:10B7C000103AF4EE407AB8EEC77AF1EE10FA58BFAC
:10B7D000B0EE670A6846CDED006A8DED017A25F07E
:10B7E00033FF236ADDED010A1868B4F8C03102683E
:10B7F0009DED000A126B13FB05F301EE103A0121D7
:10B80000B8EEC11A90476369B0EE480A18687BF039
:10B8100059FA636918687CF0B5FD03B0BDEC028B82
:10B8200030BD00BF0000C842804C002000007A44B8
:10B830002DE9F0432DED028BB64F85B00446D7F8C5
:10B84000EC00FDF787FF48B1D7F8EC00002105B008
:10B85000BDEC028BBDE8F043FDF7B4BF07F58056A1
:10B86000D7F8100102217FF09DFDD6F81C3D93ED25
:10B87000378A87F015FDB7F8E03003F481430546B9
:10B880007BB1D6F8240D7AF0FDFF2378022B08D186
:10B8900055F09CFCA04BA14A06214EF0C3FD0323AA
:10B8A000237063F0EFFF63F0D9FF48B163F0EAFF64
:10B8B00063F0DEFF20B12378012B10D9022B1DD0BD
:10B8C0002378082B00F28581DFE813F0210039008E
:10B8D00063000A013E0145015A015C012A0055F04E
:10B8E00075FC8D4B8E4A06214EF09CFDD6F8243D0A
:10B8F000D3F85433636108232370E1E755F066FC05
:10B90000854B884A06214EF08DFD0323F4E7D6F8D7
:10B91000280D03681B69984710B12046FFF7F0FC1B
:10B920002378082B00F27381DFE813F05C016401D7
:10B9300064017A017A017A017A0182018201A560AB
:10B94000D6F8243D9FED787AD3F854336361774B72
:10B9500003F6C842D2ED007AF4EEC77AF1EE10FA9F
:10B960004EDB9FED737A67EE877AD6F8283D93ED2C
:10B97000087AB0EEC77AF4EE477A4FF07E53F1EED4
:10B9800010FA48BFB0EE677A2361022384ED067A8D
:10B990002370D4ED016A9FED647AD6F8243DF0EE71
:10B9A000E67AF4EEC77AF1EE10FA0AD4D4ED057A0D
:10B9B00093EDD56A77EEC67AF4EEE76AF1EE10FA07
:10B9C00029D4DFED5C6AD4ED067A67EEA67AD3ED72
:10B9D000DB6AF4EEE76AF1EE10FA26DCA368D4ED38
:10B9E000047AEB1AB3F5FA6F21D2B4EE678AF1EE5E
:10B9F00010FAC8BFB0EE678A84ED048AE5608FE76D
:10BA0000B3F9DE32002BB8BF5B429BB207EE903A2F
:10BA1000F8EEE77AA9E70623237055F0D7FB3E4BF3
:10BA2000454A04214EF0FEFC7AE7A56078E7DFF88E
:10BA3000FC8008F6BC43D3ED006A67EEA67AF4EE0C
:10BA4000C87AF1EE10FAD9D408F54C69D9ED007A2C
:10BA5000F4EEC77AF1EE10FA22DB98F8F03C33B935
:10BA60000623237055F0B2FB2B4B344AD9E7A8F5D7
:10BA7000005008F0E9F898B198F9063D83B9B8F993
:10BA8000F23CD9ED007ADFED2A6A07EE103A67EE54
:10BA9000A67AB8EEC77AB4EEE77AF1EE10FAADDC2A
:10BAA000E068281AB0F5FA7F7FF63AAF03232370D7
:10BAB00008F6BC4855F08AFB98ED007AD4ED047A7C
:10BAC00067EE277A054617EE900AF4F71DFD124B34
:10BAD0001B4ACDE90001062128464EF0A3FC1FE7D2
:10BAE000D6F8240D7CF07CFB63F0CCFE63F0B6FE50
:10BAF00068B155F06BFB084B124A06214EF092FCE0
:10BB000063F0C0FE63F098FE0423237008E705236A
:10BB1000FBE700BF805C0020282E0D08362E0D08A4
:10BB2000402E0D08572E0D0800000034804C0020D8
:10BB30000000C842333373BF692E0D08842E0D08F0
:10BB4000B42E0D08DC2E0D0863F09CFE63F086FE1B
:10BB5000C0BB05232370404BE068DFED407AD3ED96
:10BB6000006A9FED3F7A2D1AA6EEA77A07EE905A4B
:10BB7000F8EE677AF4EEC77AF1EE10FA3FF5D0AE40
:10BB800007232370D6F8243D9FED367AD3EDC37A90
:10BB9000D3EDC66A67EE877AB6EE007A67EEA77ACB
:10BBA00067EE877A87EEA67AD4ED057A77EEC77AC4
:10BBB00093EDD57AF4EEC77AF1EE10FA3FF6B0AE17
:10BBC0000823A2E763F05EFE63F052FE0028C0D1B6
:10BBD000A6E64AF037FE40F29C524FF480114AF03C
:10BBE000E9FD9DE6204805B0BDEC028BBDE8F043C1
:10BBF000FFF7F8BBD7F8EC00FEF71AF994ED060A48
:10BC00000121B1EE400AD6F8240D7BF06BF8D6F88E
:10BC1000240D05B0BDEC028BBDE8F0437CF0B2BB57
:10BC2000D7F8EC00FEF704F99FED100A0021EAE7CF
:10BC30009FED0E8AD7F8EC008DED038AFEF7F8F839
:10BC4000D6F8240D0123B0EE480A03AA04F114012A
:10BC50007BF04EFEDBE700BF4459002000007A4431
:10BC60000000FA43CDCCCC3D087C00200000000051
:10BC700030B590F8B83185B00446F3B1684611F09C
:10BC8000B9F8414869460AF0CBFF50B104F13C00D5
:10BC900029F0B4FA002384F8B83104F59A7026F03C
:10BCA0001DFC94F890310B2B2DD8DFE803F0294BC5
:10BCB0004F534B572C5B5F632C6700F59A7026F04F
:10BCC0000DFC04F13C0590B194F84030012B0ED1ED
:10BCD00094F89031012B0AD1284629F0FDF850B193
:10BCE0002046FEF7CDF9294A02214EF09BFB28465B
:10BCF00029F020F9D5E72046FEF7C2F9244AF3E7F8
:10BD00002046FFF75BFB94F844303BB994F846308B
:10BD100023B994F840309A1E5342534194F8B92104
:10BD200082B37BBB84F8B9311A4BD3F8EC000368BB
:10BD30001B689847014618482D2205B0BDE83040E1
:10BD40004BF086BD2046FFF74DFBDCE72046FFF7B2
:10BD500087FBD8E72046FFF79BFBD4E72046FFF799
:10BD60009DFBD0E72046FFF7CFFBCCE72046FFF74F
:10BD700009FCC8E70948FFF75BFDC4E72046FFF769
:10BD8000D1FCC0E705B030BD303F0020F82E0D08D3
:10BD9000202F0D08805C0020703C00203C85002096
:10BDA0002DE9F0412DED028B074684B008460E4682
:10BDB00011F050F8032880466D4628D1FB681868BA
:10BDC0007CF0CEFF012822D12148294607F0CCFF84
:10BDD0000446B0B17B69DDED007A1B68F8EEE77AC6
:10BDE00093EDF27A77EEC77A4246FDEEE77A17EEE8
:10BDF000901AC829CDED007AB8BFC821304610F09E
:10BE0000FFFF204604B0BDEC028BBDE8F081114B72
:10BE10000FCB85E80F00304611F01CF8014628468C
:10BE200011F080F804460028EBD07B69DDED017A43
:10BE30001B68B8EEE78AD3EDF27A284638EE678AB7
:10BE400011F008F8BDEEC88A024618EE101AD5E7C0
:10BE5000802C00207079002010B543699FED126A94
:10BE60001B68D3EDF06A93EDF17AD3EDF27A86B0E8
:10BE700066EE866A27EE067A67EEC67A68460C4654
:10BE8000CDED006A8DED017ACDED027A25F002FE4E
:10BE900003A920468DED030ACDED040A8DED051AA8
:10BEA00011F008FB06B010BD0AD7233C30B50832AC
:10BEB00004461D460FCA84E80F00134301BFAB6858
:10BEC000A360EB68E360636885B093B9204610F027
:10BED000C1FF03AA0146284610F0C8FF60B10399CC
:10BEE0000191204610F0B6FF01990246204610F05D
:10BEF00087FF204605B030BD696801912846F1E70B
:10BF000030B50B6985B004460BB94B6953B30023B8
:10BF1000C4F8B43108310FC96D4685E80F002946D1
:10BF20002046FFF73DFF98B9124B0122D3F8F41CCD
:10BF3000284610F065FF4CF079F9022215214CF0EB
:10BF4000D1F82046FEF79CF80B4A02214EF06AFA1F
:10BF500029462046FFF716F810B90848FCF718FAEA
:10BF600005B030BD0123C0F8B43105B0BDE83040A4
:10BF7000FFF78AB8806C0020542F0D08802C002019
:10BF800070B51A4B04460E460FCB88B06D4685E857
:10BF90000F0020462946FFF75FFFE36818687DF031
:10BFA00079F898B1E368186803681B69984768B125
:10BFB000E368294618687CF0DFFE38B94AF042FC95
:10BFC00040F295624FF480114AF0F4FB214604A838
:10BFD0002B463246FFF76AFF04A92046FEF7D2FF40
:10BFE00010B90348FCF7D4F908B070BD707900208F
:10BFF000802C002070B5154B0C4606460FCB88B040
:10C000006D4685E80F0029463046FFF725FF2B4691
:10C010002246314604A8FFF749FF6288A388122A06
:10C020004FEA132305D1227ED20744BF03EB8303DB
:10C030005B00227A07EE903AC2F34002B8EE670A3C
:10C0400004A93046FFF7B6F808B070BD707900203B
:10C0500038B504460D46FFF793FF0023C4F894312A
:10C06000AB88A4F8923138BD7FB50D460446FFF782
:10C0700087FF05F108010FC96E4686E80F001343DC
:10C0800006D1234BD3F8F82CD3F8FC3C029203934F
:10C0900004F5D0720121304610F0E8FE94F8983192
:10C0A00070B923F0050343F0050384F89831204666
:10C0B000FDF7E6FF174A06214EF0B4F904B070BD53
:10C0C00023F0070384F898310023C4F89C31E36817
:10C0D00062691B68106893ED080A93ED0C1AD3EDA2
:10C0E000070AB0EEC00A7AF067FDE36862691B6870
:10C0F000106893ED080A93ED0C1AD3ED070AB0EE21
:10C10000C00A7AF0D3FD08212046FEF787FDD5E767
:10C11000806C0020802F0D082DE9F0438DB06D4616
:10C1200088461C46074613460A4601462846DDE96E
:10C130001469FFF7BBFE95E80F0084E80F0007A81D
:10C1400010F058FEB8F80430F3B9B8F80010013117
:10C1500005AA89B207F13C0028F06AFAA0B123468B
:10C1600005AA39462846FFF7A1FE95E80F0086E8A4
:10C170000F00BDF81630A3F152025342534189F823
:10C1800000300DB0BDE8F08394E80F0086E80F00A2
:10C190000023F4E770B58B8892B004460D4616462E
:10C1A000002B47D10DA810F025FE298801310BAADC
:10C1B00089B204F13C0028F03BFA00283AD0BDF8DF
:10C1C0002E1052291CD019D8112913D80F2913D990
:10C1D00033462A46214603A8FFF768FE03AB2146F3
:10C1E00007A80BAAFFF762FEE36807A918687DF0AD
:10C1F000B7FA01E01329EBD012B070BD5E29FAE75F
:10C2000007AD03A810F0F6FD284610F0F3FD0DF180
:10C210000B03CDE90053324603AB0BA92046FFF7D1
:10C220007BFFE0689DF80B3000682A4603A97DF08B
:10C230006DFAE1E70120DFE770B5214B04460E46B9
:10C240000FCB88B06D4685E80F0020462946FFF7E2
:10C2500003FEE36818687CF01DFF98B1E368186876
:10C2600003681B69984768B1E368294618687CF041
:10C2700083FD38B94AF0E6FA40F216624FF48011B5
:10C280004AF098FA214604A82B463246FFF70EFEE4
:10C2900004A92046FEF776FE20B90A48FCF778F894
:10C2A00008B070BD0023C4F89431B388A4F892316B
:10C2B00004AA31462046FFF76DFF0028F0D1ECE7D5
:10C2C00070790020802C0020F0B5324B04460E46D9
:10C2D0000FCB91B004AD85E80F0020462946FFF74B
:10C2E000BBFDE36818687CF0D5FE98B1E368186878
:10C2F00003681B69984768B1E368294618687CF0B1
:10C300003BFD38B94AF09EFA4FF4DF624FF48011DA
:10C310004AF050FA0CAF08A810F06CFD384610F047
:10C3200069FD0DF10F03CDE900732A4608AB3146D4
:10C330002046FFF7F1FEE0689DF80F3000683A46AE
:10C3400008A97DF029FD20B91348FCF721F811B0A8
:10C35000F0BD0023C4F89431B388A4F8923108AA40
:10C3600031462046FFF716FF0028EDD00B4B1B6827
:10C37000022B09D0032B03D1094B93F9D9321BB1FE
:10C3800006480021F9F758FF01212046FEF746FC38
:10C39000DDE700BF70790020802C0020EC840020B5
:10C3A000804C002037B504460D4686F079FFC4F86E
:10C3B000A801D5ED027AF5EEC07AF1EE10FA17DD9C
:10C3C0009FED137A67EE877AFCEEE77AC4ED697A1F
:10C3D0002046FDF755FED4F8A4214FF47A73B2FB42
:10C3E000F3F30C4A062103B0BDE830404EF01AB812
:10C3F00063F038FD0023009395F90D2095F90E3078
:10C4000095F90C1063F0CAFCC4F8A401E0E700BF82
:10C4100000007A44982F0D0810B5B1F90A30A0F841
:10C42000BC3191F90C3080F8BE31B1F90D30A0F873
:10C43000C031B1F90F3007EE903AF8EEE77A0446D2
:10C44000C0ED717A86F02CFF0B21C4F8C80120469C
:10C45000BDE81040FEF7E2BB38B504460D4686F055
:10C460001FFFC4F8B001D5ED027A9FED047A67EEA4
:10C47000877AFDEEE77AC4ED6B7A38BD00007A4426
:10C480004A7C06480B46003A91F91010D3ED030A96
:10C4900093ED020A18BF0122F9F7D8BEEC84002000
:10C4A00070B51B4E0446D6F8EC00036886B01B68D6
:10C4B0000D469847042806D16B88102B0FD0732B9C
:10C4C00020D000201CE0D6F8EC0003681B689847D9
:10C4D0000328F6D194F89031062BF2D1ECE705F160
:10C4E00008010FC902ACDFED0B0A84E80F0000233E
:10C4F00009480093B0EE600A1A46214603F0C2F9DB
:10C5000006B070BD20462946FFF7BAFF0120F7E7C5
:10C51000805C002000000000FC80002038B5D1F8CD
:10C52000093007EE903AF5EEC07AF1EE10FA0546C2
:10C530000C4605DD0B7A022B03D01ED9032B0ED03F
:10C5400038BD154B9FED150AD3F8280D27EE800A4C
:10C550007CF036FDD4F80930C5F8D031F0E70E4B49
:10C560009FED0E0AD3F8280D27EE800A7CF038FDE7
:10C57000D4F80930C5F8D431E2E7074B9FED070A3C
:10C58000D3F8280D27EE800A7CF038FDD4F8093066
:10C59000C5F8CC31D4E700BF806C00200000C84251
:10C5A00038B5114D0C4605F6BC5095F8351E59F0BE
:10C5B00061F958B195F8351E05F6BC5059F062F98D
:10C5C00020B994ED040A0948F9F7DEFE94ED041A47
:10C5D000D4ED020A94ED030A95F8351E0448BDE82F
:10C5E0003840002259F086B9806C0020EC8400208D
:10C5F0003C7A0020F0B50B69214F85B005460E4608
:10C600000BB94B6953B300233B7006F108030FCB02
:10C610006C4684E80F0021462846FFF7C1FB98B915
:10C62000184B0122D3F8F41C204610F0E9FB4BF024
:10C63000FDFD022215214BF055FD2846FDF720FD9A
:10C64000114A02214DF0EEFE21462846FEF79AFCE3
:10C6500038B90E48FBF79CFE05B0F0BD3846FEF732
:10C660004FFEB38807EE903AF8EE677A0921284624
:10C67000C7ED017A05B0BDE8F040FEF7CFBA00BFC4
:10C680003C850020806C0020A82F0D08802C002005
:10C6900010B5044C237813B1034867F0E7FB20780A
:10C6A00010BD00BFF8850020307B002000780728EF
:10C6B00094BF00200120704713B5094B0191044637
:10C6C000D3F8280D03681B69984730B101992046BB
:10C6D00002B0BDE81040FEF74FBA02B010BD00BF77
:10C6E000806C002090F8983113F0010018BFC3F35C
:10C6F00080007047094A034692F8150668B192F81F
:10C700001426043A012A07D85B6A1B6893F8A10033
:10C71000431E58425841704700207047807C0020DB
:10C7200010B5044686F0BCFDD4F8B031C01AD4F878
:10C73000AC3123EAE37398424FF0000084BFC4F8A1
:10C74000AC01012010BD000010B503680446DB6D8C
:10C750009847D4F8AC3123EAE37398424FF00000D5
:10C760003CBFC4F8AC01012010BD000008B504486E
:10C770000321F9F741FDBDE808400148F9F760BE23
:10C78000EC84002070B51C4B0446D3F8280D0368D8
:10C790001B690E469847054610B90025284670BD0E
:10C7A000D4F894315BB986F07BFDB4F89231C4F8CB
:10C7B000940123B1114A537843F00103537086F07A
:10C7C0006FFDD4F89421B4F89231801A4FF47A7244
:10C7D000B0FBF2F09842E0D323B9084A537843F013
:10C7E000010353702046FDF74BFC3388044A0621B1
:10C7F0004DF018FED2E700BF806C0020DC860020E0
:10C80000542D0D0810B590F89031042B0446164BAA
:10C810000AD1D3F8280D03681B69984718B1204640
:10C82000FEF7AAFC002010BD0A79D3F8303DDFEDF9
:10C830000F6A93ED0E6A07EE902A0A7E920748BFB0
:10C840009FED0B7AF8EE677A48BF67EE877A86EE3F
:10C85000267AB0EEC77AB4EEE77AF1EE10FAACBF02
:10C8600001200020DFE700BF806C0020DB0FC94003
:10C870000000803B13B5094B01910446D3F8280D05
:10C8800003681B69984730B10199204602B0BDE8A2
:10C890001040FEF771B902B010BD00BF806C0020DF
:10C8A00010B5044686F0FCFCD4F8A831C01AD4F8C0
:10C8B000A43198424FF0000084BFC4F8A4010120C5
:10C8C00010BD000038B505460C4686F0E9FCD5F8E9
:10C8D000C831C01A23894FF47A725343984294BFE7
:10C8E0000020012038BD0000C368186808B190F826
:10C8F000B808704710B5012104460A4805F00EF843
:10C9000028B120460321BDE81040FEF787B949F061
:10C9100099FFBDE8104040F26B124FF4801149F0CE
:10C9200049BF00BF5882002090F89031022B04D0FC
:10C93000032B04D1034804F0C1BF0120704700203D
:10C94000704700BF5882002038B50C4BD3F8885C84
:10C9500090F89031032B044605F004050AD10848ED
:10C9600004F0C4FF94F8903135B110B9023B58423D
:10C97000584138BD0020F5E70120FAE7804C00203F
:10C980005882002010B50F4A137843F080031370CB
:10C990000D4B93F9E020002A044609DBFEF73AFA32
:10C9A00070B920460822BDE810400921FDF73ABAC7
:10C9B000BDE8104001220E21A3F50270F5F712BB6D
:10C9C00010BD00BFDC860020805C0020F8B5D0F8E8
:10C9D000B44105465CB1012C1AD049F033FF40F652
:10C9E00043024FF4801149F0E5FE012407E0184BA3
:10C9F000D3F8280D03681B69984710B90024204616
:10CA0000F8BD2846FEF740FB0123C5F8B431F6E730
:10CA1000104F97F9E030002BF0DA436A1B6893F867
:10CA2000A160012EEAD13C3027F058FE04460028D0
:10CA3000E5D1D7F8103193F8CB3033B132460D2120
:10CA4000A7F50270F5F7CEFAD9E73446D7E700BF6D
:10CA5000806C0020805C002038B56E4BD3F8EC2051
:10CA60006D4B9A4204460D4601D0002072E04B887F
:10CA70005E2B55D8512B0CD8103B9AB20F2A29D9CE
:10CA80002046FDF7FDFA6B88644A04214DF0CAFC8C
:10CA900059E0523B0C2BF3D801A252F823F000BF0F
:10CAA000F7CB010881CA0108B9CB0108CDCB010839
:10CAB00081CA010881CA010881CA010881CA010826
:10CAC00081CA010881CA010881CA0108FDCB010899
:10CAD000D5CB01080F2BD3D801A252F823F000BF09
:10CAE000C7CB01086BCA0108DDCB0108E3CB010805
:10CAF000F1CB0108CDCB0108B9CB010881CA0108EF
:10CB000081CA010881CA010881CA010881CA0108D5
:10CB100081CA010881CA010881CA0108E9CB01085C
:10CB2000732B74D006D8702B6ED0722BA8D1FFF760
:10CB30000BFE44E04AF2CF62934262D0A0D8B32BFE
:10CB400009D8B12B9CD92046FDF79AFA298851F0D3
:10CB500055FE012038BDBC3B9AB2132A90D8132B46
:10CB60008ED801A252F823F047CB010847CB010829
:10CB700081CA010881CA010881CA010881CA010865
:10CB800081CA010847CB010881CA010847CB0108C7
:10CB900081CA010881CA010881CA010847CB01087E
:10CBA00081CA010881CA010881CA010847CB01086E
:10CBB00081CA010847CB01082046FFF769FD00281C
:10CBC0003FF453AFBFE7FFF7DDFDF8E72046FFF77F
:10CBD000FDFEF4E71248FFF769FDF0E7FFF712FEEC
:10CBE000EDE7FFF769FDEAE7BDE83840FFF77ABDFA
:10CBF000FFF780FDE3E7FFF73DFEE0E7FFF750FEBC
:10CC0000DDE7FFF75FFEDAE7FFF78AFDD7E7FFF71B
:10CC1000ADFDD4E7805C0020087C0020DC2F0D08EF
:10CC20003C85002090F89031032B0BD0062B06D0CA
:10CC3000012B0AD1C368186803681B6818470448A9
:10CC400002F012BA034804F0C3BE0020704700BFD0
:10CC5000FC800020588200208B88012B05D00B69B6
:10CC60003BB94B692BB9CB681BB904480021F9F7D4
:10CC7000F7BE024800220831F9F714BF802C0020CB
:10CC800010B54B885E2B04460A464DD8512B05D86B
:10CC9000103B99B20F2921D900209DE0523B0C2B6B
:10CCA000FAD801A151F823F013CE010899CC01085C
:10CCB000CDCD0108E3CD010899CC010899CC01083C
:10CCC00099CC010899CC010899CC010899CC0108AC
:10CCD00099CC01081BCE010823CE01080F2BDBD80D
:10CCE00001A151F823F000BFDBCD0108EDCD010813
:10CCF000F5CD0108FDCD01080DCE0108E3CD0108F9
:10CD0000CDCD010899CC010899CC010899CC010836
:10CD100099CC010899CC010899CC010899CC01085B
:10CD200099CC010805CE0108B32B00F0848016D8F9
:10CD3000732B7DD00ED8702B77D0722BACD1D1ED68
:10CD4000027A9FED447A67EE877AFDEEE77AC0EDCE
:10CD50006B7A40E0B22B9FD1FFF7E0FB3BE0CD2B9D
:10CD60002CD8BB2B98D9BC3B112B95D801A151F8DD
:10CD700023F000BFD7CD0108D7CD010899CC010819
:10CD800099CC010899CC010899CC010899CC0108EB
:10CD90003DCE010899CC01083DCE010899CC01088F
:10CDA00099CC010899CC01083DCE010899CC010825
:10CDB00099CC010899CC010849CE01084AF2CF620A
:10CDC00093427FF469AFFFF727FB04E002F108010B
:10CDD0002046FEF745F8012010BD1146FFF72CFA5A
:10CDE000F9E711462046FFF78BF8F4E71146FFF705
:10CDF000C7F8F0E71146FFF7FDF8ECE71146FFF73B
:10CE000027F9E8E71146FFF72FF9E4E7FFF772FD8E
:10CE1000E1E71146FFF758FADDE71146FFF7C2FADE
:10CE2000D9E71146FFF7E6FBD5E7FFF715FBD2E799
:10CE3000FFF726FBCFE7FFF70FFFCCE7064802F12D
:10CE40000801F9F7C1FAC6E711462046FFF7A8FB2B
:10CE5000C1E700BF0000C842EC840020704700001A
:10CE6000704700007047000090F8280080F0010033
:10CE700070470000024B436040F605030381704792
:10CE80000001020490F85501704700000F20704720
:10CE90000020704700207047002070470020704736
:10CEA0000048704788300D080048704794300D08DE
:10CEB00008B5094800F50053D3F8DC3CB3F9083055
:10CEC00000EE103AB8EEC00AF5F726FBBDE80840C0
:10CED0000248FCF709BF00BF802C0020E07D002045
:10CEE00010B514482DED028B1C4600F5005300F5DB
:10CEF0008040B3F9A832D0F81C0D08EE103A036850
:10CF000082B09B6ECDE900219847B8EEC88AF0EE5A
:10CF1000400ADDE90021B0EE480A0748FCF734FB7F
:10CF20000548FCF743FF84ED000A02B0BDEC028B1C
:10CF300010BD00BF802C0020E07D0020F8B51C4D06
:10CF400005F5005405F580462846D6F8247DF5F70A
:10CF5000D1FAB4F9E43201EE103AB4F9E23200EE5B
:10CF6000903A434200EE103AB8EEC11AF8EEE00AE9
:10CF7000B8EEC00A384679F01FFE2846D6F8246D70
:10CF8000F5F7B8FAB4F9E43201EE103AB4F9E23246
:10CF900000EE903A434200EE103A3046B8EEC11A25
:10CFA000BDE8F840F8EEE00AB8EEC00A79F07EBEBF
:10CFB000802C002038B5144C04F5804504F57F64BE
:10CFC000D5F81C0D03689B689847692100F194020D
:10CFD00020464AF015F9D5F81C0D0368DB68984720
:10CFE0006A2100F1940220464AF00AF9D5F81C0D96
:10CFF00003681B6998476B2100F194022046BDE845
:10D0000038404AF0FDB800BF802C0020014807F0EE
:10D010000FB800BF802C00203C3084F005BD00001C
:10D0200008B549F00FFCBDE8084072224FF48011AA
:10D0300049F0C0BB08B549F005FCBDE808406622D0
:10D040004FF4801149F0B6BB08B549F0FBFBBDE8D1
:10D05000084080224FF4801149F0ACBB73B51F4DDE
:10D060000646D5F8EC0003681B6B9847044680B36E
:10D0700095F9E130002B2FDBD5F8103193F8CB4038
:10D080003CB395F8E03003F0A003202B24D1D5F871
:10D09000EC0003681B689847052808D0D5F8EC0019
:10D0A00003681B689847A0F110035C425C410C4A7E
:10D0B00002F550630193A2F500532146D3F8F43DE5
:10D0C0000093D2F8243DD2F81C2D304684F05AFC4F
:10D0D0000446204602B070BD0024FAE7805C0020C0
:10D0E000806C00203C30FFF7B9BF000038B5114D0F
:10D0F00004461148F5F7AAFE95F9E030002B14DA42
:10D10000236A93F8A120012A06D0D5F8EC0000216B
:10D11000BDE83840FCF756BB0D21A5F50270F4F7C9
:10D1200061FF95F9E030002BEFDB2046BDE8384089
:10D1300084F064BF805C0020802C00203C30FFF72E
:10D14000D5BF0000012070470120704701207047C3
:10D150000120704711207047012070470020704760
:10D16000002070470020704700487047D8310D08F4
:10D1700000487047E0310D0838B5436904461D6822
:10D1800080697DF057F925F0BFF8DFED1B0A2846CE
:10D1900079F0F8FA6369A0691D687DF04BF925F014
:10D1A000B3F8DFED150A284679F064FB6369186867
:10D1B0007AF034FD6369DFED110A18689FED0E1AED
:10D1C000B0EE600A79F0F8FC6369DFED0C0A1868CC
:10D1D0009FED091AB0EE600A79F068FD636918687E
:10D1E00079F0FEFD18B9636918687AF07DFF0023B5
:10D1F0002364012038BD00BF00803B4400007A4317
:10D2000070B52DED028B88B00446FCF7A3FA70B11F
:10D2100020460021FCF7D6FA63699FED310A1868B1
:10D2200008B0BDEC028BBDE870407BF039B8636A92
:10D23000022118687EF0B6F82A4B93F8E1305B06BD
:10D2400003D56369186879F01DFB9FED258A606935
:10D250008DED018A8DED028A8DED038A8DED048AB4
:10D2600003AA01A90068012379F076FB63691868B5
:10D270007AF0EAFD236A1D682B68DE6C6369186822
:10D2800079F0BEFE0122CDED060A8DED071A05A943
:10D290008DED050A2846B0EE480AB0476369B0EE46
:10D2A000480A186879F00EFD636918687BF06AF81F
:10D2B000236C8BB185F0F4FFE36BC01A236C9842AA
:10D2C0000AD309480C220521FCF7BAFB20B906480D
:10D2D0000C220221FCF7B4FB08B0BDEC028B70BD40
:10D2E00000000000805C0020802C002038B504463F
:10D2F0000D4685F0D5FFC4E90F0538BD07207047FE
:10D3000001207047002070470020704701207047BF
:10D310000048704778320D080048704780320D0889
:10D3200070B52DED028B0025C36880F83C501B685A
:10D33000DFED488AD3ED0A0A42699FED478A93EDF3
:10D34000060AF4EEE80A0446F1EE10FA88B0106816
:10D35000B8BFF0EE480A79F015FAE36862691B6815
:10D360001068D3ED0A0A93ED060AF4EEE80AF1EE2E
:10D3700010FAB8BFF0EE480A79F07CFA63692046EB
:10D380001E68FCF781FE6368B3F93820B3F93630C4
:10D3900000EE903A434201EE102A00EE103AB8EE49
:10D3A000C11AF8EEE00AB8EEC00A304679F004FC83
:10D3B000636920461E68FCF767FE6368274CB3F973
:10D3C0003820B3F9363000EE903A434200EE103A7E
:10D3D00001EE102A3046B8EEC11AF8EEE00AB8EEB7
:10D3E000C00A79F063FCD4F8300D7BF0E7FAD4F88A
:10D3F000306D338B1B0723D504A80FF0FBFC09F01D
:10D400002BFE9FED170A044606F11C0024F07EFB5C
:10D4100001AA04A920468DED010ACDED020A8DED89
:10D42000031A09F0E7FD80B10322294604A80FF092
:10D43000E7FC0C4B186804AA90F8791058F076FBBA
:10D4400009480821F8F7D8FE012008B0BDEC028B8E
:10D4500070BD00BF0000003400007A43806C0020E3
:10D460000AD7233C6C900020EC84002030B52DEDD1
:10D47000048BC3689FED898A1B684269D3ED0A7AE1
:10D48000DFED870A93ED060AF4EEC87AF1EE10FAA2
:10D490000446A8BFF0EE670A106889B079F072F907
:10D4A000636920461D68FCF7EFFD6368B3F9382017
:10D4B000B3F9363000EE903A434200EE103A01EEF6
:10D4C000102A2846774DB8EEC11AF8EEE00AB8EEF9
:10D4D000C00A79F071FBD5F8300D7BF0B1FBA5F5F2
:10D4E000805393F80531D90747D4D5F8303D1A8BCE
:10D4F000D20742D593ED0A9AB4EEC89AF1EE10FA2B
:10D50000B8BF93ED049AE36A186855F091FCD5F81A
:10D51000283DD3ED067AA36B20EE270AD3ED007ADF
:10D52000F0EE498AE0EE278AB0EE490AF5EEC08AAD
:10D53000F1EE10FAD8BFDFED5C8AF0EE680A20F059
:10D54000ADFF28B9D5F8300DB0EE680A7BF0F6F8DB
:10D55000636893F95130272B0FD0A36A186855F0F0
:10D5600067FCF0EEC07AF4EEC87AF1EE10FAB0EE95
:10D57000407A20D5002384F83C30236B1B68B3F934
:10D58000083000EE103A2046B8EEC00AFCF73EFC28
:10D590002046FCF7A9FB2046B0EE408AFCF7DAF8FB
:10D5A000002848D00021204609B0BDEC048BBDE81E
:10D5B0003040FCF707B9D5F8303D9FED3C0AD3ED7C
:10D5C0000F7AD3ED0B6AA36B27EE800AF4EEC86ADC
:10D5D000D3ED007AF1EE10FA67EE277A10DB9FEDBB
:10D5E000341ADFED310A552037EE800A21F05AF85F
:10D5F000012384F83C30D5F8300D7BF08FF8BCE780
:10D600009FED2C7AF4EEC76AF1EE10FA05D89FED83
:10D61000261ADFED290A5920E6E7F0EEE66AF4EE75
:10D62000C86AF1EE10FAE3D594F83C30002B08BF3D
:10D63000B0EE670ADCE7636A022118687DF0B2FE8B
:10D640001E4806F0ADFBB0EE480AD5F8300D7BF071
:10D65000F9F901461A48FAF789FD636918687AF002
:10D6600091FE236A1D686369186879F0C9FC05ACEE
:10D67000204614498DED020ACDED030A8DED041A02
:10D68000F8F7B0FF079B009394E80C0002A9284626
:10D6900076F082FD09B0BDEC048B30BD0000003493
:10D6A00000007A43806C002000000000E02E6542FC
:10D6B0000000B442000000B40000B4C2005A0020D0
:10D6C000802C0020EC84002008B5064BD3F8303DB8
:10D6D000D868243023F066FFFCEEC07A17EE900A7B
:10D6E00008BD00BF806C0020024BD3F8303DD868E5
:10D6F00079F030BD806C00200B207047012070470E
:10D700000020704701207047002070470048704794
:10D7100018330D080048704720330D08012070476A
:10D7200008B5DFED237AF4EEE70AF1EE10FA2DEDFD
:10D73000028BF0EE408AB0EE608A35DDDFED1D7AB7
:10D74000F4EEE70AF1EE10FA2ED5F6EE007A70EE5E
:10D75000E77ADFED196A9FED190ADFED190AF0EE9D
:10D76000E77A87EEA67A8720B7EE001A30EE470AEE
:10D7700020F098FFDFED137A9FED131ADFED130A07
:10D7800020EE270A8A2020EE280A20F08BFF30EEB8
:10D79000080ABDEC028BDFED0A0ABDE808408D20C7
:10D7A000B7EE001A20F07EBF9FED050AEFE700BF3D
:10D7B000AC1C5A3ED578493F8FC2753E9A99993F25
:10D7C00000000000FAEDEBBA9A99993E9A9999BE39
:10D7D00030B52DED048B7D4BB3F9A83200EE903AB5
:10D7E000F8EEE00A83B0044601AA6946B0EE600A8A
:10D7F000FBF7CAFEA0697CF01DFEE369D0ED008A4C
:10D80000D3ED946AD3ED977A90ED016AA3689FED0A
:10D81000701ADFED700A27EEE80A68EEA68A03F6B2
:10D820003813E6EE278A05463B20DFED6B7AB0EE33
:10D83000E87AB4EEE77AF1EE10FA58BFB0EE677A04
:10D84000DFED667AC7EE275AF7EE007A77EEE57AD3
:10D850009DED007A67EE877A93ED007A67EE877A1E
:10D860009FED5F7AA6EE260A87EE879A20F01AFFD0
:10D870003C209FED571ADFED570AB0EE408AB0EE1C
:10D88000680A20F00FFF626B564B1268DFED567A84
:10D89000B2F90820D3ED006A9FED541ADFED540A67
:10D8A00007EE102AB8EEC77AF0EE408A27EE277A04
:10D8B000DFED507AA6EEA77A4520F4EE007AA7EEC7
:10D8C000678ABAEE000A28EE000A83ED007A8DED31
:10D8D000000A20F0E7FEDDED017A9FED477A474B25
:10D8E0008DED000AF0EEE77AF4EEC77AF1EE10FA69
:10D8F00051D593ED007ADFED427A77EE277AB2EEDA
:10D90000007AF4EEC77AF1EE10FA58BFF0EE477ADB
:10D91000C3ED007A67EEA87ACDED017A636A1868E4
:10D9200090F8CB10002939D17DF03CFD636A1B686B
:10D9300093F8A110012939D0032940D039B9236ABD
:10D94000186877F011F9236A186876F05DFB236A8E
:10D95000DDED010A18689DED000A0368B0EE491A72
:10D96000DB6A9847204695ED028AFCF709F82046C5
:10D97000F0EE400AB0EE480AFFF7D2FE236A626872
:10D980001868D2ED020A036801215B6E984703B064
:10D99000BDEC048B30BD00221A60BFE7194B93F930
:10D9A000E130002BB4BF01210221BDE7236A1868D2
:10D9B00077F0DAF8236A186876F03CFBC7E7D97984
:10D9C0000029C4D12046FCF755FBC0E7804C00205D
:10D9D00000000C4400000CC40000FA4400409C45C8
:10D9E00000003442588500200AD7233D00A08C4512
:10D9F00000A08CC58FC2753F000000345C850020FC
:10DA00008FC2F53C805C00200E20704700207047DC
:10DA100000207047002070470020704700207047AA
:10DA200000487047B8330D0800487047B8330D08F8
:10DA300070B52DED028B436A1B6893F8CB3004461A
:10DA4000FBB9052384F848302046FBF799FF636A49
:10DA500002211868B0EE408A7DF0A4FC94F95030A1
:10DA6000E2696BB3D2F8F8515D4394F84820052A77
:10DA70004FD8DFE812F02B005F008400B100DF0018
:10DA80001E01836A1B68B3F90830002BB8BF5B42E4
:10DA90009BB2B3F57A6FD4D2C36A1B68B3F908306E
:10DAA000002BB8BF5B429BB2B3F57A6FC9D285F049
:10DAB000F7FBE36CC01A40F6C4139842C1D8C3E721
:10DAC00094F95150D2F8FC215543CEE7226A94F9DB
:10DAD000511010689FED801A49F64042534351435C
:10DAE00000EE103A00EE901A0268F8EEE00A926B2F
:10DAF000B8EEC00A9047DFED797A41F293139D4268
:10DB000038EE278A05DD94F950308BB1012384F873
:10DB10004830236A62681868D2ED020A0368B0EEE2
:10DB2000480ABDEC028B5B6EBDE8704000211847CF
:10DB30000223ECE7226A9FED681A106849F640421A
:10DB4000534300EE103A0268B8EEC00A926BF0EE52
:10DB5000410A9047DFED627A38EE678A05F50C5589
:10DB6000B5EEC08AF1EE10FA05F1270543F2BA438B
:10DB7000D8BF9FED598A9D42CBD80423C7E7236ABB
:10DB80009FED551A186894F9513049F640425343B5
:10DB900000EE903A0268F8EEE00A926BB0EE410AAD
:10DBA0009047DFED4F7AE36938EE678AD3F8F831B2
:10DBB000B5EEC08AF1EE10FAD8BF9FED478A002B70
:10DBC000B8BF5B4242F228329342A2DD41F2941385
:10DBD0009D429EDD03239AE7236A9FED3F1A186852
:10DBE00094F9513049F64042534300EE903A0268AE
:10DBF000F8EEE00A926BB0EE410A9047DFED387A1A
:10DC0000E36938EE678AD3F8F831B5EEC08A03F5D8
:10DC10000C53F1EE10FA03F1270344F24E62D8BF21
:10DC20009FED2D8A93423FF674AF2E4B9D42FFF637
:10DC300070AFA2E7236A94ED111A1868D4ED100AA8
:10DC4000036894ED0F0A1B6B00219847DFED237AE0
:10DC500094F95020E36938EE278A1AB393ED7E7A5F
:10DC6000D4ED0F7AB8EEC77A77EEC77A9FED1E7AB9
:10DC7000F0EEE77AF4EEC77AF1EE10FA3FF649AF2C
:10DC80000D2294F849101948FBF7DAFE024618B93C
:10DC900001461648FBF7D4FE4AF0C8FA16214AF0AE
:10DCA00001FA36E793ED7F7AD4ED107AB8EEC77AB1
:10DCB000DAE70D2294F849100C48FBF7C1FE024642
:10DCC00018B901460948FBF7BBFE4AF0AFFA022239
:10DCD0000D214AF007FA1CE700000000CDCC4C3EB5
:10DCE0008FC2753E6DEEFFFF0000FA43802C0020CE
:10DCF00073B5474D0446D5F8EC0003685B6B984755
:10DD000018B90026304602B070BD95F9E130002BFD
:10DD10005FDBA36A1B68B3F90830002BB8BF5B4216
:10DD20009BB2B3F57A6FECD2636A1B6893F8CB6051
:10DD3000002EE6D095F9E030002BE2DBD5F8EC00C0
:10DD400003681B689847002584F8490084F8485008
:10DD500085F0A6FAE36AE064A4F850501B68B3F9B2
:10DD60000830B3F5967F43DD012384F851304AF043
:10DD70005DFA15214AF096F9264BB3F9A83201EE67
:10DD8000103AE369B8EEC11A93ED7E0A8DED011ADF
:10DD9000F1EE410A5320B8EEC00ACDED000A20F0A2
:10DDA00081FCE36984ED0F0A93ED7F0A9DED011A72
:10DDB000DDED000AB8EEC00A542020F073FCE369E0
:10DDC00084ED100AD3ED807AF8EEE77AC4ED117A8B
:10DDD00098E7D5F8EC0003681B689847012890D0B5
:10DDE000D5F8EC0003681B689847002891D188E7B4
:10DDF00013F5967F01DAFF23B7E7A36A1B68B3F92F
:10DE00000830002BACBF0123FF2384F85030AEE76D
:10DE1000805C0020804C0020162070470020704756
:10DE200000207047012070470020704781F00100FA
:10DE300070470000012070470048704750340D08BB
:10DE40000048704720150D0803681BB1007900F0E9
:10DE50000100704718467047F0B5494D95F9356E89
:10DE600085B00446A5F50055002E00F08580454894
:10DE7000FFF7EAFF064600287ED0636920461F6848
:10DE8000FCF702F96368B3F93820B3F9363000EED5
:10DE9000903A434201EE102A00EE103AB8EEC11A51
:10DEA000F8EEE00AB8EEC00A384678F085FE6369FD
:10DEB00020461F68FCF7E8F86368B3F93820B3F927
:10DEC000363000EE903A434200EE103A01EE102A4E
:10DED0003846B8EEC11AF8EEE00AB8EEC00A78F09B
:10DEE000E5FE05F58043D3F8240D78F079FF18B9E5
:10DEF000636918687AF0F8F8B5F9A43004F13C00C9
:10DF00001BB9B5F8A230A5F8A430B5F8A43007EED7
:10DF1000903AF8EE677A04F1980203A90027CDED54
:10DF2000037A4BF047FE04F15C00C4F8A070019046
:10DF30006DF0DEF8002384F8A530B5F9A43001981F
:10DF40001BB9B5F8A230A5F8A430B5F8A43007EE97
:10DF5000903AF8EEE77AB7EE000A80EE270A6DF005
:10DF6000EBF809487CF062FAC4F8C870DFED077A74
:10DF700020EE270A84ED310A304605B0F0BD00BF1F
:10DF8000804C0020B05A0020807900200AD7233C22
:10DF900010B50446FBF7BCF92046154B40F83C3B56
:10DFA0004BF094FD134B2365134B9FED142A9FED0B
:10DFB000141ADFED140A9FED140A6365F1EE041ADA
:10DFC00004F15C006DF0CEF8002320460F49C4F840
:10DFD000A830C4F8AC30C4F8B030C4F8B430C4F8D9
:10DFE000B830C4F8BC3042F0E9FC204610BD00BF98
:10DFF00058350D08CDCCCC3D000040400AD7233B1E
:10E0000000803B459A99993ECDCC4C3EF0340D08AA
:10E010002DE9F0432DED028B9BB0914604460D4651
:10E0200085F03EF9B8499FEDB98A0646A1F108008E
:10E0300023F0EAF994ED161ACDED110A7E20F1EEE7
:10E04000410A8DED100A20F02DFB94ED161A8DED8E
:10E05000100AF1EE410A7F209DED110A20F022FB0B
:10E0600010A904F13C008DED110A4BF0C1FDA84848
:10E07000CDED130A8DED120A7CF0D8F9D4ED327A89
:10E08000D4ED140A94ED151AE0EE087A892004F113
:10E090005C074FF00008B0EE670A20F003FB12A8FF
:10E0A00023F0FEF99B4812A909F028FA14A9384672
:10E0B0008DED140ACDED150A6CF0FAFE3846CDF858
:10E0C0005880CDF85C806CF037FF8DED160ACDEDF1
:10E0D000170AB9F1000F00F001810123C4F8D060E4
:10E0E00084F8CC308C4E04F1A80116A823F0B4F9C2
:10E0F000B6F9A83200EE103A16A8B8EEC00A23F01E
:10E10000CFF916A9A6F5556009F0E4F918A9284633
:10E110008DED180ACDED190A23F09EF9B6F9A83253
:10E1200095ED007A07EE903AF8EEE77AB0EEC77A0E
:10E13000B4EEE77AF1EE10FA00F3CE8095ED017AB5
:10E14000B0EEC77AF4EEC77AF1EE10FA4CBF0123B5
:10E15000002384F8A530B6F9A83295ED000A5A429A
:10E1600007EE903A00EE902AB8EEE71AF8EEE00AD1
:10E17000CA2020F097FA85ED000AB6F9A83295ED8D
:10E18000010A5A4200EE902A07EE903AF8EEE00AB1
:10E19000B8EEE71ACB2020F085FA85ED010A94F855
:10E1A000A4305A1C84F8A4201422B3FBF2F102FB21
:10E1B0001133DBB2002B34D14AF038F8064685F033
:10E1C00077F88046D4F8AC000F46F2F79DF9CDE918
:10E1D0000E01D4F8A800F2F797F9CDE90C01D4F8B4
:10E1E000A000F2F791F9CDE90A016868F2F78CF91D
:10E1F000CDE908012868F2F787F9CDE906011398FF
:10E20000F2F782F9CDE904011298F2F77DF9CDE930
:10E210000087CDE90201414B414A4249304649F06D
:10E220007BFD1BB0BDEC028BBDE8F08312A823F090
:10E23000B9F9DFED3D7AB4EEE70AF1EE10FA57D402
:10E2400094F8CC3063B956E038466CF0D5FE94F8BB
:10E25000CC3084ED2A0AC4ED2B0A002B3FF442AFE8
:10E26000DFED325ADFED324A9FED324ADFED323ACE
:10E2700012AA2B4605F10801B2EE0E5AB7EE003A8B
:10E28000B2EC016A94F99D00B0EEC67A67EE256A99
:10E2900007EE900A76EE842AF8EEE77AB0EE647A1A
:10E2A000A7EE857AC3EEA27A27EE087A77EE837A14
:10E2B00027EE267AB5EEC06A67EE877AF1EE10FA9D
:10E2C00048BFF1EE677AE3EC017A9942D8D1CDF8F4
:10E2D0005C80CDF8588005E701233AE794F8CC300C
:10E2E0004BB1D4F8D00040F6B833361A9E429DD9CF
:10E2F000002384F8CC3094F8A530002BA4D1384604
:10E300006CF0E0FEA3E700BFDC5A00200AD7233CF4
:10E3100080790020303F0020804C0020F4FF0C0862
:10E320005C340D0820150D089A99993E0000C842EA
:10E330000000BE42000070420000FA432DE9F04F99
:10E340002DED048B0446A5B0BD487CF06FF8BD4BA5
:10E35000DFEDBD7A1B68DB6A93F89C3060EE278A9C
:10E3600033B9F1EE687AC4ED327AC4ED318A47E010
:10E37000B64D05F54053D3F8103193F8A090B9F19C
:10E38000020FEED184F08CFF05F58043D3F8343DC5
:10E39000C01A40F2DB539842E3D99FEDAD8A95F85D
:10E3A000DB1B8DED218A18AB21AA05F6C8008DED87
:10E3B000228A8DED238A1EF09DFC08B3A54821A971
:10E3C00021F024FAD4ED2C7A8DED210A37EE800A63
:10E3D000D4ED2D7ACDED220A77EEA00A9E4884ED89
:10E3E0002C0AC4ED2D0A8DED231AFFF72DFD60B91F
:10E3F00084F056FF84ED2D8AC4F8C00084ED2C8A89
:10E4000025B0BDEC048BBDE8F08F05F5005BD4F8BA
:10E41000C020DBF8643E42B9C4F8C03084ED2D8AD8
:10E4200084ED2C8A84ED328AEAE79A42E8D08B4860
